:020000040800F2
:10000000F0B601209D010008895700088D480008BE
:10001000F1500008B9160008BD8700080000000074
:10002000000000000000000000000000957B0008B8
:10003000551E0008000000000B020008017D0008AA
:10004000B7010008B7010008B7010008B7010008B0
:10005000B7010008B7010008B7010008B7010008A0
:10006000B7010008B7010008B7010008B701000890
:10007000B7010008B7010008B7010008B701000880
:10008000B7010008B7010008B7010008B701000870
:10009000B7010008B7010008B7010008B701000860
:1000A000B7010008B7010008B7010008B701000850
:1000B000B7010008B7010008B7010008B701000840
:1000C000B7010008B7010008B7010008B701000830
:1000D000B7010008B7010008B70100088D7D0008CE
:1000E000B7010008B7010008B7010008B701000810
:1000F000B7010008B7010008B7010008B701000800
:10010000B7010008B7010008B7010008B7010008EF
:10011000B7010008B7010008B7010008B7010008DF
:10012000B7010008B7010008B7010008B7010008CF
:10013000B701000885250008B7010008B7010008CD
:10014000B7010008B7010008B7010008B7010008AF
:10015000C1170008B7010008B7010008957D000825
:10016000B7010008B7010008B7010008B70100088F
:10017000B7010008B7010008B7010008B70100087F
:10018000B7010008DFF810D001F070F80048004710
:10019000D1380108AFF30080F0B60120064880474F
:1001A00006480047FEE7FEE7FEE7FEE7FEE7FEE75C
:1001B000FEE7FEE7FEE7FEE7257D00088501000873
:1001C000EFF3108072B6704780F3108870471F48B5
:1001D0004FF0FF010170002080F309881C4801687E
:1001E00081F308881B48012101701B484FF08051A2
:1001F000016062B6FEE718484FF080510160704719
:1002000015484FF080510160704772B6EFF30980D6
:1002100028B1203880E8F00F10490968086000B55F
:100220000F4880475DF804EB0E480F490A780270CA
:100230000A480E490A680260106890E8F00F203002
:1002400080F309884EF0040E62B6704722ED00E09C
:10025000D80000209D00002004ED00E0A400002054
:10026000216700089600002097000020AC000020C5
:100270002DE9F05F0546002092469B4688460646DB
:10028000814640241BE0284641464746224600F06E
:100290000CFE53465A46C01A914110D311461846D7
:1002A000224600F0F3FD2D1A67EB01084F46224667
:1002B0000120002100F0EAFD17EB00094E41201E4D
:1002C000A4F10104DFDC484631462A464346BDE836
:1002D000F09FA0F14101192900D82030704740EA71
:1002E00001039B0703D009E008C9121F08C0042AB4
:1002F000FAD203E011F8013B00F8013B521EF9D29B
:100300007047D2B201E000F8012B491EFBD27047C2
:100310000022F6E710B513460A4604461946FFF7D1
:10032000F0FF204610BD421E12F8013F002BFBD10A
:1003300011F8013B02F8013B002BF9D1704730B5B1
:1003400005462A460B4612F8010B13F8014B08B17B
:10035000A042F8D01CB1002802D06D1CF1E728465D
:1003600030BD421C10F8011B0029FBD1801A7047D8
:1003700010B5002200E0521C835C8C5CA34201D1CA
:10038000002BF8D1D8B2E1B2401A10BD30B5044606
:100390000020034600E05B1C934203D2E05CCD5C8E
:1003A000401BF8D030BD034611F8012B00F8012B9B
:1003B000002AF9D11846704730B50546002003469B
:1003C00000E05B1C934205D2EC5CC85C201A01D1B2
:1003D000002CF6D130BD00000FB400B58DB010A9CF
:1003E00009900B9000914FF0FF300A9000200C9084
:1003F00005480690054807906A4609A80F9900F03D
:1004000099FD0DB05DF814FB510F00086F0F000847
:100410002DE9FF5F1D464FF0FF3BD5E901469146B0
:100420005F464FF00008A9697F1C01988847296A38
:10043000824688470028F6D1BAF1FF3F0CD024F459
:10044000C064002E19DD600614D5BAF12B0F09D057
:10045000BAF12D0F0ED103E0584604B0BDE8F09F6D
:1004600044F48064A9697F1C01988847761E8246FF
:10047000002E02DDBAF1300F03D0B9F1000F26D003
:1004800032E0A969761E44F400747F1C0198884705
:100490008246002E05DDBAF1780F06D0BAF1580F6A
:1004A00003D0B9F1000F10D01EE0B9F1000F02D057
:1004B000B9F1100F18D1A969761E24F400747F1CBD
:1004C000019888478246102002E0082000E00A20B8
:1004D000814609E008FB0908A969761E44F4007406
:1004E0007F1C019888478246002E05DD494650460C
:1004F00000F00BFD0028EDDAE96901988847A005B6
:1005000002D46FF00100A8E7E00725D1600613D5FB
:10051000600502D5C8F1000000E0404629680A1DC8
:100520002A600968220501D5087015E0220701D567
:10053000088011E008600FE02868011D296000684C
:10054000210502D580F8008006E0210702D5A0F839
:10055000008001E0C0F8008038467EE72DE9FF5FAB
:10056000D2E901A74FF00008916999461446DDF8D9
:1005700038B0464601988847054659EA0B0005D031
:1005800009E0A169761C019888470546216A28463A
:1005900088470028F5D1681C03D05FEACA7005D0EF
:1005A00015E04FF0FF3004B0BDE8F09F2068011D5A
:1005B0002160D0F800800AE05FEACA7001D108F833
:1005C000015BA169761C7F1E019888470546002FB4
:1005D0001ADD681C18D0B9F1000F0DD0E81705EB33
:1005E000D060421120F01F0059F822102A1A012071
:1005F00090400142E0D107E0BBF1000FDCD1216A5D
:10060000284688470028D7D0E16901988847BBF180
:10061000000F07D1002E05DD5FEACA7002D100216C
:1006200088F80010A068B84203DDBBF1000F03D0CA
:1006300017B16FF00100B6E73046B4E72DE9FF4F80
:10064000087883B09946FF2805D0491C2D2804D08E
:100650000024002008E000200BE00124F9E700EB73
:10066000800003EB4000491C0B78FF2BF7D104B14D
:10067000404200230293147819461D462D2C01D0C8
:100680002B2C04D1521C2D2C13D000240294AA46EA
:100690001478FF2C0FD00A25A3FB057801FB0581F8
:1006A0004FF0000C03FB0C11521CE3194AEB010143
:1006B000EEE70124EAE7814453EA010002D019F58C
:1006C000C87F06DA03980021C0E9001107B0BDE831
:1006D000F08F0025AE4E2F46DFF8B882184600F0A6
:1006E000A0FDCDE90001B9F1000002DAC9F1000472
:1006F00000E004460023A74A1AEB030B42EB045A1E
:1007000012E0E00707D02A4633463846414600F05B
:1007100024FA074688462A4633461046194600F012
:100720001CFA05460E466410002CEAD1DDE90001F2
:10073000B9F1000F5A46534606DA00F080FA3A46FD
:10074000434600F07CFA05E000F007FA3A464346DB
:1007500000F003FA029A0AB181F00041039AC2E95B
:100760000001B3E72DE9FF4F1F468DB0D7E90146E1
:100770004FF0FF382E2045464FF000090B90B96925
:100780006D1C0E988847396A824688470028F6D142
:10079000BAF1FF3F0AD024F4D064002E11DDBAF183
:1007A0002B0F08D0BAF12D0F0BD102E0404611B04B
:1007B0008DE744F48064B9696D1C0E9888478246C1
:1007C000761E6946600501D52D2000E02B208DF8AE
:1007D000000001F1010B0DF1200809E0B9696D1C61
:1007E0000E98884782460F9844F40074761E056080
:1007F000002E02DDBAF1300FF0D00B998A453ED1C0
:1008000044F0800406E00F99681CA9F1010944F442
:1008100000740860B9696D1C761E0E988847824680
:100820003028F0D02BE00B998A4505D1200603D45F
:1008300044F08004761E18E0504608F065FA08B3CC
:100840000DF11301761E44F400748B4508D2AAF111
:1008500030000BF8010B200607D5A9F1010003E0D9
:10086000200602D409F101008146A00502D50F99A6
:10087000681C0860B9696D1C0E9888478246002E76
:10088000D1DC53E0002E51DDBAF1650F02D0BAF190
:10089000450F4BD1A00549D5B9696D1C24F44074AE
:1008A000761E0E9888478246002E0CDD2B2804D039
:1008B000BAF12D0F07D144F48074B9696D1C0E98FC
:1008C00088478246761EE00501D52D2100E02B21C8
:1008D00008F8011BCDF82C8021E00DF12901761ECE
:1008E00044F4007488450CD2AAF1300010F0FF00E7
:1008F00088F8000002D10B99884509D908F1010850
:1009000006E0E00501D5244801E042F20F7081467F
:10091000B9696D1C0E98884782460F980560002EB5
:1009200004DD504608F0F0F90028D6D1F9690E9898
:100930008847FF208BF8000088F800000020069010
:1009400007904B466A4608A906A8FFF777FEA00560
:1009500002D46FF001002AE714F0240F0AD0E00758
:1009600014D1DDE906123868031D3B600068C0E958
:1009700000120BE0DDE9060100F056FA0146E0073F
:1009800004D13868021D3A600068016028460EE70D
:10099000000014400000F03FF1D8FFFF2DE9F047C0
:1009A00091460F4680460446002614F8015B2DB19F
:1009B00000F09EFA0068405DC007F6D12B2D02D0F2
:1009C0002D2D18D0641E4A463946204600F0E0FA24
:1009D00027B13968A14201D1C7F8008071054FF0F5
:1009E00002040BD54042002803DD07F0D7FF046066
:1009F000A007BDE8F08746F48066E4E70028F8DA4F
:100A000007F0CCFF04606FF00040F2E72DE9FE4FE5
:100A1000804681EA0300C00F0C46009021F000419F
:100A200023F00045B8EB0200A94105D2404621461B
:100A300090461C460B46024623F00040104347D028
:100A4000270DC7F30A00C3F30A510290401A019020
:100A500040286BDAC3F3130040F4801B00989246E1
:100A600020B10023D2EB030A63EB0B0B019859462C
:100A7000C0F14002504600F009FA06460D465046C5
:100A80005946019A00F021FA10EB08006141002458
:100A900087EA115284EAE7731A4340D0009A62B39E
:100AA000019A012A4FEA075215DC001B61EB020193
:100AB0004FF0004202EA0752CDE90042001C41F526
:100AC000801132462B4600F047FB03B0BDE8F08FA3
:100AD00040462146F9E7001B61EB0201001C41F58D
:100AE000801300185B412018A2F5001747EB0301A3
:100AF00040EAD570B6196D4111E06D084FEA36062F
:100B000045EAC0754FEA0752001B61EB0201001C69
:100B100041F5801149084FEA300000195141324631
:100B20002B4603B0BDE8F04F00F007BB0098012250
:100B300040000023D0EB020263EBE07300982146F3
:100B40004FEAE074B8EB000061EB0401E9E783F0E1
:100B500000435BE781F0004158E72DE9FE4F81EA51
:100B6000030404F0004421F0004100944FF0000B16
:100B700023F0004350EA01045ED052EA03045BD044
:100B8000C3F30A54C1F30A552C44A4F2F33401947C
:100B9000A0FB0254C1F3130141F48011C3F313030A
:100BA00043F4801301FB024400FB034E840A970ABE
:100BB00044EA815447EA8357A4FB076802958D0AEB
:100BC00005FB07854FEA932C04FB0C542705029D77
:100BD0004FEA065847EA1637B5EB08056EEB070CE7
:100BE000870E920E47EA811742EA8312A7FB0201A1
:100BF000B6EB0B0164EB00042B0D43EA0C335E18DB
:100C000044EB1C50DA465146E7FB0201C5F31304DE
:100C10004FEA0B3343EA14534FEA0432019C43EA90
:100C20000603A4F10C040294009CCDE900B400F08A
:100C300093FA03B0BDE8F08F00200146F9E72DE9F3
:100C4000F04D81EA030404F0004B21F00045144606
:100C50004FF0000A23F0004150EA050220D054EA88
:100C600001021DD0C5F30A570246C5F31303C1F3B1
:100C70001300C1F30A5640F4801543F48013A7EB28
:100C80000608101BD64608F2FD3873EB050002D3A8
:100C900008F1010801E092185B41B8F1000F03DA96
:100CA00000200146BDE8F08D00204FF4801106467B
:100CB00084460EE0171B73EB050705D3121B63EB8D
:100CC000050306434CEA010C49084FEA300092182C
:100CD0005B4150EA0107EDD152EA030012D082EAEB
:100CE000040083EA0501084305D0101BAB4106D27E
:100CF0000122002306E000224FF0004302E06FF0E3
:100D0000010253101AEB06004CEB085110EB0A00DD
:100D100041EB0B01BDE8F04D00F00FBA9623002225
:100D2000114600F0DCB90EB5C10F80EAE07008444E
:100D3000CA07002140F233438DE80E000A460B46F5
:100D400000F00AFA03B000BD0EB540F23341029143
:100D50000021CDE900110A460B4600F0FDF903B071
:100D600000BD70B5C1F30A5201F000450024C1F383
:100D7000130140F2FF3341F480119A4201DA00205E
:100D800070BD40F233439A42A2F2334203DC524236
:100D900000F08BF800E090402C43F1D0404270BD51
:100DA00000F0004230F000400AD0C10D01F5607142
:100DB000C0F3160042EA0151C208400711437047D0
:100DC000002001467047000030B5041E71F1000498
:100DD00004DB4FF00044404264EB0101141E73F148
:100DE000000405DB1C464FF00043524263EB040352
:100DF0008B4208BF824230BD30B5041E71F1000441
:100E000004DB4FF00044404264EB0101141E73F117
:100E1000000405DB1C464FF00043524263EB040321
:100E2000994208BF904230BD01F0004330B421F038
:100E3000004150EA010206D00A0DA2F56072C1F32A
:100E40001301002A02DC30BC00207047440F44EA42
:100E5000C104C100E01830BC00EBC25000F036B94C
:100E600030B50B46014600202022012409E021FA7A
:100E700002F59D4205D303FA02F5491B04FA02F577
:100E80002844151EA2F10102F1DC30BD202A04DB4A
:100E9000203A00FA02F1002070479140C2F120038D
:100EA00020FA03F3194390407047202A04DB203ACC
:100EB00021FA02F00021704721FA02F3D040C2F17A
:100EC00020029140084319467047202A06DBCB17C1
:100ED000203A41FA02F043EAE07306E041FA02F3F5
:100EE000D040C2F1200291400843194670470000EB
:100EF000004870471C8A040810B50446FFF7F8FF45
:100F00000068005D00F0010010BD3A2800D23038C2
:100F100020F02002412A01D3A2F13700884201D3F8
:100F20004FF0FF30704700000268114413780160F1
:100F300018467047D160044951610449116200218B
:100F40001161114600F0A4B9290F0008F90E00083C
:100F5000426842B1016811F8013B23B1521EC0E959
:100F60000012184670470121C160881E7047426810
:100F70005AB1C368016843B983688B4205D0491EE2
:100F8000521CC0E90012002070474FF0FF3070473C
:100F90002DE9F05F82460078002715468B460AF15E
:100FA0000104B946302801D09DB113E014F8010BBB
:100FB0000127782803D0582801D045B10AE00DB1A7
:100FC000102D07D10027102514F8010B02E0082589
:100FD00000E00A250026B0460EE005FB080005FBF0
:100FE00006F1012701EB10461FFA80F8B6F5803FA5
:100FF00000D3B94614F8010B2946FFF786FF0028F5
:10100000EBDABBF1000F05D00FB1641E00E05446CF
:10101000CBF80040B9F1000F06D007F0BFFC022169
:101020000160C81EBDE8F09F48EA0640FAE70000EC
:101030000FB4002300B589B00CA900910B996FF093
:101040000042CB601E4B06931E4B07930423CDE951
:1010500001321D4A089202466B460020FFF782FBD0
:1010600009B05DF814FB70B586B006464FF0FF304E
:101070000091CDE90101002015460C46049032464E
:10108000694604A8FFF7D4FF02460498211825B149
:1010900008B1084600E020462860049800280DD0DA
:1010A000002A02DD0098884208D0081B0094CDE990
:1010B00001043246694604A8FFF7BAFF06B070BDC6
:1010C000510F00086F0F0008F90E00080029A8BF93
:1010D0007047401C490008BF20F00100704710B461
:1010E000B0FA80FC00FA0CF050EA010404BF10BC16
:1010F000704749B1CCF1200421FA04F411FA0CF143
:1011000018BF012121430843A3EB0C01CB1D4FEA7B
:1011100000614FEA102042BF002010BC704700EB76
:10112000C35010440029A4BF10BC7047401C4900A4
:1011300008BF20F0010010BC704710B5141E73F1F9
:10114000000408DA401C41F1000192185B411A4387
:1011500001D120F0010010BD2DE9F04D92469B46D3
:1011600011B1B1FA81F202E0B0FA80F22032904679
:10117000FFF78CFE04460F4640EA0A0041EA0B01E5
:1011800053465A46084313D0114653EA010019D07A
:10119000C8F140025046FFF788FE05460E4650460D
:1011A00059464246FFF772FE084305D0012004E08D
:1011B00020463946BDE8F08D0020054346EAE0763A
:1011C0002C4337430A986305E40AA0EB0800002289
:1011D000FD0A44EA47540A3002D500200146E9E7F7
:1011E000010510196941DDE9084500196941BDE8AB
:1011F000F04DA2E770B521F0004303430CD0C1F3DA
:101200000A550024D5EB040564EB0403D617AD1A88
:10121000B34102DB0020014670BD201841EB0251B2
:1012200070BD0EB540F2334202920022CDE9002299
:101230001346FFF791FF03B000BDC1F30A52C1F39B
:10124000130140F2FF3341F480119A4202DA002088
:101250000146704740F233439A42A2F2334202DC25
:101260005242FFF722BEFFF711BE0000064C074DA9
:1012700006E0E06840F0010394E807009847103466
:10128000AC42F6D3FEF782FFF88C0408188D0408F0
:101290002DE9F34F8BB04FF0000801F10C000C4624
:1012A0004FF0010B46460DF1080A019062690121D9
:1012B00001989047051E2DD0252D2CD0216A8847F6
:1012C000C0B16269012101989047216A88470028CE
:1012D000F7D1411E62690198904700E0761CA16930
:1012E0000B988847216A88470028F7D1E1690B9855
:1012F0008847DBE7A1690B9888470746A84201D1D8
:10130000761CD3E7E1690B9888477F1C02D1B8F1BE
:10131000000F6FD047E1002762693D4639460198CA
:1013200090472A2804D1626901210198904701253C
:10133000DFF888926269012101989047A0F130019D
:101340000A290AD24F45E5DC07EB870100EB41078C
:10135000303FDFD445F01005ECE7E90601D46FF02B
:1013600000476C280AD04C2814D0682815D06A2869
:101370000DD074281CD07A281AD01DE06269012192
:10138000019890476C2802D045F0040514E045F020
:1013900002050DE045F020050AE06269012101988F
:1013A0009047682802D045F0080505E045F400653F
:1013B0006269012101989047C4E9015765283DD031
:1013C00019DC58287AD00CDC452837D004DC2528D5
:1013D00026D0412831D131E046282FD047282CD1C2
:1013E0002CE05B2877D0612828D063287CD0642843
:1013F00023D15AE0D1E06F2848D008DC66281DD000
:1014000067281BD0692821D06E2816D127E07028C4
:1014100045D0732868D0752847D078280DD14DE085
:10142000A1690B988847054625283FF469AFE16913
:101430000B9888476D1C3FF46AAFB4E023466A46B8
:101440006FF001000B99FFF78DF99FE045F0400028
:101450006060A80723464FF0000236D43EE0E8075C
:101460007FF447AF2068011D21600068290501D580
:1014700006701BE7290701D5068017E7A90703D5E2
:10148000F117C0E9006111E706600FE745F0400081
:101490006060A80723464FF0080216D41EE040F60D
:1014A0000E0125EA0100606016E045F04000606032
:1014B000A80723464FF00A0207D40FE045F040008A
:1014C0006060A80708D5234610226FF001000B9931
:1014D000AFF300805AE007E0234610226FF00100CE
:1014E0000B99FEF795FF51E04FF000094F464B4630
:1014F000632802D05B2807D041E02079C00601D4E0
:101500000120A06001273AE062690121019890471B
:101510005E2805D14FF0010962694946019890475C
:10152000216939B900210A46534643F82120491C54
:101530000829FADBB0B3216969B9C11700EBD162A0
:1015400053110AEB830122F01F02821A01200B685B
:10155000904003430B6062690121019890475D2828
:10156000E8D1B9F1000F09D00020514651F82020F0
:10157000D24341F82020401C0828F7DB02AB22466A
:1015800000976FF001000B99FEF7E8FF00280CDAD6
:10159000401C08D1BBF1000F05D04FF0FF300DB05B
:1015A000BDE8F08FFFE74046F9E7E90701D108F110
:1015B000010806444FF0000B78E60000CCCCCC0CC0
:1015C0002DE9F04D00231A461B1A8A4103DB002047
:1015D0000146BDE8F08DC1F30A52C1F3130141F495
:1015E00080154FF0000BD10702D100186D41521E3B
:1015F0000027044640F2FF11384601EB620A3E46DE
:101600008046024600204FF48011FFF74EFCC219BD
:101610007141BB1846EB0100B4EB030C75EB000CF9
:1016200004D3E41A65EB000517460E46241908F1A9
:1016300001006D4180463428E3DDF91946EB0600D0
:10164000091BA84103D24FF0FF32134601E00022EC
:1016500013461BEB070046EB0A51BDE8F04DFFF7C0
:101660006CBD70B58C1810F8015B15F0070301D143
:1016700010F8013B2A1106D110F8012B03E010F8F5
:10168000016B01F8016B5B1EF9D12B0705D4002318
:10169000521E0DD401F8013BFAE710F8013BCB1ABA
:1016A000921C03E013F8015B01F8015B521EF9D5AF
:1016B000A142D8D3002070BD00BFFEE72DE9F04362
:1016C00087B007460D4691461C46DDF8388014B1B8
:1016D000681CC6B200E02E460121880405F09AFD80
:1016E0000121042005F07CFE4FF4406001900220AF
:1016F0008DF8080000208DF80A0001208DF80B00FD
:1017000002208DF8090001A92A4802F073FD072282
:101710000B21284802F03EFE07220A21254802F04C
:1017200039FE0397092E02D14FF4805000E00020CB
:10173000ADF810000020ADF81200ADF81400012C37
:1017400002D14FF4C06004E0022C01D1600200E03D
:101750000020ADF814000C20ADF816000020ADF804
:10176000180003A9144806F0A3FE0121124806F050
:1017700093FC4021114806F031FC012240F2255132
:101780000D4806F0F5FD012240F224410A4806F01A
:10179000EFFD27208DF8000000208DF801008DF866
:1017A000020001208DF80300684603F0F5FF07B042
:1017B000BDE8F083000802400048004000100140EE
:1017C00010B50549054800F0E9F918B10249034888
:1017D00000F08CF810BD0000008800102864024062
:1017E00070B504460D46344884423AD03248183029
:1017F000844236D030483030844232D02E4848308F
:1018000084422ED02C48603084422AD02A48783036
:10181000844226D028489030844222D02648A830DE
:1018200084421ED0254884421BD02448183084426C
:1018300017D022483030844213D0204848308442A8
:101840000FD01E48603084420BD01C487830844250
:1018500007D01A489030844203D01848A8308442F8
:1018600000D104E040F2214115A008F0DBF805F0BA
:101870004050B0F1405F07D005F0405020B119480A
:10188000284008B905B104E040F222410CA008F05C
:10189000C9F80A48844202D2074E103E01E0074EC2
:1018A000103E05F0005018B10F482840F06002E0EB
:1018B0000D482840B06070BD1060024010640240C6
:1018C0002E2E5C4C69627261726965735C7372631F
:1018D0005C73746D3332663278785F646D612E6349
:1018E0000000000082F082C07D0F7D0F70B50446BD
:1018F0000D46344884423AD032481830844236D0BB
:1019000030483030844232D02E48483084422ED085
:101910002C48603084422AD02A487830844226D02D
:1019200028489030844222D02648A83084421ED0D5
:10193000254884421BD024481830844217D02248BE
:101940003030844213D02048483084420FD01E48A3
:10195000603084420BD01C487830844207D01A484B
:101960009030844203D01848A830844200D104E06B
:1019700040F2D64115A008F055F805F04050B0F1FE
:10198000405F07D005F0405020B11DB118482840F5
:1019900000B904E040F2D7410CA008F043F80A482F
:1019A000844202D2074E103E01E0074E103E05F081
:1019B000005018B10F482840F06002E00D48284060
:1019C000B06070BD10600240106402402E2E5C4C6E
:1019D00069627261726965735C7372635C73746D62
:1019E0003332663278785F646D612E6300000000E8
:1019F000820082407D0F7D0F70B504460D462C4855
:101A000084423AD02A481830844236D028483030B0
:101A1000844232D02648483084422ED02448603058
:101A200084422AD022487830844226D02048903000
:101A3000844222D01E48A83084421ED01D488442D1
:101A40001BD01C481830844217D01A4830308442CA
:101A500013D01848483084420FD016486030844272
:101A60000BD014487830844207D01248903084421A
:101A700003D01048A830844200D104E04FF4EC7148
:101A80000DA007F0CFFF0DB1012D00D104E040F211
:101A9000D91109A007F0C6FF25B1206840F0010068
:101AA000206003E0206820F00100206070BD00008D
:101AB00010600240106402402E2E5C4C696272611C
:101AC000726965735C7372635C73746D3332663212
:101AD00078785F646D612E630000000010B50446E5
:101AE000234884423AD022481830844236D02048D5
:101AF0003030844232D01E48483084422ED01C48B8
:101B0000603084422AD01A487830844226D018485F
:101B10009030844222D01648A83084421ED0154806
:101B200084421BD013481830844217D011483030FB
:101B3000844213D00F48483084420FD00D486030A3
:101B400084420BD00B487830844207D0094890304B
:101B5000844203D00748A830844200D104E040F218
:101B6000832105A007F05EFF606880B210BD000011
:101B700010600240106402402E2E5C4C696272615B
:101B8000726965735C7372635C73746D3332663251
:101B900078785F646D612E63000000002DE9F047E6
:101BA00005460C464FF000080027B94678488542A4
:101BB0003AD077481830854236D075483030854263
:101BC00032D07348483085422ED07148603085420B
:101BD0002AD06F487830854226D06D4890308542B3
:101BE00022D06B48A83085421ED06A4885421BD05F
:101BF00068481830854217D066483030854213D087
:101C00006448483085420FD06248603085420BD02E
:101C100060487830854207D05E489030854203D0D6
:101C20005C48A830854200D104E040F286415AA0C9
:101C300007F0F8FE6148844278D06148844275D04C
:101C40006048844272D0604884426FD05F488442CA
:101C50006CD05F48844269D05E48844266D05E485A
:101C6000844263D05848FC3084425FD057483F30AC
:101C700084425BD05948844258D05948844255D058
:101C80005848844252D0584884424FD057488442E2
:101C90004CD05748844249D05648844246D0564892
:101CA000844243D05548844240D0554884423DD078
:101CB000544884423AD05448844237D053488442EE
:101CC00034D05348844231D0524884422ED05248B6
:101CD00084422BD05148844228D05148844225D098
:101CE0004B48FC30844221D04A483F3084421DD0CA
:101CF0004C4884421AD04C48844217D04B48844206
:101D000014D04B48844211D04A4884420ED04A48ED
:101D100084420BD04948844208D04948844205D0C7
:101D20004848844202D04848844200D104E040F24E
:101D3000874119A007F076FE1648854202D2144E5C
:101D4000103E01E0134E103E4048204030B11E20AE
:101D500000EAD427286800EA070902E0686900F071
:101D6000800904F0005008B1776800E0376838480F
:101D7000074007EA040028B1B9F1000F02D04FF084
:101D8000010801E04FF000084046BDE8F087000080
:101D900010600240106402402E2E5C4C6962726139
:101DA000726965735C7372635C73746D333266322F
:101DB00078785F646D612E63000000002080001061
:101DC00010400010082000100410001001000090C6
:101DD0000088001000440010002200100080201035
:101DE00000401010002008100010041000000190A6
:101DF00000800018004000140020001200100011A4
:101E0000000040902080002010400020082000208A
:101E100004100020010000A00088002000440020E1
:101E200000220020008020200040102000200820F8
:101E300000100420000001A00080002800400024C1
:101E40000020002200100021000040A03C0F3C0FA9
:101E50007D0F7D0F7047000030B5ADF5197D05464B
:101E60002A4616A1684606F071FD002215A10DA8AC
:101E70000DF074FC04461CB1214613A006F056FD7B
:101E800068460DF0DFFE044624B9294614A006F08A
:101E90004DFD0BE0042C04D1294616A006F046FDAA
:101EA00004E0224629461AA006F040FD002205A1C2
:101EB00010460DF053FC0DF5197D30BD303A2F253D
:101EC00073000000303A0000B9D2D4D8CEC4BCFEB2
:101ED000CFB5CDB3CAA7B0DC20282564290D0A00F0
:101EE000C9BEB3FDCEC4BCFE20257320B3C9B9A6BC
:101EF0000D0A0000C3BBD3D0B7A2CFD6CEC4BCFE60
:101F0000BBF2C4BFC2BC203A25730D0A000000001A
:101F1000C9BEB3FD2573CAA7B0DC28B4EDCEF3B4B7
:101F2000FAC2EB203D2025642920CEC4BCFED6BBDE
:101F3000B6C1BBF2C4BFC2BCB7C7BFD50D0A000053
:101F400010B500F0A5F901F07DF800F0B7FF0848E2
:101F5000007800F0010008B101F056F80EF010FC16
:101F600028B10348006840F010000149086010BD26
:101F70006400002010B504460648204008B904B1AA
:101F800004E040F2927104A007F04CFD0B4844615C
:101F900010BD00000018FEFF2E2E5C4C69627261BD
:101FA000726965735C7372635C73746D333266322D
:101FB00078375F6574682E6300000000009002406F
:101FC00070B504460D461048204008B904B104E03D
:101FD00040F243710DA007F025FD0DB1012D00D198
:101FE00004E040F2447109A007F01CFD2DB1104837
:101FF000C06920430E49C86104E00D48C069A04390
:102000000B49C86170BD00000018FEFF2E2E5C4C0D
:1020100069627261726965735C7372635C73746D1B
:102020003332663278375F6574682E6300000000D3
:102030000090024010B504460CB1012C00D104E020
:102040004FF4FF6108A007F0EDFC34B10F48806940
:1020500040F002000D49886105E00C48806920F0DD
:1020600002000A49886110BD2E2E5C4C69627261C3
:10207000726965735C7372635C73746D333266325C
:1020800078375F6574682E6300000000009002409E
:1020900070B50C4613460021124D286000BF18E0B1
:1020A00000EB01124FF00045156044F2F455556005
:1020B000C1EBC11505EB450504EB850595605D1E7B
:1020C0008D4204D900EB01151035D56000E0D060D9
:1020D000491C9942E4D3044DE860044D044E356038
:1020E00070BD0000480000200090024060C9002040
:1020F0004C00002070B504460D460DB1012D00D1F5
:1021000004E040F2666107A007F08CFC25B160682E
:1021100020F00040606003E0606840F000406060D4
:1021200070BD00002E2E5C4C69627261726965732D
:102130005C7372635C73746D3332663278375F65DB
:1021400074682E630000000010B504460CB1012C29
:1021500000D104E040F2E17108A007F063FC34B163
:102160000F48806940F400500D49886105E00C4833
:10217000806920F400500A49886110BD2E2E5C4C05
:1021800069627261726965735C7372635C73746DAA
:102190003332663278375F6574682E630000000062
:1021A0000090024030B50C46134600210F4D2860C8
:1021B00000BF15E000EB01124FF480151560C1EB74
:1021C000C11505EB450504EB850595605D1E8D4247
:1021D00004D900EB01151035D56000E0D060491C32
:1021E0009942E7D3024D286130BD00004400002031
:1021F0000090024070B505460C4644B1B4F5800F1E
:1022000005D0B4F5000F02D0B4F5400F00D104E0C2
:1022100040F2975103A007F005FC2868204328608E
:1022200070BD00002E2E5C4C69627261726965732C
:102230005C7372635C73746D3332663278375F65DA
:1022400074682E630000000010B50121480605F0F7
:102250001BF800214FF0007005F016F810BD01B515
:1022600081B0002000900198009002E00098401E8C
:10227000009000980028F9D10CBD00000348806947
:1022800040F48010014988617047000000900240CE
:102290001CB50121572004F0BDFF0121880305F082
:1022A0009FF8002005F078FC03208DF8050002203F
:1022B0008DF8040000208DF806008DF807008F20AF
:1022C00000906946364801F095FF0B220021344802
:1022D00002F060F80B220121314802F05BF80B227A
:1022E00002212F4802F056F80B2203212C4802F05D
:1022F00051F80B2207212A4802F04CF840F2035013
:1023000000906946274801F075FF0B2200212548FF
:1023100002F040F80B220121224802F03BF80B2288
:102320000821204802F036F80B220A211D4802F04D
:1023300031F83E20009069461B4801F05BFF0B22FC
:102340000121194802F026F80B220221164802F05A
:1023500021F80B220321144802F01CF80B2204215F
:10236000114802F017F80B2205210F4802F012F86D
:102370004FF4D040009069460C4801F03BFF0B221F
:1023800011460A4802F006F80B220D21074802F018
:1023900001F80B220E21054801F0FCFF1CBD0000D6
:1023A0000000024000040240000802400018024001
:1023B00070B504460025B4F1005F2AD0B4F1805F07
:1023C00027D0B4F1006F24D0B4F5803F21D0B4F50C
:1023D000004F1ED0B4F5804F1BD0B4F5005F18D06D
:1023E000B4F5806F15D0B4F5007F12D0B4F5807FBE
:1023F0000FD0802C0DD0402C0BD0202C09D0102CCD
:1024000007D0082C05D0042C03D0022C01D0012CBD
:1024100000D104E040F2FE6105A007F003FB0D4887
:102420004069204008B1012500E00025284670BD24
:102430002E2E5C4C69627261726965735C737263A3
:102440005C73746D3332663278375F6574682E63FF
:10245000000000000090024000200449096801F0DB
:10246000010109B1012000E0002070470090024006
:102470000FB5002101910291039100916FE0009945
:10248000491C00913D490968096801F40071A1B136
:102490003A490968096801F4807171B937490968D6
:1024A000374A126811600121354A12689160334938
:1024B0000968C968314A116051E030490968096802
:1024C00001F4807191B92D490968096801F400711E
:1024D00061B92B4909688968491C294A12689160C9
:1024E00026490968C968254A116038E02349096806
:1024F000234A12685160224909688968491C204AA8
:10250000126891601E4909688968012904D11B4934
:1025100009681B4A12681160184909680968C1F303
:102520000D41091F0191164909688968012905D9DA
:102530001349096809688968029103E00F4909682D
:10254000896802910D49096803910C490968C968B5
:102550000A4A116001A90EC980E80E000FBD0749A3
:102560000968096801F0004111B90099082986D36A
:1025700001A90EC980E80E0000BFEFE74800002067
:102580004C00002010B54020FFF712FF012803D1B6
:102590000548006803F03CFE4020FFF7EBFC4FF4D9
:1025A0008030FFF7E7FC10BD980100202DE9F041D5
:1025B00086B004460F464FF0000800250020059025
:1025C000F84E00902068012801D0206800B904E08E
:1025D0004FF48C71F4A007F025FA606818B16068B8
:1025E000B0F5000F00D104E040F21911EEA007F0A1
:1025F00019FAA06818B1A068B0F5800F00D104E006
:102600004FF48D71E8A007F00DFAE068D8B1E068EA
:10261000B0F5003F17D0E068B0F5802F13D0E06828
:10262000B0F5C02F0FD0E068B0F5002F0BD0E068F8
:10263000B0F5202F07D0E068B0F5402F03D0E06858
:10264000B0F5602F00D104E040F21B11D6A007F0D6
:10265000E9F9206918B12069B0F5803F00D104E0A4
:102660004FF48E71D0A007F0DDF9606918B1606990
:10267000B0F5804F00D104E040F21D11CAA007F070
:10268000D1F9A06918B1A069B0F5005F00D104E0EC
:102690004FF48F71C4A007F0C5F9E069B0F5805F11
:1026A00001D0E06900B904E040F21F11BEA007F0BC
:1026B000B9F9206AB0F5006F01D0206A00B904E0D2
:1026C0004FF49071B8A007F0ADF9606AB0F5806F73
:1026D00001D0606A00B904E040F22111B2A007F015
:1026E000A1F9A06A18B1A06AB0F5007F00D104E09A
:1026F0004FF49171ACA007F095F9E06A802801D001
:10270000E06A00B904E040F22311A7A007F08AF9BB
:10271000206B40B1206B202805D0206B402802D0D0
:10272000206B602800D104E04FF492719EA007F066
:1027300079F9606B102801D0606B00B904E040F2B9
:10274000251199A007F06EF9A06BB0F1004F01D0F0
:10275000A06B00B904E04FF4937193A007F062F905
:10276000E06BB0F5007F05D0E06BB0F5407F01D0A5
:10277000E06B00B904E040F227118BA007F052F99A
:10278000206C402805D0206C802802D0206CC02806
:1027900000D104E04FF4947183A007F043F9606C1A
:1027A00010B1606C202800D104E040F229117EA015
:1027B00007F038F9A06C10B1A06C082800D104E033
:1027C0004FF4957178A007F02DF940F20441206D87
:1027D000884207D0206D042804D0206D10B1206DF0
:1027E000102800D104E04FF496716FA007F01AF999
:1027F00040F20241606D884204D0606D022801D031
:10280000606D00B904E040F22D1167A007F00AF9ED
:10281000206EB0F5803F00D204E04FF4977162A0C3
:1028200007F000F9606E10B1606E802800D104E0FE
:1028300040F22F115CA007F0F5F8A06E40B1A06E39
:10284000102805D0A06E202802D0A06E302800D11C
:1028500004E04FF4987154A007F0E4F8E06E082803
:1028600001D0E06E00B904E040F231114EA007F053
:10287000D9F8206F042801D0206F00B904E04FF48C
:10288000997149A007F0CEF8606F022801D0606FFF
:1028900000B904E040F2331143A007F0C3F8A06F81
:1028A000B0F5803F01D0A06F00B904E04FF49A71F9
:1028B0003DA007F0B7F8E06FB0F5803F00D204E02C
:1028C00040F2351138A007F0ADF8D4F8800020B1FF
:1028D000D4F88000B0F1806F00D104E040F23711ED
:1028E00031A007F09FF8D4F88400B0F1007F02D047
:1028F000D4F8840000B904E04FF49C712AA007F0DA
:1029000091F8D4F8880020B1D4F88800B0F1807F25
:1029100000D104E040F2391123A007F083F8D4F885
:102920008C00B0F5001F02D0D4F88C0000B904E090
:102930004FF49D711CA007F075F8D4F8900010B307
:10294000D4F89000B0F5804F1DD0D4F89000B0F5C9
:10295000004F18D0D4F89000B0F5404F13D0D4F801
:102960009000B0F5803F0ED0D4F89000B0F5A03FB5
:1029700009D0D4F89000B0F5C03F04D0D4F890004E
:10298000B0F5E03F00D104E040F23B1106A007F0B3
:1029900049F8D4F89400802802D0D4F89400A8B95B
:1029A0001AE00000008793032E2E5C4C696272616E
:1029B000726965735C7372635C73746D3332663213
:1029C00078375F6574682E63000000004FF49E71D5
:1029D000AFF22C0007F026F8D4F89800402802D077
:1029E000D4F8980000B905E040F23D11AFF248007C
:1029F00007F018F8D4F89C0058B1D4F89C000828C7
:102A000007D0D4F89C00102803D0D4F89C001828D4
:102A100000D105E04FF49F71AFF2740007F002F8A7
:102A2000D4F8A000042802D0D4F8A00000B905E032
:102A300040F23F11AFF2900006F0F4FFD4F8A4008A
:102A4000B0F1007F02D0D4F8A40000B905E04FF443
:102A5000A071AFF2AC0006F0E5FFD4F8A800B0F525
:102A6000803F02D0D4F8A80000B905E040F241113F
:102A7000AFF2CC0006F0D6FFD4F8AC00B0F5003FC2
:102A800036D0D4F8AC00B0F5802F31D0D4F8AC00FB
:102A9000B0F5002F2CD0D4F8AC00B0F5801F27D0B3
:102AA000D4F8AC00B0F5001F22D0D4F8AC00B0F5DB
:102AB000800F1DD0D4F8AC00B0F1817F18D0D4F8CD
:102AC000AC00B0F1827F13D0D4F8AC00B0F1847FB9
:102AD0000ED0D4F8AC00B0F1887F09D0D4F8AC00A7
:102AE000B0F1907F04D0D4F8AC00B0F1A07F00D159
:102AF00005E04FF4A171AFF2501006F093FFD4F847
:102B0000B000B0F5807F36D0D4F8B000B0F5007FCB
:102B100031D0D4F8B000B0F5806F2CD0D4F8B0002C
:102B2000B0F5006F27D0D4F8B000B0F5805F22D0A8
:102B3000D4F8B000B0F5005F1DD0D4F8B000B0F10B
:102B4000012F18D0B149D4F8B000884213D0B04951
:102B5000D4F8B00088420ED0AE49D4F8B000884214
:102B600009D0AD49D4F8B000884204D0AB49D4F8BC
:102B7000B000884200D105E040F24311AFF2D81016
:102B800006F050FFD4F8B4001F2800D805E04FF439
:102B9000A271AFF2EC1006F045FFD4F8B80090B186
:102BA000D4F8B800B0F5804F0DD0D4F8B800B0F527
:102BB000004F08D0D4F8B800B0F5404F03D0D4F897
:102BC000B800022800D105E040F24511AFF22820FC
:102BD00006F028FF9248056925F01C0501A804F0BD
:102BE00039FC029E8F48864205D38F48864202D226
:102BF00045F0080511E08C48864205D38B48864293
:102C000002D245F00C0508E08848864203D3884884
:102C1000864200D201E045F00405814805614FF489
:102C200000420021384600F08DFB18B9002006B0A4
:102C3000BDE8F0817F48FFF712FB2068A0B300BF1A
:102C40000098401C00900121384600F09DFA00F0E9
:102C5000040018B9784900988842F1D37649009861
:102C6000884201D10020E2E7002000904FF480521A
:102C70000021384600F066FB08B90020D7E700BF06
:102C80000098401C00900121384600F07DFA00F0C9
:102C9000200018B9684900988842F1D36649009825
:102CA000884202D10020C2E719E0002000901021E4
:102CB000384600F069FA804608F0040018B14FF475
:102CC0000060206201E00020206208F0020010B1E4
:102CD0000020606116E04FF48040606112E0206ADD
:102CE000C0F3CF006169C1F34F0140EA0102002146
:102CF000384600F027FB08B9002098E76FF07F40C6
:102D0000FFF7ADFA464805684C480540D4E9010193
:102D10000843E16808432169084361690843A169E0
:102D20000843E1690843216A0843616A0843A16ACC
:102D30000843E16A0843216B0843616B084305437C
:102D400037480560D4E90E010843216C0843616CE3
:102D50000843A16C0843E16C0843216D0843616D91
:102D600008432F494860A06D8860E06DC860084640
:102D700085694FF641700540B4F86010606E40EA16
:102D80000140A16E0843E16E0843216F0843616F63
:102D90000843054322488561D4E91E0108432049C0
:102DA000C8612748856927480540D4E920010843C0
:102DB000D4F888100843D4F88C100843D4F8901045
:102DC0000843D4F894100843D4F898100843D4F872
:102DD0009C100843D4F8A0100843054318488561A7
:102DE000D4E929010843D4F8AC100843D4F8B01052
:102DF0000843D4F8B41040EA8100D4F8B81008436E
:102E000040F400000E490860012010E700020001B4
:102E10000004000100080001001000010020000172
:102E200000800240002D3101C00E1602008793037E
:102E300000E1F505FFFF0F00FFFF04000F8120FFF9
:102E400000900240233FDEF870B504460D462CB1D9
:102E5000082C03D0102C01D0182C00D104E04FF422
:102E60004F710CA006F0DEFD2879697940EA012651
:102E7000114820440664E8780006A97840EA014039
:102E8000697840EA0120297840EA01060A4820448E
:102E9000466470BD2E2E5C4C696272617269657306
:102EA0005C7372635C73746D3332663278375F655E
:102EB00074682E63000000000080024000B5AFB0CF
:102EC00001214FF0606004F0A5F9FFF7BDF900F0B3
:102ED000B5F900BFFFF7C0FA0128FBD0684600F043
:102EE000D7F901200090002007904FF400700A905D
:102EF00000200B900E9011901390149015904FF4A9
:102F000080600990002020904FF000702190001107
:102F1000239000202590269004202890C005299019
:102F200040122A9080012B9040122C9040002E904D
:102F300001216846FFF73AFB18B1012003490860F8
:102F400002E00020014908602FB000BD64000020AD
:102F500010B504460CB1012C00D104E040F28D21E3
:102F600008A006F05FFD34B10F48006840F004008F
:102F70000D49086005E00C48006820F004000A498B
:102F8000086010BD2E2E5C4C6962726172696573B7
:102F90005C7372635C73746D3332663278375F656D
:102FA00074682E63000000000080024010B50446E3
:102FB0000CB1012C00D104E040F2752108A006F00C
:102FC00031FD34B10F48006840F008000D49086039
:102FD00005E00C48006820F008000A49086010BDB0
:102FE0002E2E5C4C69627261726965735C737263E8
:102FF0005C73746D3332663278375F6574682E6344
:10300000000000000080024008B53D208DF800005F
:1030100002208DF8010000208DF8020001208DF8BB
:103020000300684602F0B8FB4020FEF7A3FF4FF410
:103030008030FEF79FFF01210148FEF7C1FF08BD68
:10304000400001001CB50121102004F0E3F8042029
:10305000009002208DF8050001208DF8040000206A
:103060008DF806008DF8070069460C4801F0C2F89B
:1030700004210A4801F030FB0A2016F019F8042157
:10308000064801F0D5FA0A2016F012F80421034888
:1030900001F022FB0A2016F00BF81CBD00100240C4
:1030A00070B50246002300250024354800680068FA
:1030B00000F0004008B1002070BD3148016840F2C6
:1030C000F450824208DD92FBF0F392FBF0F600FB35
:1030D000162010B15B1C00E00123012B1AD12848F7
:1030E0000068006840F04050254E36683060C2F3FA
:1030F0000C00234E3668706021480068006840F07C
:1031000000401F4E366830601D480068C0681C4E85
:10311000306028E0002422E03CB9194800680068CB
:1031200040F08050164E3668306040F2F4504860EF
:10313000581EA0420DD1086840F000500860581E8B
:10314000C0EBC01000EB4000A2EB8005C5F30C0003
:103150004860086840F000400860C968641C9C42F0
:10316000DAD3074801600748406900F0040020B145
:103170000420044E70610020706001209CE7000074
:103180004400002000900240F8B506460D46002499
:1031900000200090202E00DC04E040F692011CA0EC
:1031A00006F040FC1DB1012D01D0102D00D104E02E
:1031B00040F6930116A006F035FC1E48046904F0A1
:1031C0001C044FF4784000EAC62004434FF4F86032
:1031D00000EA8510044324F0020444F00104154879
:1031E000046100BF0098401C00901248046904F07C
:1031F000010018B1104900988842F3D30E49009895
:10320000884201D10020F8BD0A48406980B2FAE73F
:103210002E2E5C4C69627261726965735C737263B5
:103220005C73746D3332663278375F6574682E6311
:103230000000000000800240FFFF04000348006817
:1032400040F0010001490860704700000090024012
:1032500010B50120FFF7AAFEFFF710F80120FFF7D5
:1032600077FE0120FEF770FF0120FEF7E3FE10BDA0
:1032700010B50020FEF768FF0020FEF7DBFE0020FF
:10328000FFF766FEFEF7FAFF0020FFF78FFE10BD86
:1032900001210160002141608160C16001614FF442
:1032A0008041416100218161C1614FF4006101628F
:1032B000002141628162C162016341638163C16334
:1032C000402101642021416400218164C1640165C1
:1032D00041658165C1650166802141660021816685
:1032E000C166016741678167C1674FF08061C0F8BF
:1032F00080104910C0F884100021C0F888104FF4E5
:103300000011C0F88C100021C0F89010C0F8941083
:10331000C0F89810C0F89C10C0F8A0104FF00071D1
:10332000C0F8A4104912C0F8A8108901C0F8AC1068
:103330004912C0F8B0100021C0F8B410C0F8B8109D
:1033400070470000F8B506460D46174600240020D9
:103350000090202E00DC04E040F6C1011BA006F026
:1033600061FB1DB1012D01D0102D00D104E040F60C
:10337000C20116A006F056FB1D48046904F01C04A7
:103380004FF4784000EAC62004434FF4F86000EAA6
:103390008510044344F0020444F0010414484761DA
:1033A000046100BF0098401C00901148046904F0BB
:1033B000010018B10F4900988842F3D30D490098D5
:1033C000884201D10020F8BD0120FCE72E2E5C4C84
:1033D00069627261726965735C7372635C73746D48
:1033E0003332663278375F6574682E630000000000
:1033F00000800240FFFF040070B504460D46102C0B
:1034000002D0B4F5807F00D104E04FF4E8711AA037
:1034100006F008FB0DB1012D00D104E040F2D111FE
:1034200015A006F0FFFA9DB1102C08D14FF02040F6
:10343000006E40F004004FF0204108661BE0174882
:10344000006840F004004FF02041C1F8800012E015
:10345000102C08D14FF02040006E114908404FF069
:103460002041086607E00D4800680D4908404FF00C
:103470002041C1F8800070BD2E2E5C4C69627261E3
:10348000726965735C7372635C73746D3332663238
:1034900078785F66736D632E63000000800000A083
:1034A000FBFF0F002DE9F041044600250026002710
:1034B0002068102803D02068B0F5807F00D104E098
:1034C00040F2751170A006F0ADFA606810B1606846
:1034D000022800D104E04FF4BB716BA006F0A2FA01
:1034E000A06810B1A068102800D104E040F2771164
:1034F00065A006F097FAE06810B1E068402800D1B6
:1035000004E04FF4BC7160A006F08CFA206998B119
:103510002069B0F5003F0FD02069B0F5802F0BD0A7
:103520002069B0F5C02F07D02069B0F5002F03D077
:103530002069B0F5202F00D104E040F2791152A0AB
:1035400006F070FA6069FF2800D804E04FF4BD71FE
:103550004DA006F067FAA069FF2800D804E040F209
:103560007B1149A006F05EFAE0690068FF2800D8E8
:1035700004E04FF4BE7144A006F054FAE0694068DC
:10358000FF2800D804E040F27D113FA006F04AFA7F
:10359000E0698068FF2800D804E04FF4BF713AA0CA
:1035A00006F040FAE069C068FF2800D804E040F265
:1035B0007F1135A006F036FA206A0068FF2800D88F
:1035C00004E04FF4C07130A006F02CFA206A406885
:1035D000FF2800D804E040F281112BA006F022FA67
:1035E000206A8068FF2800D804E04FF4C17126A04B
:1035F00006F018FA206AC068FF2800D804E040F2FC
:10360000831121A006F00EFA606840F00800A1685E
:103610000843E168084321690843616940EA4120A1
:10362000A16940EA4135E0690068E169496840EA1A
:103630000120E169098940EA0140E169097B40EA2A
:103640000166206A0068216A496840EA0120216A0F
:10365000098940EA0140216A097B40EA0167206844
:10366000102805D14FF0204005668666C76608E041
:103670000E4805604FF02040C0F888600B480C30C1
:103680000760BDE8F08100002E2E5C4C696272611B
:10369000726965735C7372635C73746D3332663226
:1036A00078785F66736D632E63000000800000A071
:1036B0002DE9F04107460D4616469846002016496A
:1036C000087016490E70301208700D70280A0870C4
:1036D000280C0870302010490870002401E0601C9C
:1036E00084B2142CFBDB00BF40210D4800F020FF0A
:1036F0000028F9D000240AE0385D4FF0E041097855
:10370000884202D00120BDE8F081601C84B24445AB
:10371000F2DB0020F7E700000000017000000270FB
:10372000000C024010B50446602007490870A4014F
:1037300006490C70200A0870200C0870D02002493D
:10374000087000F005F810BD000001700000027064
:1037500070B54FF48034402500F010FA054603E0C0
:1037600000F00CFA0546641E402D01D0002CF7D164
:1037700004B98025284670BD00B58FB001210846E8
:1037800003F0BCFD0121182003F044FD0C220021B0
:103790003F4800F0FFFD0C2201213D4800F0FAFDFA
:1037A0000C2204213A4800F0F5FD0C22052138488E
:1037B00000F0F0FD0C220621354800F0EBFD0C2254
:1037C0000721334800F0E6FD0C220B21304800F0C1
:1037D000E1FD0C2211462E4800F0DCFD0C220721F1
:1037E0002C4800F0D7FD0C2208212A4800F0D2FD19
:1037F0000C220921274800F0CDFD0C220A21254882
:1038000000F0C8FD4DF6B3000D9002208DF8390090
:103810008DF8380000208DF83A008DF83B000DA996
:103820001B4800F0E7FC4FF4F0600D900DA919481B
:1038300000F0E0FC40200D9002208DF839000020BF
:103840008DF8380001208DF83B000DA9104800F0DC
:10385000D1FC0120009002200190029003901020E2
:1038600004900020059006904020079000030890E7
:10387000002009900A90CDF82CD0CDF830D004A8C3
:10388000FFF710FE01211020FFF7B6FD0FB000BDBD
:10389000000C02400010024070B504460D4604F0D2
:1038A000400005F04001884206D02A4621461EA06D
:1038B00005F03CF8012070BD002028490870284917
:1038C000087008700C70200A0870200C08703520F1
:1038D00022490870002601E0701CC6B2142EFBDBE2
:1038E00000BF40211F4800F023FE0028F9D08520AA
:1038F0001A49087000201A49087008700D70280ACB
:103900000870280C0870102014490870FFF720FF79
:10391000402801D10020CEE72A46214612A005F01A
:1039200005F80120C7E700004572726F72203A2047
:1039300046534D435F4E414E445F50616765436F50
:1039400070794261636B4578287372633D25642CFE
:10395000207461723D256429200D0A000000017069
:1039600000000270000C02404572726F723A2046ED
:10397000534D435F4E414E445F50616765436F70E6
:10398000794261636B2825642C202564290D0A0087
:103990002DE9F84304460D4690461F46DDF8209079
:1039A00004F0400005F04001884207D02A46214635
:1039B000284804F0BBFF0120BDE8F8830020264919
:1039C00008702649087008700C70200A0870200CD6
:1039D0000870352020490870002601E0701C86B26E
:1039E000142EFBDB00BF40211D4800F0A1FD002884
:1039F000F9D085201849087000201849087008700F
:103A00000D70280A0870280C08708520124908706B
:103A100012490F7038120870002606E018F80600E8
:103A20004FF0E0410870701C86B24E45F6DB102066
:103A300009490870FFF78CFE402801D10020BBE740
:103A40003B462A4621460748CDF8009004F06EFF19
:103A50000120B1E7448A04080000017000000270F0
:103A6000000C0240CC8A04082DE9F04105460E46C0
:103A700017461C46B4F5006F06DD214606A004F08B
:103A800055FF0120BDE8F08123463A4631462846DD
:103A900000F014F8F6E700004572726F723A2046A3
:103AA000534D435F4E414E445F52656164446174BF
:103AB0006128292025640D0A000000002DE9F0414D
:103AC00007460D46164698460020144908701449CA
:103AD0000E70301208700D70280A0870280C0870DB
:103AE00030200E490870002401E0601C84B2322CA2
:103AF000FBDB00BF40210B4800F01AFD0028F9D085
:103B0000002405E04FF0E04000783855601C84B296
:103B10004445F7DB0020BDE8F081000000000170A3
:103B200000000270000C02402DE9F04106460F46ED
:103B300015461C46402C06DD214607A004F0F6FE83
:103B40000120BDE8F08105F5006082B223463946C8
:103B50003046FFF7B3FFF4E74572726F723A2046C2
:103B6000534D435F4E414E445F52656164537061F3
:103B7000726528292025640D0A00000000207022AB
:103B8000084B1A701206117801F001020AB10120E7
:103B900006E001F04002402A01D1402000E0002070
:103BA000704700000000017010B5FF200449087044
:103BB000FFF7CEFD402801D1002010BD0120FCE719
:103BC000000001702DE9F04105460E4617461C46DF
:103BD000B4F5006F06DD214606A004F0A7FE012023
:103BE000BDE8F08123463A463146284600F014F8F5
:103BF000F6E700004572726F723A2046534D435FFC
:103C00004E414E445F57726974654461746128295E
:103C10002025640D0A0000002DE9F04106460D46FE
:103C20001746984680202749087027490F70381298
:103C300008700D70280A0870280C0870002401E034
:103C4000601C84B2142CFBDB002405E0305D4FF0D7
:103C5000E0410870601C84B24445F7DB102019492C
:103C60000870002401E0601C84B2142CFBDB00BF50
:103C70004021164800F05CFC0028F9D0FFF768FDF1
:103C8000402816D143463A4629461148FFF716FF09
:103C9000424631460E48FCF779FB40B143463A466E
:103CA00029460CA004F042FE0120BDE8F08100206E
:103CB000FBE743463A46294615A004F037FE0120AB
:103CC000F3E700000000017000000270000C0240E9
:103CD0006CD100204572726F72313A2046534D43C9
:103CE0005F4E414E445F5772697465506167652845
:103CF000706167653D25642C20616464723D2564B4
:103D00002C20636F756E743D2564290D0A00000038
:103D10004572726F72323A2046534D435F4E414EA8
:103D2000445F5772697465506167652870616765A3
:103D30003D25642C20616464723D25642C20636FF2
:103D4000756E743D2564290D0A0000002DE9F041CF
:103D500006460F4615461C46402C06DD214607A0A8
:103D600004F0E4FD0120BDE8F08105F5006082B2B9
:103D7000234639463046FFF74FFFF4E74572726F2E
:103D8000723A2046534D435F4E414E445F5772692D
:103D90007465537061726528292025640D0A00003E
:103DA00070B504460D462CB1022C03D0042C01D072
:103DB000062C00D104E04FF4867111A005F032FE0C
:103DC0000DB1012D00D104E040F20D110CA005F061
:103DD00029FE55B1A000A0F1C040006840F00101EB
:103DE000A000A0F1C040016009E0A000A0F1C04027
:103DF00000680C490840A100A1F1C041086070BDF5
:103E00002E2E5C4C69627261726965735C737263B9
:103E10005C73746D3332663278785F66736D632ECF
:103E200063000000FEFF0F0010B50446206840B19B
:103E30002068022805D02068042802D020680628BF
:103E400000D103E09021C8A005F0ECFD606810B13E
:103E50006068022800D103E09121C3A005F0E2FDD3
:103E6000A06828B1A068042802D0A068082800D162
:103E700003E09221BCA005F0D5FDE06810B1E06838
:103E8000102800D103E09321B7A005F0CBFD2069F5
:103E900018B12069B0F5807F00D103E09421B2A071
:103EA00005F0C0FD606918B16069B0F5004F00D140
:103EB00003E09521ACA005F0B5FDA06918B1A0699B
:103EC000B0F5007F00D103E09621A7A005F0AAFD80
:103ED000E06918B1E069B0F5806F00D103E0972187
:103EE000A1A005F09FFD206A18B1206AB0F5006F0F
:103EF00000D103E098219CA005F094FD606A18B100
:103F0000606AB0F5805F00D103E0992196A005F0CA
:103F100089FDA06A18B1A06AB0F5005F00D103E086
:103F20009A2191A005F07EFDE06A18B1E06AB0F533
:103F3000804F00D103E09B218BA005F073FD206B27
:103F400018B1206BB0F5002F00D103E09C2186A0B2
:103F500005F068FD606B00680F2800D803E09D2124
:103F600081A005F05FFD606B40680F2800D803E07A
:103F70009E217DA005F056FD606B806820B1606BCE
:103F80008068FF2800D803E09F2177A005F04AFD54
:103F9000606BC0680F2800D803E0A02172A005F074
:103FA00041FD606B00690F2800D803E0A1216EA0DD
:103FB00005F038FD606B40690F2800D803E0A221AE
:103FC00069A005F02FFD606B806970B1606B80693E
:103FD000B0F1805F09D0606B8069B0F1005F04D000
:103FE000606B8069B0F1405F00D103E0A3215EA067
:103FF00005F018FDD4E901010843E168084321698F
:10400000084361690843A1690843E1690843216ADB
:104010000843616A0843A16A0843E16A0843216BC7
:10402000084321688900A1F1C0410860A068082800
:104030000BD120688000A0F1C040006840F0400132
:1040400020688000A0F1C0400160606B0068616B77
:10405000496840EA0110616B896840EA0120616BA0
:10406000898940EA0140616B098A40EA0150616B2D
:10407000097D40EA0160616B896908432168491C38
:104080008900A1F1C0410860E06AB0F5804F62D1BB
:10409000A06B00680F2800D803E0C52132A005F00E
:1040A000C1FCA06B40680F2800D803E0C6212EA0F9
:1040B00005F0B8FCA06B806820B1A06B8068FF2879
:1040C00000D803E0C72128A005F0ACFCA06B006974
:1040D0000F2800D803E0C82123A005F0A3FCA06BA3
:1040E00040690F2800D803E0C9211FA005F09AFC01
:1040F000A06B806970B1A06B8069B0F1805F09D05E
:10410000A06B8069B0F1005F04D0A06B8069B0F152
:10411000405F00D103E0CA2113A005F083FCA06B2F
:104120000068A16B496840EA0110A16B896840EA08
:104130000120A16B098A40EA0150A16B097D40EA88
:104140000160A16B8969084321688900A1F1C04120
:10415000C1F8040107E06FF0704120688000A0F111
:10416000C040C0F8041110BD2E2E5C4C6962726113
:10417000726965735C7372635C73746D333266323B
:1041800078785F66736D632E6300000000B597B0AA
:1041900003F01AFB0121084603F0B0F8002001905B
:1041A000029002200390002004900F2005900690BA
:1041B0000020079004200890002009900A90102009
:1041C0000B9000200C900D900E900F9010904FF4DB
:1041D00080501190002012901390149001A8159017
:1041E000169008A8FFF720FE01210420FFF7D8FD54
:1041F00017B000BD2DE9F04104460D46002600270A
:10420000B0465248844217D05148844214D0514895
:10421000844211D0504884420ED0504884420BD082
:104220004F48844208D04F48844205D04E488442CB
:1042300002D04E48844200D103E0BA214CA005F0E0
:10424000F1FB002010B9286800B103E0BB2148A0B1
:1042500005F0E8FB287940B12879012805D02879B4
:10426000022802D02879032800D103E0BC2140A015
:1042700005F0D8FBE87928B1E879012802D0E8797F
:10428000022800D103E0BD2139A005F0CBFB0026B8
:1042900057E0012000FA06F7286800EA0708B84549
:1042A0004ED1206872000321914088432060287914
:1042B000710088402168084320602879012802D0D5
:1042C0002879022830D1687940B16879012805D071
:1042D0006879022802D06879032800D103E0CF2151
:1042E00023A005F09FFBA068720003219140884342
:1042F000A060687971008840A1680843A060A8792F
:1043000010B1A879012800D103E0D62118A005F04A
:1043100089FB61680120B040814361606068A979D0
:10432000B14089B208436060E068720003219140A7
:104330008843E060E87971008840E1680843E06004
:10434000761C102EA5D3BDE8F081000000000240CD
:104350000004024000080240000C0240001002402D
:104360000014024000180240001C024000200240DD
:104370002E2E5C4C69627261726965735C73726344
:104380005C73746D3332663278785F6770696F2E54
:10439000630000002DE9F04106460D461446002753
:1043A000B8465148864217D05048864214D05048EB
:1043B000864211D04F4886420ED04F4886420BD0DD
:1043C0004E48864208D04E48864205D04D48864227
:1043D00002D04D48864200D104E040F215214BA0A6
:1043E00005F020FBEDB1012D1BD0022D19D0032DBE
:1043F00017D0042D15D0052D13D0062D11D0072D63
:104400000FD0082D0DD0092D0BD00A2D09D00B2D62
:1044100007D00C2D05D00D2D03D00E2D01D00F2D62
:1044200000D104E040F2162138A005F0FBFA9CB35D
:10443000092C31D084B37CB374B36CB3012C2BD072
:104440002AD0022C28D027D026D0032C24D0042C0C
:1044500022D021D020D0052C1ED01DD0092C1BD05D
:10446000062C19D0092C17D0072C15D014D013D036
:10447000082C11D010D00FD0092C0DD00CD00A2C44
:104480000AD009D00B2C07D00C2C05D004D003D0B7
:104490000D2C01D00F2C00D104E040F217211BA0FD
:1044A00005F0C0FA6807C00E04FA00F7E91006F13B
:1044B000200050F821006907CA0E0F21914088435F
:1044C000EA1006F1200141F82200E91006F120006F
:1044D00050F8210040EA0708E91006F1200040F8F2
:1044E0002180BDE8F081000000000240000402408D
:1044F00000080240000C024000100240001402407C
:1045000000180240001C0240002002402E2E5C4C8D
:1045100069627261726965735C7372635C73746DF6
:104520003332663278785F6770696F2E63000000FF
:1045300070B505460C4600262B48854217D02B48FF
:10454000854214D02A48854211D02A4885420ED08F
:10455000294885420BD02948854208D02848854201
:1045600005D02848854202D02748854200D104E082
:1045700040F22F1125A005F055FA012C25D0022C70
:1045800023D0042C21D0082C1FD0102C1DD0202C7F
:104590001BD0402C19D0802C17D0B4F5807F14D0BC
:1045A000B4F5007F11D0B4F5806F0ED0B4F5006F74
:1045B0000BD0B4F5805F08D0B4F5005F05D0B4F53A
:1045C000804F02D0B4F5004F00D104E04FF4987151
:1045D0000EA005F027FA2869204008B1012600E066
:1045E0000026304670BD000000000240000402407A
:1045F00000080240000C024000100240001402407B
:1046000000180240001C0240002002402E2E5C4C8C
:1046100069627261726965735C7372635C73746DF5
:104620003332663278785F6770696F2E63000000FE
:1046300070B504460D461648844217D0154884428A
:1046400014D01548844211D0144884420ED0144826
:1046500084420BD01348844208D01348844205D0CA
:104660001248844202D01248844200D104E040F251
:10467000911110A005F0D6F9002008B905B104E0A9
:104680004FF4C9710BA005F0CDF92804A06170BDED
:10469000000002400004024000080240000C0240FA
:1046A000001002400014024000180240001C0240AA
:1046B000002002402E2E5C4C696272617269657343
:1046C0005C7372635C73746D3332663278785F67E3
:1046D00070696F2E6300000070B504460D461648E1
:1046E000844217D01548844214D01548844211D012
:1046F000144884420ED0144884420BD0134884429C
:1047000008D01348844205D01248844202D012488F
:10471000844200D104E04FF4BF7110A005F082F98B
:10472000002008B905B104E040F27F110BA005F0AC
:1047300079F9A56170BD000000000240000402404C
:1047400000080240000C0240001002400014024029
:1047500000180240001C0240002002402E2E5C4C3B
:1047600069627261726965735C7372635C73746DA4
:104770003332663278785F6770696F2E63000000AD
:1047800070B505460C4616462E48854217D02E4871
:10479000854214D02D48854211D02D4885420ED037
:1047A0002C4885420BD02C48854208D02B488542A6
:1047B00005D02B48854202D02A48854200D104E02A
:1047C00040F2A51128A005F02DF9012C25D0022CCE
:1047D00023D0042C21D0082C1FD0102C1DD0202C2D
:1047E0001BD0402C19D0802C17D0B4F5807F14D06A
:1047F000B4F5007F11D0B4F5806F0ED0B4F5006F22
:104800000BD0B4F5805F08D0B4F5005F05D0B4F5E7
:10481000804F02D0B4F5004F00D104E04FF4D371C3
:1048200011A005F0FFF80EB1012E00D104E040F216
:10483000A7110DA005F0F6F80EB1AC6101E020045F
:10484000A86170BD00000240000402400008024060
:10485000000C024000100240001402400018024008
:10486000001C0240002002402E2E5C4C69627261E6
:10487000726965735C7372635C73746D3332663234
:1048800078785F6770696F2E6300000000BFFEE7F5
:104890002DE9FE4F04460D4616461F46DDF830A0B2
:1048A0000020029001978046814601A813F0FCFD8C
:1048B0008DF808000298C0F3C00028700298C0F379
:1048C000031020706946019800F034F9814601997F
:1048D00008440190DDE9001000EB01080198A8EB05
:1048E0000000022800DA06E001A813F0E4FD3080A1
:1048F0004FF0010900BF4846BDE8FE8F2DE9FF4794
:1049000004460D461646994600200390029600275D
:104910008046009002A813F0C7FD8DF80C000398A4
:10492000C0F30310022800D01FE001A9029800F094
:1049300001F98046029908440290DDE90110471808
:104940000298381A022800DA0FE002A813F0ACFD32
:104950008DF80000009800F00100207002A813F00C
:10496000A3FD28704FF0010800BF404604B0BDE829
:10497000F0872DE9FF5F06460C4617469846DDE9AD
:104980000FABDDF8389000200390119802900025BD
:1049900000200190009002A813F086FD8DF80C0015
:1049A0000398C0F30310032800D032E00398C0F34B
:1049B000C00030700398C0F341002060039800F0FD
:1049C000010038706946029800F0B4F8019002992D
:1049D000084402900099029845182A4602A94846C0
:1049E00013F076FD10B10298281A00D511E0206866
:1049F000002804DD02A813F05EFDA8F8000002986C
:104A0000281ACBF800000298CAF800000120019093
:104A100000BF019804B0BDE8F09F2DE9FE4F0546A8
:104A20000E4614461F46DDE90C9B00200290CDF88F
:104A300004908046824601A813F036FD8DF80800E8
:104A40000298C0F30310092800D02CE069460198B1
:104A500000F070F88246019908440190DDE90010E9
:104A600000EB01080198A8EB0000022800DA1AE028
:104A700001A813F020FD2880002020600DE02068B0
:104A8000B04202DD4FF0FF3A0DE001A813F00CFD3B
:104A90002268511C216047F8220001984045EED35E
:104AA0004FF0010A00BF5046BDE8FE8FFEB5044638
:104AB0000D46164600200290019000272B46224604
:104AC00001A902A80096FFF7E3FE07469DF808003B
:104AD0000B2800D101273846FEBD2DE9F8430546D5
:104AE0000C46012600270020206000BF4FF0FF3851
:104AF000781C0746042801DD00BF17E00121684645
:104B0000A8478046B8F1010F00D00FE09DF80010D3
:104B100001F07F01206801FB06002060F6019DF88E
:104B2000000000F080000028E0D100BF3846BDE85A
:104B3000F883000070B504460D460348046029461A
:104B40000248FFF7CAFF70BDA8010020299A00089B
:104B500030B50246002300BF0846CD1701EB55656E
:104B6000ED11A1EBC515ECB2CD1701EB5565E911BF
:104B7000002901DD44F0800418465B1C1454002910
:104B8000EADC184630BD0000401C802801DA401CD9
:104B90000AE0B0F5804F01DA801C05E00349884245
:104BA00001DAC01C00E0001D70470000FFFF1F007D
:104BB0002DE9FC4104460F4615464FF0FF38002012
:104BC00001900026009001212046A847012800D02E
:104BD0001EE0012669462846FFF77FFF601C00990A
:104BE000FFF7B6FF064400983044B84200DD0FE0FE
:104BF000009830B1A0190099A8470099884200D0C8
:104C000006E020788DF804000198C0F3031800BF77
:104C10004046BDE8FC812DE9FC4704460E4615469A
:104C20001F46DDF828800020019081460094042E64
:104C300002DA6FF0010924E0019865F30710019092
:104C4000019867F3C3000190062D01D1012100E016
:104C50000021019861F3420001909DF8041068461C
:104C600018F0F1FC02210098FFF772FF0099084448
:104C700000904146684618F0ECFC0098A0EB04094F
:104C800000BF4846BDE8FC872DE9FE4305460E46B9
:104C90001446029500200190009000274FF0FF3845
:104CA000204600F0A5F807468146FFF76DFFB042A9
:104CB00002DD6FF001088FE000208DF804000198FC
:104CC00020F0F000103001909DF8041002A818F0B8
:104CD000BAFC39460298FFF73BFF0299084402905C
:104CE000207A042808D13EA102A818F098FC0421DB
:104CF00002A818F0A8FC07E03BA102A818F08FFC5E
:104D0000032102A818F09FFC00208DF80000A17E6E
:104D1000009861F341000090E07E08B1012100E0BD
:104D20000021009861F3820000900098C0F3800099
:104D300058B194F83D10009861F3C400009094F8C5
:104D40003C10009861F345100090206C08B9A06CED
:104D500020B1009820F0800080300090E06C08B90D
:104D6000606D20B1009820F04000403000909DF828
:104D7000001002A818F067FC218B02A818F069FC4B
:104D800002A8D4E90423E16818F07BFCE07E58B166
:104D900002A8D4E90A23616A18F073FC02A8D4E9D6
:104DA0000D23216B18F06DFC0098C0F3C01028B1E2
:104DB00002A8D4E91123216C18F063FC0098C0F319
:104DC000801028B102A8D4E91423E16C18F059FC32
:104DD0000298A0EB050800BF4046BDE8FE83000036
:104DE0004D515454000000004D514973647000004F
:104DF00070B504460025207A032801D10C2503E074
:104E0000207A042800D10A25D4E90412E06800F0D1
:104E100063F9801C0544E07E68B1D4E90A12606A37
:104E200000F05AF9861CD4E90D12206B00F054F9F9
:104E30003044801C0544206C08B9A06C30B1D4E922
:104E40001112206C00F048F9801C0544E06C08B990
:104E5000606D30B1D4E91412E06C00F03DF9801CB3
:104E60000544284670BD70B504460D460C222946FF
:104E7000204600F00BF970BDF8B505460E46144605
:104E800000230422314628460094FFF7C4FEF8BDF3
:104E9000F8B505460E46144600230722314628463B
:104EA0000094FFF7B8FEF8BD2DE9F04F87B0054636
:104EB0000F4690461C46DDE915B6DDE9109A0695C9
:104EC00000200590049003900096204612A90EC978
:104ED00000F042F804900290FFF756FEB84203DD5E
:104EE0006FF00100039033E0059820F0F0003030BF
:104EF0000590059868F3C3000590059864F3420097
:104F00000590059869F3000005909DF8141006A817
:104F100018F099FB04990698FFF71AFE06990844C1
:104F2000069006A812A90EC918F0ABFB002C03DDF1
:104F3000514606A818F08DFB324659460698FBF7F5
:104F4000CEF90698304406900698401B039000BFA7
:104F5000039807B0BDE8F08F7FB50546089E002492
:104F600001A807C800F0B8F8801C30440444002DA4
:104F700000DDA41C204604B070BDF8B506460F46FF
:104F800014461D4623460522394630460095FFF754
:104F900042FEF8BDF8B506460F4614461D462346A8
:104FA0000622394630460095FFF735FEF8BD2DE95B
:104FB000FF5F05460E4617469846DDE90E9A0395B3
:104FC000002002900190009000245146484600F0D5
:104FD00046F883460190FFF7D7FDB04202DDA01EE0
:104FE000009038E000208DF80800029820F0F000D2
:104FF00080300290029867F3C3000290029820F07C
:105000000600801C02909DF8081003A818F01BFBF6
:1050100001990398FFF79CFD0399084403904146CA
:1050200003A818F016FB00240FE004EB44000AEB81
:10503000800C03A89CE80E0018F023FB109810F8D1
:10504000241003A818F0FFFA641C4C45EDDB03980C
:10505000401B009000BF009804B0BDE8F09F2DE910
:10506000F04105460E46022700240AE004EB440006
:1050700006EB800393E8070000F02EF8C01C0744FD
:10508000641CAC42F2DB3846BDE8F0812DE9FC41FE
:1050900004460D46164600200190471E0094022D3E
:1050A00001DA871E15E000208DF80400019866F3F0
:1050B000071001909DF80410684618F0C4FA00210A
:1050C0000098FFF745FD0099084400900098071BE1
:1050D00000BF3846BDE8FC8137B50024009820B1F8
:1050E0000098FBF73EF9044600E0019C20463EBDD7
:1050F00000BFFEE738B5002406E04FF6FF702C49EC
:1051000021F81400601C84B2B4F5806FF5DB002434
:1051100021E0A101042300226846FEF705FD9DF869
:105120000000FF2815D19DF802109DF8030001EB47
:10513000002085B2B5F5806F0BDA1D4830F81500F8
:105140004FF6FF71884201D0012038BD184820F881
:105150001540601C84B2B4F5806FDADB00240AE0ED
:10516000134830F81400B0F5806F02DB114804805A
:1051700004E0601C84B2B4F5806FF1DB00BF0D4821
:105180000088642801DA0120DFE70AE0084830F8E7
:1051900014004FF6FF71884201D00120D5E7601C52
:1051A00084B2044800888442F0DB0020CDE7000090
:1051B0006CC900205C00002070B5054640F2FF3449
:1051C00005F0400028B104F0010038B9601E84B237
:1051D00004E004F0010008B1601E84B20CE0204637
:1051E00000F040F808B1204670BD022C02DA4FF6FC
:1051F000FF70F9E7A01E84B2F1E7000004480088C0
:1052000062225043642290FBF2F148047047000090
:105210005C00002010B5FEF7AFFAFEF7C5FCFFF703
:1052200069FF0446204610BD38B50446A10101239C
:1052300000226846FEF778FC9DF80000FF2801D0A8
:10524000012038BD012000EB84110346002268468E
:10525000FEF76AFC9DF80000FF2801D00120F0E76E
:105260000020EEE738B504462046FFF7DDFF08B121
:10527000002038BDA10101231A466846FEF754FC00
:105280009DF80000FF2801D10120F2E70020F0E79F
:10529000014606480088814202D34FF6FF707047EE
:1052A000034830F811201046F9E700005C000020A8
:1052B0006CC9002038B5044621460AA003F036FB2D
:1052C000A501002000900123002229466846FEF730
:1052D0003DFD012805D101230022691C6846FEF727
:1052E00035FD38BD4E414E445F4D61726B42616485
:1052F000426C6F636B282564290D0A0038B504469B
:10530000A501F020009001231A4629466846FEF7C1
:105310001DFD012800D138BD0020FCE72DE9FF5F0D
:1053200081460F4614469A4600253BE04FF4006044
:1053300090FBF4F080017919B1FBF0FB5846FFF7C0
:10534000A7FF0646B6F5806F07D3314617A003F0D6
:10535000EDFA012004B0BDE8F09F7819A0FB04101D
:105360004FF400320023CDE9001008460199FAF706
:105370007FFF9046B00100EBD8200390C8F30A00ED
:10538000029005FB04902346DDE90221FEF76CFB49
:10539000012806D11448DDE9022103F0C7FA0120F3
:1053A000D8E76D1C5545C1D30020D3E74572726F15
:1053B000723A204E414E445F526561644D756C7483
:1053C00069536563746F727328292C206E6F742083
:1053D000666F726D61742C20757350424E203D20B3
:1053E00025640D0A00000000888A04082DE9FF4F9B
:1053F00083B006468946144600257DE04FF40060E0
:1054000090FBF4F0800109EB0501B1FBF0FA504686
:10541000FFF73EFF0746B7F5806F08D33A4651467F
:10542000384803F083FA012007B0BDE8F08F4FF44D
:10543000006090FBF4F0800109EB0501B1FBF0F294
:1054400000FB121000FB04FBB80100EBDB28CBF3E0
:105450000A000290FF2221462B48FAF752FF23460A
:1054600041462948029AFEF723F9002832D105FB6C
:10547000046023464146029AFEF7A4FB012816D198
:1054800022A003F053FA05FB046123464046029A2A
:1054900000F084F80190019820B128A003F046FAAA
:1054A0000120C1E74FEA9810FFF704FF23E04FEA1D
:1054B0009810FFF723FF01281CD105FB0461234648
:1054C0004046029A00F06AF80190019808B1012064
:1054D000AAE710E005FB046123464046029A00F06B
:1054E0005DF80190019820B120A003F01FFA01207F
:1054F0009AE700E000BF6D1C06988542FFF47EAF7E
:10550000002091E7148B04086CD100204572726F63
:1055100072333A204E414E445F57726974654D753F
:105520006C7469536563746F727328292C205772E9
:10553000697465204661696C650D0A004572726F79
:1055400072343A204E414E445F57726974654D750E
:105550006C7469536563746F727328292C205772B9
:10556000697465204661696C650D0A004572726F49
:1055700072353A204E414E445F57726974654D75DD
:105580006C7469536563746F727328292C20577289
:10559000697465204661696C650D0A002DE9FC5F40
:1055A0008046894692469B46C8F38F1608F03F0016
:1055B0000190002761E04046FFF7FEFD0546B5F586
:1055C000806F06DB294633A003F0B0F90120BDE867
:1055D000FC9F00242CE00198844215D104EB851136
:1055E00004EB861053464A46CDF800B0FEF7D0F9DA
:1055F00001281BD1314630A003F098F92846FFF767
:1056000059FEFFF777FD15E004EB851104EB8610DA
:10561000FEF742F9012809D1314630A003F086F99E
:105620002846FFF747FEFFF765FD03E0601C84B2E4
:10563000402CD0DB00BF402C1CD12846FFF75EFE7B
:10564000012805D12846FFF735FEFFF753FD12E08C
:105650003046FEF767F8402809D0314628A003F00D
:1056600065F93046FFF726FEFFF744FD03E0FFF73C
:1056700041FD04E000BF781C87B20A2F9BDB00BF0E
:105680000A2F05D1394628A003F050F901209EE7E2
:1056900000209CE74572726F72313A204E414E44B1
:1056A0005F5772697465546F4E6577426C6F636BB8
:1056B00028292025640D0A004572726F72323A2043
:1056C0004E414E445F5772697465546F4E65774220
:1056D0006C6F636B28292025640D0A004572726F78
:1056E00072333A204E414E445F5772697465546F6D
:1056F0004E6577426C6F636B28292025640D0A0084
:105700004572726F72343A2046534D435F4E414E9C
:10571000445F4572617365426C6F636B28292C206E
:1057200025640D0A000000004572726F72353A2040
:1057300046534D435F4E414E445F4572617365422F
:105740006C6F636B2829206E3D25640D0A000000F4
:105750001CB50121202001F05DFD4FF48070009008
:1057600001208DF8040000208DF8060001208DF83E
:10577000070000208DF8050069460248FEF73AFD53
:105780001CBD000000140240704710B54FF4A0602B
:1057900000F066F810BD00002DE9F0410446002538
:1057A00000270F26E07810B1E078012800D103E04F
:1057B000862122A004F036F96078102800DA03E090
:1057C00087211EA004F02EF9A078102800DA03E04B
:1057D00088211AA004F026F9E07818B31D48006863
:1057E00000F4E060C0F5E060C0F30725C5F10400F7
:1057F000C7B22E416078B840C5B2A07830400543AA
:105800002807050E144821784554207800F01F0120
:105810000120884021784911890001F1E021C1F877
:10582000000109E0207800F01F01012088400B49A9
:105830002278521141F82200BDE8F0812E2E5C4CF6
:1058400069627261726965735C7372635C6D6973BE
:10585000632E63000CED00E000E400E080E100E076
:1058600010B50446B4F5E06F0BD0B4F5C06F08D0A6
:10587000B4F5A06F05D0B4F5806F02D0B4F5407FC9
:1058800000D103E0722104A004F0CCF808482043C2
:105890000849086010BD00002E2E5C4C69627261E0
:1058A000726965735C7372635C6D6973632E630008
:1058B0000000FA050CED00E02DE9F04105460E462A
:1058C000144600271148007818B112202070BDE856
:1058D000F0812878012808D0022807D0032802D0B8
:1058E000042804D100E000BF00BF00BF02E0012097
:1058F0002070ECE700BFFAF763FC07462E613846DC
:10590000FAF762FC0020207000BFE0E7940000205E
:1059100010B500F015F801F05FFA01F07BFA01F024
:105920009BFA01F029FA01F0E9F901F005FB01F019
:105930002FFB01F0CFFA01F001F800F019F810BDCB
:105940000748802102E0491E002204C00029FAD144
:10595000044A054B1A600022044B1A80704700006D
:1059600084F9002080FB0020D8000020DC0000200B
:105970007047000006480078012808D105480078E3
:10598000FF2804D203480078401C02490870704781
:105990009D0000209400002010B500241A480078D3
:1059A000012830D1FAF70CFC04461848007820B1E1
:1059B00016480078401E1549087014480078F8B958
:1059C00013480078E0B901F047FB12481249097802
:1059D00050F82100114908600F48007810490978F3
:1059E00088420DD00D480068806B401C0B49096847
:1059F00088630C480068401C0A490860FAF700FCFC
:105A00002046FAF7E1FB10BD9D0000209400002025
:105A10009500002020E8002097000020AC00002026
:105A2000960000208800002070B5044600262078EB
:105A3000012801D0002070BDFAF7C2FB0646656858
:105A4000002060603046FAF7BFFB2846F3E700000D
:105A500070B5054600261048007808B1002070BDDA
:105A6000FAF7AEFB06460D480468006820B10B4803
:105A700000684068094908603046FAF7A5FB4CB158
:105A80000120207000202081656005A02061204653
:105A900001F026F92046E2E7940000208C00002067
:105AA0003F0000002DE9F04105460F4614464FF037
:105AB00000082878012804D0012020700020BDE8CB
:105AC000F0813648007818B1022020700020F6E7F7
:105AD0003348007818B10D2020700020EFE7FAF766
:105AE0006FFB80466E6846B1002068604046FAF75A
:105AF0006BFB002020703046E1E72A48006890F8F0
:105B0000300040F002002749096881F83000002089
:105B10002449096881F8310022480068C762284694
:105B200001F0A0F84046FAF74FFB01F05BFAFAF7F4
:105B300047FB80461B48006890F8310020B10128DF
:105B40000DD002280AD105E016480068066A002038
:105B500020700DE000260E20207009E000BF2946CD
:105B60001048006801F068F800260A20207000BF85
:105B700000BF00200B49096881F830000949096815
:105B800081F8310007490968C86106490968086257
:105B90004046FAF719FB304691E7000094000020D8
:105BA00095000020A400002070B504460D46002694
:105BB0002078012801D0012070BDFAF701FB0646CC
:105BC000A07A60B1002302222946204600F0F2FFAD
:105BD0003046FAF7F9FA01F005FA0020ECE76068C0
:105BE00020B13046FAF7F0FA1420E5E76560304658
:105BF000FAF7EAFA0020DFE72DE9F04106460F4602
:105C00004FF000082048007810B10020BDE8F08176
:105C1000FAF7D6FA80461D480468006820B11B4890
:105C200000684068194908604046FAF7CDFAFCB1AF
:105C3000FAF7C6FA804616480568D5B100680068CC
:105C4000134908604046FAF7BFFA6E6006EB87001A
:105C5000A860EE602E61AF820020E88202202070F2
:105C60000020208165600BA02061204601F038F8FB
:105C700008E0064800686060044804604046FAF79F
:105C8000A3FA00242046C1E7940000208C000020E5
:105C9000BC0000203F0000002DE9F0470446894683
:105CA00015464FF0000A2078022804D00120287001
:105CB0002046BDE8F0873548007818B10F202870DD
:105CC0002046F6E7FAF77CFA8246A07A10B14FF048
:105CD000010801E04FF00008B9F1000F03D0B9F15D
:105CE000010F49D121E0B8F1000F17D128A02061A0
:105CF00066682848006830602648066000202070EA
:105D000025480068606000202081234804605046D8
:105D1000FAF75AFA00202870002705E05046FAF7F3
:105D200053FA4920287027462DE005E0002304227D
:105D30001946204600F03EFFA07A0028F6D114A0B4
:105D400020616668134800683060124806600020D1
:105D50002070114800686060002020810E480460B7
:105D60005046FAF731FAB8F1010F01D101F03AF9D2
:105D700000202870002706E05046FAF725FA072091
:105D80002870274600BF00BF384692E794000020E5
:105D90003F000000BC0000208C00002070B50546CC
:105DA0000026FAF70DFA06466C686068E0606068E5
:105DB00020610020E0823046FAF706FA002070BD2C
:105DC0002DE9F0470746884615464FF00009387818
:105DD000022804D0012028700020BDE8F0873C484C
:105DE000007818B1022028700020F6E739480078C2
:105DF00018B10D2028700020EFE7FAF7E1F981468D
:105E00007C68E08A98B12169081D20610E68E08AEB
:105E1000401EE082A1682069884201D1606820614B
:105E20004846FAF7D1F9002028703046D5E72A48CD
:105E3000006890F8300040F004002749096881F8B4
:105E4000300000202449096881F8310022480068A8
:105E5000C0F82C80384600F005FF4846FAF7B4F940
:105E600001F0C0F8FAF7ACF981461B48006890F8D9
:105E7000310020B101280DD002280AD105E01648D2
:105E80000068066A002028700DE000260E202870A9
:105E900009E000BF39461048006800F0CDFE00263A
:105EA0000A20287000BF00BF00200B49096881F854
:105EB00030000949096881F8310007490968C8615B
:105EC0000549096808624846FAF77EF9304684E7D2
:105ED0009400002095000020A40000202DE9F0414E
:105EE00005460E4600272878022802D00120BDE88A
:105EF000F081FAF765F90746A87A60B10023042219
:105F00003146284600F056FE3846FAF75DF901F0B2
:105F100069F80020EBE76C68E08AA18A884204DB1C
:105F20003846FAF751F91E20E1E7E168081DE06004
:105F30000E60E08A401CE082D4E90210884201D160
:105F40006068E0603846FAF73FF90020CFE70000CC
:105F500010B500240B480078012811D1FAF730F968
:105F600004460948007840B908480078FF2804D260
:105F700006480078401C054908702046FAF724F9C5
:105F800010BD00009D00002094000020950000201E
:105F900010B5002413480078012821D1FAF710F930
:105FA000044611480078C0B10F480078401E0E49E1
:105FB00008700846007860B90C48007828B9204677
:105FC000FAF702F901F00EF80AE02046FAF7FCF8B9
:105FD00006E02046FAF7F8F802E02046FAF7F4F86F
:105FE00010BD00009D0000209500002094000020BE
:105FF00070B5054600261048007808B1002070BD35
:10600000FAF7DEF806460D480468006820B10B4830
:1060100000684068094908603046FAF7D5F84CB185
:106020000320207025810020606005A020612046AB
:1060300000F056FE2046E2E7940000208C0000208D
:106040003F0000002DE9F0470446884615464FF012
:1060500000092078032804D0012028702046BDE8DC
:10606000F0872D48007818B10F2028702046F6E7F9
:10607000FAF7A6F88146A07A08B1012700E00027C8
:10608000B8F1000F03D0B8F1010F3AD119E08FB980
:1060900022A020610020207021480068606000205C
:1060A00020811F4804604846FAF78EF800202870C7
:1060B000002605E04846FAF787F84920287026466A
:1060C00026E005E0002301221946204600F072FD7B
:1060D000A07A0028F6D111A020610020207010487D
:1060E00000686060002020810D4804604846FAF78F
:1060F0006BF8012F01D100F075FF002028700026F9
:1061000006E04846FAF760F807202870264600BFE8
:1061100000BF3046A3E70000940000203F000000CD
:106120008C0000202DE9F04105460E46144600275C
:106130002878032803D001202070BDE8F081314881
:10614000007810B102202070F7E72F48007810B1D6
:106150000D202070F1E7FAF733F80746288940B19F
:106160002889401E28813846FAF72EF80020207032
:10617000E3E72648006890F8300040F0010023492A
:10618000096881F8300000202049096881F8310051
:106190001E480068C662284600F064FD3846FAF7DB
:1061A00013F800F01FFFFAF70BF8074617480068CE
:1061B00090F8310020B1012809D0022806D102E070
:1061C000002020700BE00E20207008E000BF294660
:1061D0000E48006800F030FD0A20207000BF00BFAC
:1061E00000200A49096881F830000849096881F8E7
:1061F000310006490968C8613846F9F7E5FF00BF74
:106200009BE700009400002095000020A4000020DF
:1062100070B5044600252078032801D0012070BD08
:10622000F9F7CEFF0546A07A60B100230122194696
:10623000204600F0BFFC2846F9F7C6FF00F0D2FE6A
:106240000020ECE720894FF6FF71884207D22089B1
:10625000401C20812846F9F7B7FF0020DFE72846D9
:10626000F9F7B2FF3320DAE710B50B48007890B9A0
:1062700000F0F2FE0948007809490870094807490A
:10628000097850F821000849086008460068074965
:106290000860F9F79CFF10BD9D00002097000020CA
:1062A0009600002020E80020AC000020A400002080
:1062B000704700002DE9FE4F06460F4690461C46EB
:1062C0004FF00009F9F77CFF81461F48007828B19C
:1062D0004846F9F779FF3C20BDE8FE8F1B4850F88F
:1062E000240060BB0120194941F824004846F9F711
:1062F0006BFF002342463946304600F06FF9824674
:10630000002000900190034602465146029020462C
:1063100000F0B8FE054635B90D48007801280CD1CB
:1063200000F060FE09E0F9F74BFF814600200749C5
:1063300041F824004846F9F747FF2846CCE748468D
:10634000F9F742FF2820C7E79400002020E800204A
:106350009D0000202DE9F04F85B081468A46934686
:106360001C46DDE90F78129D00200390F9F728FF05
:1063700003902348007830B10398F9F725FF3C20BB
:1063800005B0BDE8F08F1F4850F8240088BB0120FD
:106390001C4941F824000398F9F716FF2A464146A4
:1063A000384600F029FF2B465A465146484600F031
:1063B00015F904901198CDE9008002953A462046DF
:1063C0000E9B049900F05EFE064636B90E48007832
:1063D00001280CD100F006FE09E0F9F7F1FE039068
:1063E0000020084941F824000398F9F7EDFE3046F3
:1063F000C6E7FFE70398F9F7E7FE2820C0E70000AB
:106400009400002020E800209D000020704700003C
:106410002DE9F041054600274748007810B140209B
:10642000BDE8F0811F2D01D13E20F9E7F9F7C8FE44
:106430000746FF2D03D14148006890F8325040488C
:1064400050F8254024B93846F9F7BEFE4320E7E767
:10645000012C04D13846F9F7B7FE3D20E0E714F8E7
:10646000340F3849085C617888432178354A5054A4
:1064700014F834091146085C30B994F836103248E3
:106480000078884330490870E06918B12046E16916
:1064900000F0D2FB666A16B1304600F05BFC0020CB
:1064A000E06284F8300084F8310028480078FF2842
:1064B00004D226480078401C244908703846F9F771
:1064C00083FE00F075FBF9F77BFE07461F48007856
:1064D00020B11E480078401E1C490870204600F07C
:1064E00041F81B480078401E1949087000201449E3
:1064F00041F82500A06930B900206169886115491B
:106500006069086005E0D4E905014861D4E9051037
:1065100088611148006860610F4804600FA0E06462
:106520003846F9F751FE0E480078012801D100F0F5
:1065300059FD002074E7000094000020A400002012
:1065400020E80020990000209800002095000020FD
:106550009E000020B0000020A80000203F000000A6
:106560009D000020704770472DE9F04106460F4618
:1065700014464FF000081548007818B1122020701A
:10658000BDE8F081F9F71CFE8046FF2E03D11048CC
:10659000006890F832600F4850F826502DB94046F8
:1065A000F9F712FE43202070EAE7012D05D140469D
:1065B000F9F70AFE43202070E2E7EF644046F9F75E
:1065C00003FE0020207000BFDAE7000094000020E6
:1065D000A400002020E800207047000070B50446A9
:1065E00010464FF080750560051F28462C60214E2F
:1065F000051F28462E604FF01236051F28462E60D4
:106600004FF00336051F28462E604FF00236051F57
:1066100028462E607610051F28462E60051F284646
:1066200029604FF01136051F28462E604FF01036B6
:10663000051F28462E604FF00936051F28462E609C
:106640004FF00836051F28462E604FF00736051F0D
:1066500028462E604FF00636051F28462E604FF064
:106660000536051F28462E604FF00436051F2846C4
:106670002E6070BDE17100082DE9F04105464FF034
:106680000008F9F79DFD8046FF2D05D120480068E0
:1066900090F83250012608E01D48006890F832005A
:1066A000A84201D1012600E000261A4850F82540F2
:1066B0002CB94046F9F788FD4820BDE8F081012C4F
:1066C00004D14046F9F780FD4320F6E794F8347092
:1066D0001148C05D94F8351088430F49C8550846E5
:1066E000C05D30B994F836100C48007888430B49E7
:1066F000087094F8300040F0080084F830004046FC
:10670000F9F762FD012E01D100F06CFC0020D4E706
:10671000A400002020E8002099000020980000201C
:106720007047000070B5054600261748007800B194
:1067300070BD1648007800B1FAE71DB3F9F740FDC7
:1067400006461348006890F834401248005D10492E
:10675000096891F8351088430E4908550846005DD0
:1067600040B90B48006890F836100B480078884311
:106770000949087006480068C5623046F9F724FDEB
:1067800000F030FC00BFD3E794000020950000200B
:10679000A400002099000020980000202DE9F0417D
:1067A00005460E4617461C461248007810B1552083
:1067B000BDE8F0811048007808B13220F8E74FF4C6
:1067C0007A7060434FF47A71B0FBF1F14FF461607D
:1067D0006843C6EB061200EB8200384400EB40022F
:1067E000C2EBC01001EBC0084046FFF79BFF002042
:1067F000DEE70000940000209500002070B5002521
:10680000F9F7DEFC0546034804682846F9F7DCFC86
:10681000204670BDC000002070B5002600F072F860
:10682000F9F7CEFC064631480068401C2F49086045
:106830003046F9F7C9FC2E480078012853D12D487D
:10684000007820B1012804D0022809D103E00125F5
:106850000BE0002509E0012501202649087004E02D
:10686000012500202349087000BF00BF05B970BD95
:106870002148046833E0F9F7A3FC0646E06A50B308
:10688000E06A401EE062E06A28BB94F8300000F045
:10689000370040B114F8300F00F0C800207001201C
:1068A0006070303C02E0002084F8310094F8300041
:1068B00000F0080078B93434A0781049097808430A
:1068C0000E49087020780E49085C6178084314F876
:1068D00034190B4A505464693046F9F775FC94F842
:1068E00032001F28C7D100BFC1E70000C000002050
:1068F0009D000020B4000020B0000020980000207F
:106900009900002010B507480088401C0549088000
:10691000084600880A2803DB0020088000F004F8FD
:1069200010BD0000DC00002010B503480068FFF730
:106930006FFC0446204610BDD0000020F8B54FF48F
:106940002071284800F0EEFA4021274800F0EAFACA
:10695000002514E0681C86B205EB8500214901EB97
:10696000C00406EB860001EBC00764202070002005
:1069700084F82500E7601DA02062681C85B20F2DF9
:10698000E8D305EB8500174901EBC00464202070B3
:10699000002084F82500E06014A020620020144943
:1069A0000860144908801020134908800D481349D5
:1069B00008600120FFF71CFB114908600020FFF769
:1069C00017FB104908606A460FA10D480068FEF7E2
:1069D00073FF6A4611A10B480068FEF76DFF00F0D7
:1069E00027F8F8BDC4F4002044F900203F0000005F
:1069F000C8000020C6000020C4000020D4000020F1
:106A0000CC000020D000002075432F4F532D494962
:106A100020546D724C6F636B0000000075432F4F64
:106A2000532D494920546D725369676E616C0000A3
:106A300000B587B00320002180220A4BCDE9013246
:106A4000CDE903104FF6FD700123074A0090074877
:106A5000FFF780FC06AA06A10120FFF785FD07B01D
:106A600000BD000044F7002040F90020ED6A000856
:106A700075432F4F532D494920546D72000000007B
:106A800070B50B46032580F82550012B05D1154E16
:106A9000C5693668354445610CE085692DB9114EEC
:106AA000C56936683544456104E00E4E856936682F
:106AB00035444561057D05F007040B4D05EBC40128
:106AC0000D682DB908600025C56001258D8006E0A0
:106AD0000A680860C26010618D886D1C8D80002579
:106AE000056170BDC800002044F9002008B500BF52
:106AF00000BF6A4600211A480068FFF713FBFFF742
:106B000027FA18480068401C1649086008460078B3
:106B100000F00708144800EBC8073C681AE0E66874
:106B2000104960690968884213D1204600F01EF8B8
:106B300094F82400022804D101212046FFF7A0FF89
:106B400002E0022084F82500656815B12046A1689E
:106B5000A8473446002CE2D1FFF71AFAC9E7000033
:106B6000D0000020C800002044F9002030B5057D89
:106B700005F007040D4D05EBC4031D68854205D1E2
:106B8000C168196039B100250D6104E00169C2686E
:106B9000CA6002B11161012580F825500025C56049
:106BA00005619D886D1E9D8030BD000044F9002068
:106BB000704700002DE9F04F05460F469046994674
:106BC000A87A19490E5C05F10B00805D11F800B040
:106BD0000BEBC60000F0FF0A144850F82A400020D2
:106BE0002034E0602760207C20EA0800207484F8CC
:106BF0001190207C203C00F0080068B994F8360021
:106C00000B49097808430A4908700A48805D94F8DE
:106C100035100843074988552946204600F00CF8EE
:106C20005046BDE8F08F0000CE84040820E8002024
:106C3000980000209900002010B590F8342001F150
:106C40000B039B5C90F83540A34301F10B04A35464
:106C500023469B5C23B98B7A90F83640A3438B7212
:106C600010BD000010B51B4A1268D061194A1268A5
:106C700092F8343000F10B02D25C164B1B6893F88B
:106C800035301A43134B1B6893F8344000F10B0363
:106C90001A55827A0F4B1B6893F836301A4382726A
:106CA0000C4A126892F834100B4A525C094B1B686C
:106CB00093F835309A43084B5A541A46525C42B9FD
:106CC000044A126892F83630044A12789A43034B09
:106CD0001A7010BDA4000020990000209800002028
:106CE000014600228A72002005E0002301F10B0218
:106CF0001354421CD0B20428F7D370472DE9F04159
:106D00005021114800F00EF900250DE0681C86B2F4
:106D10000D4800EB051400EB06170020207067609B
:106D20000AA0E060681C85B2042DEFD3064800EB92
:106D3000051400202070606004A0E060024804494F
:106D40000860BDE8F0810000D0E500203F000000B1
:106D50009000002030B501464A6808682AB9CC681E
:106D6000606028B10025456002E0106000B142601B
:106D70008B6800255D6230BD70B54FF420711348FB
:106D800000F0D0F8002411E0601C85B204EB840010
:106D90000E4901EB800305EB850001EB8006002026
:106DA00018705E600AA01861601C84B21F2CEBD3BF
:106DB00004EB8400054901EB800300201870586043
:106DC00003A0186108460349086070BD50E3002025
:106DD0003F0000008C0000200020074908600749A0
:106DE0000870074908700749087007490870074983
:106DF0000860074908607047C00000209400002028
:106E0000950000209E0000209D00002088000020AA
:106E1000A000002000210A4A1170002004E0002197
:106E2000084A1154411CC8B20428F8D30021064A6C
:106E30001170064A1170064A1160064A11607047C7
:106E40009800002099000020960000209700002064
:106E5000AC000020A400002070B540F62C2118489A
:106E600000F060F88021174800F05CF8002413E07F
:106E7000601CC5B2C4EBC40000EB4000104901EB3C
:106E80008003C5EBC50000EB400001EB80065E61AE
:106E90000DA0D864601CC4B21E2CE9D3C4EBC4009E
:106EA00000EB4000064901EB80030020586106A07A
:106EB000D86400200549086001480549086070BD94
:106EC000A0E8002020E800203F000000B0000020E3
:106ED000A800002000B587B00320002180220A4BC3
:106EE000CDE90132CDE903104FF6FF701F23074AA9
:106EF00000900748FFF72EFA06AA06A11F20FFF709
:106F000033FB07B000BD000020E600201CE8002095
:106F1000B971000875432F4F532D49492049646CBE
:106F20006500000004E0002200F8012B4A1E91B227
:106F30000029F8D17047000070B578211148FFF79B
:106F4000F1FF00240EE004EB44000E4901EBC00504
:106F5000601C00EB400001EBC00068600AA06861A3
:106F6000601C84B2042CEED304EB4400054901EB11
:106F7000C0050020686004A06861084603490860F5
:106F800070BD0000CCF200203F000000B8000020DF
:106F90002DE9F0414FF4C0711048FFF7C3FF002402
:106FA0000DE0601C86B204EB44000C4901EBC00507
:106FB00006EB460001EBC0072F60601C84B20F2C6B
:106FC000EFD304EB4400054901EBC0050020286025
:106FD000084603490860BDE8F081000044F3002042
:106FE000BC00002010B50024F9F7EAF80446134865
:106FF0000078F8B912480078E0B900F02DF811488F
:107000001149097850F82100104908600E480078AD
:107010000F49097888420DD00C480068806B401CED
:107020000A49096888630B480068401C09490860E0
:10703000F9F7E1F82046F9F7C7F810BD94000020F1
:107040009500002020E8002097000020AC000020E0
:1070500096000020880000200649074A1278885CC4
:107060000649095C034A515C01EBC001044A1170F6
:1070700070470000CE84040898000020990000208A
:10708000970000202DE9F84F05460F469046994697
:10709000DDE90AAB00200090F9F792F800903F4834
:1070A0000468002C74D0183454F8040C3B49086070
:1070B0000098F9F789F844F8187CA5760020207626
:1070C0006076606144F814BC44F80CAC44F8108C51
:1070D0000C9824F8080C24F8069C0020E077E810AF
:1070E000207705F00700E076217F01208840A07717
:1070F000E17E01208840607700206060E060A06051
:107100002062A0626062E062206325A06063183C98
:10711000002606E0002104F1500040F82610701C03
:10712000C6B2012EF6DB2046FFF7C2F82046FFF775
:107130006DF9F9F745F800901A4840F825401A48CB
:10714000006860610020A0611748006810B116480F
:1071500000688461144804603434A07813490978C5
:1071600008431249087020781149085C6178084387
:1071700014F834190E4A50540E480078401C0D493A
:1071800008700098F9F720F80020BDE8F88FFFE7B5
:107190000098F9F719F84220F7E70000A80000204E
:1071A0003F00000020E80020B000002098000020F0
:1071B000990000209E000020002400BF00BFF8F7C7
:1071C000FFFF044605480068401C0449086020464B
:1071D000F8F7FAFFFFF7C7F9F1E70000A000002079
:1071E00010B504480068FFF7F7F9FF20FFF710F922
:1071F00010BD0000A400002002F0010343B102F022
:1072000002032BB102E0491E002308C00029FAD175
:107210007047000070B504460D461048204008B97C
:1072200004B104E040F244410DA002F0FBFB0DB1BB
:10723000012D00D104E040F2464109A002F0F2FB2A
:107240002DB11048006820430E49086004E00D4845
:107250000068A0430B49086070BD000000EE9B81F0
:107260002E2E5C4C69627261726965735C73726325
:107270005C73746D3332663278785F7263632E6349
:10728000000000003038024070B504460D4610483A
:10729000204008B904B104E04FF4A0610DA002F051
:1072A000C1FB0DB1012D00D104E040F2015109A054
:1072B00002F0B8FB2DB11048006820430E49086069
:1072C00004E00D480068A0430B49086070BD000051
:1072D00000EE9FDD2E2E5C4C6962726172696573EF
:1072E0005C7372635C73746D3332663278785F728C
:1072F00063632E63000000001038024070B504463E
:107300000D4624F0010008B904B104E040F27F41C9
:107310000CA002F087FB0DB1012D00D104E04FF469
:10732000906108A002F07EFB2DB10F480068204359
:107330000D49086004E00C480068A0430A49086051
:1073400070BD00002E2E5C4C6962726172696573BB
:107350005C7372635C73746D3332663278785F721B
:1073600063632E63000000003838024070B50446A5
:107370000D461048204008B904B104E040F2B14184
:107380000DA002F04FFB0DB1012D00D104E040F241
:10739000B24109A002F046FB2DB11048006820431D
:1073A0000E49086004E00D480068A0430B490860DE
:1073B00070BD0000003601C92E2E5C4C69627261FE
:1073C000726965735C7372635C73746D33326632B9
:1073D00078785F7263632E630000000040380240DB
:1073E00070B504460D461048204008B904B104E0C9
:1073F00040F2D9410DA002F015FB0DB1012D00D1D5
:1074000004E040F2DA4109A002F00CFB2DB1104873
:10741000006820430E49086004E00D480068A0435E
:107420000B49086070BD0000CCA0F8FF2E2E5C4C0C
:1074300069627261726965735C7372635C73746DA7
:107440003332663278785F7263632E630000000027
:1074500044380240F0B50021002200240225002615
:107460000223324F3F6807F00C0121B1042905D0F7
:10747000082937D105E02E4F076036E02D4F076011
:1074800033E02A4F3F1F3F68C7F38056274F3F1F07
:107490003F6807F03F036EB1264FB7FBF3F7DFF805
:1074A0008CC0ACF1040CDCF800C0CCF3881C07FBEA
:1074B0000CF40CE01E4FB7FBF3F7DFF870C0ACF133
:1074C000040CDCF800C0CCF3881C07FB0CF4174F4D
:1074D0003F1F3F68C7F301477F1C7D00B4FBF5F7F2
:1074E000076002E0124F076000BF00BF0F4F3F6808
:1074F00007F0F0010909104F7A5C0768D740476030
:107500000A4F3F6807F4E051890A0B4F7A5C4768DD
:10751000D7408760054F3F6807F46041490B064F2D
:107520007A5C4768D740C760F0BD00000838024069
:107530000024F40040787D01310000202DE9F04F57
:1075400089B083465E46B0690468B069856803E126
:10755000707D03287ED1012082490870E08B00EB0A
:10756000D071491008910899480001F09FFA8246AD
:10757000B07D0CF00FFF6078032801D1012000E0FE
:1075800000206178012900D100E000210843002893
:1075900070D0E78B07EBD7735A10E18A20785346F7
:1075A0000CF0A8FD07900798002862D0E08B042813
:1075B00006D1BAF80000BAF8021040EA010904E066
:1075C000E08B022801D1BAF8009094F8200058B955
:1075D00084F819904FEA0920A0764FEA0940E07636
:1075E0004FEA0960207721E094F82000F9F7ACFB1E
:1075F00007463A460B4600205B4910F0D5F8CDE926
:1076000002014846F9F78AFB0746F9F7C9FBCDE9BD
:107610000001DDE90223F9F712FBCDE90401F9F7D6
:1076200003FC06900698C4F8190000BF4F48F8F70D
:1076300098FE4E494718A31C721C4DA13846CDF840
:10764000009001F083F9646A94B94848F8F789FE1C
:10765000464900E012E00844471E4FA1384601F0B9
:1076600075F9504601F09EF9002009B0BDE8F08F91
:1076700000BF00BF504601F095F96DE0707D042811
:1076800003D101203749087066E0707D022802D0DE
:10769000707D012860D1022032490870002085F8F1
:1076A00029000690079008900A2105F12000F8F7BC
:1076B0002FFEB0698168394805F097FA707D02287D
:1076C00007D1012306AA3548E96905F035FA47B222
:1076D00009E0707D012806D1022306AA2F48E96936
:1076E00005F02AFA47B2781CF8B1042F05DC069899
:1076F0002862042085F829001AE0052F09D1069890
:1077000028629DF81C0085F82400052085F82900D2
:107710000EE0052F0CDD092206A905F12000F8F77F
:10772000DEFD092085F8290002E0002085F8290007
:107730000E48F8F716FE0D4900EB010805F1200090
:10774000AB1D721C16A10090404601F0FFF8ED6AD7
:107750000DB9002089E700BFB06900287FF4F8AEBA
:10776000012082E730000020000024404C5400201B
:107770007B2264617461223A5B7B22646576696373
:10778000654964223A222573222C222573223A2548
:10779000647D5D7D2C00000000000000E001002001
:1077A0007B2264617461223A5B7B22646576696343
:1077B000654964223A222573222C222573223A2518
:1077C000737D2C5D7D0000001CB501217820FFF742
:1077D00021FD00208DF806008DF8070002208DF8AD
:1077E000040003208DF80500012000906946E5485B
:1077F000FCF700FD0C220021E248FCF7CBFD022043
:1078000000906946DF48FCF7F5FC0C220121DD48B9
:10781000FCF7C0FD042000906946DA48FCF7EAFC5A
:107820000C220221D748FCF7B5FD082000906946DC
:10783000D448FCF7DFFC0C220321D248FCF7AAFD58
:10784000102000906946CF48FCF7D4FC0C2204219C
:10785000CC48FCF79FFD202000906946C948FCF702
:10786000C9FC0C220521C748FCF794FD4FF4805059
:1078700000906946C348FCF7BDFC0C221146C14884
:10788000FCF788FD4FF4005000906946BD48FCF7B6
:10789000B1FC0C220D21BB48FCF77CFD4FF480406D
:1078A00000906946B748FCF7A5FC0C220E21B548AC
:1078B000FCF770FD4FF4004000906946B148FCF7BA
:1078C00099FC0C220F21AF48FCF764FD01200090C9
:1078D0006946AD48FCF78EFC0C220021AA48FCF753
:1078E00059FD022000906946A748FCF783FC0C2252
:1078F0000121A548FCF74EFD042000906946A248EE
:10790000FCF778FC0C2202219F48FCF743FD08207D
:10791000009069469C48FCF76DFC0C2203219A48B4
:10792000FCF738FD1020009069469748FCF762FC90
:107930000C2204219448FCF72DFD2020009069467C
:107940009148FCF757FC0C2205218F48FCF722FDDB
:107950004FF40060009069468C48FCF74BFC0C2209
:107960000B218A48FCF716FD4FF4805000906946C1
:107970008648FCF73FFC0C2211468448FCF70AFDC0
:107980004FF40050009069468048FCF733FC0C220D
:107990000D217E48FCF7FEFC4FF4804000906946C4
:1079A0007A48FCF727FC0C220E217848FCF7F2FC01
:1079B0004FF40040009069467448FCF71BFC0C2211
:1079C0000F217248FCF7E6FC0120009069466F48E1
:1079D000FCF710FC0C2200216C48FCF7DBFC0220B9
:1079E000009069466948FCF705FC0C2201216748B4
:1079F000FCF7D0FC8020009069466548FCF7FAFB54
:107A00000C2207216248FCF7C5FC4FF480700090FF
:107A100069465F48FCF7EEFB0C2208215C48FCF746
:107A2000B9FC4FF40070009069465948FCF7E2FB3E
:107A30000C2209215648FCF7ADFC4FF48060009001
:107A400069465348FCF7D6FB0C220A215048FCF744
:107A5000A1FC4FF40060009069464D48FCF7CAFB5A
:107A60000C220B214A48FCF795FC4FF48050009003
:107A700069464748FCF7BEFB0C2211464448FCF718
:107A800089FC4FF40050009069464148FCF7B2FB76
:107A90000C220D213E48FCF77DFC4FF48040009005
:107AA00069463B48FCF7A6FB0C220E213848FCF740
:107AB00071FC4FF40040009069463548FCF79AFB92
:107AC0000C220F213248FCF765FC4FF480700090C7
:107AD00069462E48FCF78EFB0C2208212B48FCF748
:107AE00059FC4FF40070009069462848FCF782FB6F
:107AF0000C2209212548FCF74DFC4FF480600090D2
:107B000069462248FCF776FB0C220A211F48FCF745
:107B100041FC4FF48060009069461B48FCF76AFB0B
:107B20000C220A211848FCF735FC202000906946F9
:107B30001648FCF75FFB0C2205211448FCF72AFCD1
:107B40001020009069461148FCF754FB0C220421D8
:107B50000E48FCF71FFC0220009069460C48FCF719
:107B600049FB0C2201210A48FCF714FC012000907B
:107B700069460748FCF73EFB0C2200210448FCF74D
:107B800009FC1CBD0014024000180240000C024019
:107B9000001002407047000010B504460CB1012CE3
:107BA00000D103E0942103A001F03CFF0A480460E7
:107BB00010BD00002E2E5C4C6962726172696573A3
:107BC0005C7372635C73746D3332663278785F73A2
:107BD00079736366672E6300DC0027420CB50020D2
:107BE000019000902D48006840F480302B490860D7
:107BF00000BF2A48006800F4003000900198401C43
:107C00000190009818B90198B0F5A06FF1D1234800
:107C1000006800F4003010B10120009001E0002065
:107C200000900098012838D11C48083000681B4992
:107C3000083108600846006840F4004008600846C3
:107C4000006840F4A05008601548091F0860081F2C
:107C5000006840F08070091F086000BF0F4800688E
:107C600000F000700028F9D040F203700D49086060
:107C70000A480830006820F003000849083108600D
:107C80000846006840F00200086000BF0348083062
:107C9000006800F00C000828F8D10CBD0038024044
:107CA000193C4005003C024010B50446042C01D0AC
:107CB000601D00B903E0DB210BA001F0B3FE042C32
:107CC00008D14FF0E020006940F004004FF0E021BF
:107CD000086107E04FF0E020006920F004004FF059
:107CE000E021086110BD00002E2E5C4C69627261BB
:107CF000726965735C7372635C6D6973632E630094
:107D000010B507480078012808D1FDF733FEFEF7CB
:107D100083FDFDF741FE012011F0C2F910BD000006
:107D20009D00002010B51348006840F00100114983
:107D3000086000200F49083108600E4800680E49AD
:107D400008400C4908600D48091D0860081F0068BC
:107D500020F48020091F0860002006490C310860CB
:107D600000F010F8FFF73AFF4FF000600449086098
:107D700010BD000000380240FFFFF6FE1030002466
:107D800008ED00E010B5FCF701FA10BD10B50CF0DD
:107D900047F910BD10B540F22441104800F03EFAFA
:107DA000D0B10E480488001D048800210C48F9F762
:107DB00023FE0B48F9F792FE41F28831081A09496F
:107DC000086009490648F9F70BFD01210448F9F755
:107DD00013FE01200549087010BD00000014014089
:107DE0002864024058000020008800105400002041
:107DF00000B587B001210846FFF70CFA01211020D9
:107E0000FFF7EEFA07220A212948FCF7C3FA0722F6
:107E100009212748FCF7BEFA4FF4C0600190022008
:107E20008DF8080000208DF80A0001208DF80B0065
:107E300002208DF8090001A91D48FCF7DBF94FF479
:107E4000E13003900020ADF81000ADF81200ADF85D
:107E500014000C20ADF816000020ADF8180003A99E
:107E6000144800F025FB0121124800F015F94021CB
:107E7000104800F0B3F8012240F225510D4800F0FF
:107E800077FA012240F224410A4800F071FA2520D5
:107E90008DF8000000208DF801008DF8020001200F
:107EA0008DF803006846FDF777FC07B000BD0000C1
:107EB000000002400010014010B5012211030248E9
:107EC000FCF75EFC10BD0000000802401CB501215B
:107ED0000420FFF79FF94FF48050009001208DF8A7
:107EE000040000208DF806008DF8070002208DF8B0
:107EF000050069460148FCF77DF91CBD00080240F9
:107F000000B587B0FFF7E2FF01210420FFF782F9F7
:107F100001218804FFF72AFA07220B212D48FCF7DC
:107F200039FA07220A212B48FCF734FA4FF4806013
:107F3000019002208DF8080000208DF80A008DF8CD
:107F40000B0002208DF8090001A92248FCF752F924
:107F50004FF40060019002208DF8080001A91D482F
:107F6000FCF748F94FF4165003900020ADF81000CC
:107F7000ADF81200ADF814000C20ADF8160000208A
:107F8000ADF8180003A9144800F092FA0121124834
:107F900000F082F84021104800F020F8012240F261
:107FA00025510D4800F0E4F9012240F224410A482D
:107FB00000F0DEF927208DF8000000208DF8010088
:107FC0008DF8020001208DF803006846FDF7E4FB00
:107FD00007B000BD000802400048004070B50446EC
:107FE0000D461E4884420ED01D4884420BD01D48C9
:107FF000844208D01C48844205D01C48844202D0E8
:108000001B48844200D104E040F22B5119A001F03A
:1080100009FD4FF69F40284008B905B104E040F241
:108020002C5114A001F0FEFC05F40070B0F5007FA7
:1080300011D10A48844208D00948844205D0094831
:10804000844202D00A48844200D104E040F2315117
:1080500008A001F0E7FCE843208070BD001001405B
:108060000044004000480040004C004000500040E8
:10807000001401402E2E5C4C696272617269657356
:108080005C7372635C73746D3332663278785F75DB
:10809000736172742E63000070B504460D46164875
:1080A00084420ED0154884420BD01548844208D033
:1080B0001448844205D01448844202D013488442B4
:1080C00000D104E04FF4CD7111A001F0ABFC0DB173
:1080D000012D00D104E040F29B110DA001F0A2FCA3
:1080E00025B1A08940F40050A08104E0A0894DF69C
:1080F000FF710840A08170BD0010014000440040A5
:1081000000480040004C0040005000400014014076
:108110002E2E5C4C69627261726965735C73726366
:108120005C73746D3332663278785F757361727424
:108130002E63000070B505460C460026284885428F
:108140000ED0284885420BD02748854208D02748C2
:10815000854205D02648854202D02648854200D176
:1081600004E040F2FB4124A001F05CFC012C13D0A0
:10817000802C11D0402C0FD0202C0DD0102C0BD0E7
:10818000B4F5807F08D0B4F5007F05D0082C03D06B
:10819000042C01D0022C00D104E040F2FC4116A0D6
:1081A00001F040FCB4F5007F11D10D48854208D0A4
:1081B0000C48854205D00C48854202D00D488542C6
:1081C00000D104E040F201510BA001F02BFC288803
:1081D000204008B1012600E00026304670BD0000B6
:1081E000001001400044004000480040004C0040A6
:1081F00000500040001401402E2E5C4C69627261F8
:10820000726965735C7372635C73746D333266326A
:1082100078785F75736172742E6300002DE9F04702
:1082200005460C4600270026B046B1464148854227
:108230000ED0414885420BD04048854208D0404886
:10824000854205D03F48854202D03F48854200D153
:1082500004E040F24F513DA001F0E4FB282C27D070
:1082600040F22770844223D040F2266084421FD01F
:1082700040F2255084421BD040F22440844217D063
:1082800040F64600844213D040F66A1084420FD074
:10829000B4F5587F0CD040F22530844208D0B4F5B4
:1082A000587F05D0B4F5187F02D0B4F5B07F00D167
:1082B00004E04FF4AA6125A001F0B4FB40F66A1077
:1082C000844211D11B48854208D01B48854205D005
:1082D0001A48854202D01C48854200D104E040F291
:1082E00055511AA001F09EFBC4F3421804F01F067A
:1082F000012000FA06F6B8F1010F02D1A889064064
:1083000007E0B8F1020F02D1288A064001E0A88AEE
:1083100006402712012000FA07F7288807401EB1FF
:1083200017B14FF0010901E04FF000094846BDE8E0
:10833000F087000000100140004400400048004069
:10834000004C004000500040001401402E2E5C4CB8
:1083500069627261726965735C7372635C73746D78
:108360003332663278785F75736172742E63000001
:108370002DE9F04704460D4617464FF00008C24667
:10838000C14600263B4884420ED03B4884420BD075
:108390003A48844208D03A48844205D03948844259
:1083A00002D03948844200D104E040F2BC4137A0F9
:1083B00001F038FB282D19D040F22770854215D0E6
:1083C00040F22660854211D040F2255085420DD002
:1083D00040F22440854209D040F64600854205D04F
:1083E00040F66A10854201D0602D00D104E040F2D1
:1083F000BD4126A001F016FB0FB1012F00D104E012
:1084000040F2BE4121A001F00DFB40F66A1085420A
:1084100011D11848844208D01748844205D0174823
:10842000844202D01848844200D104E040F2C341A3
:1084300016A001F0F7FA2646C5F3421805F01F0A08
:10844000012000FA0AF9B8F1010F01D10C3605E05C
:10845000B8F1020F01D1103600E0143627B13068B0
:1084600040EA0900306003E0306820EA090030602B
:10847000BDE8F08700100140004400400048004083
:10848000004C004000500040001401402E2E5C4C77
:1084900069627261726965735C7372635C73746D37
:1084A0003332663278785F75736172742E630000C0
:1084B0002DE9FF4705460C460026B14600BFB046F1
:1084C0006D4885420ED06D4885420BD06C48854280
:1084D00008D06C48854205D06B48854202D06B4875
:1084E000854200D103E0EA2169A001F09BFA2068EF
:1084F00020B170492068884200D203E0EB2164A0DB
:1085000001F090FAA08818B1A088B0F5805F00D182
:1085100003E0EC215EA001F085FAE08858B1E08824
:10852000B0F5805F07D0E088B0F5005F03D0E08849
:10853000B0F5405F00D103E0ED2155A001F072FAE3
:10854000208938B12089B0F5806F03D02089B0F53B
:10855000C06F00D103E0EE214DA001F063FA608905
:108560004FF6F371084010B9608900B103E0EF21C4
:1085700047A001F057FAA08958B1A089B0F5807FD3
:1085800007D0A089B0F5007F03D0A089B0F5407F67
:1085900000D103E0F0213EA001F044FAA08980B1AF
:1085A0003548854208D03548854205D03448854253
:1085B00002D03648854200D103E0F52134A001F015
:1085C00031FA2E8A26F44056E08806432E82AE8980
:1085D00041F20C608643A0882189084361890843E1
:1085E0000643AE81AE8A26F44076A0890643AE8269
:1085F0006846FEF72FFF2048854202D02348854277
:1086000002D1DDF80C9001E0DDF80890A88900F4B3
:10861000004040B109EBC90000EB09102168490096
:10862000B0FBF1F707E009EBC90000EB0910216886
:108630008900B0FBF1F76420B7FBF0F006013009C8
:10864000642101FB1078A88900F4004040B1322079
:1086500000EBC800B0FBF1F000F00700064308E0B3
:10866000322000EB08106421B0FBF1F000F00F00A5
:1086700006432E81BDE8FF87001001400044004002
:1086800000480040004C00400050004000140140F1
:108690002E2E5C4C69627261726965735C737263E1
:1086A0005C73746D3332663278785F75736172749F
:1086B0002E630000E170720010B504460D4884423C
:1086C0000ED00D4884420BD00C48844208D00C4890
:1086D000844205D00B48844202D00B48844200D12A
:1086E00004E04FF40B7109A001F09CF9A088C0F3DD
:1086F000080010BD00100140004400400048004048
:10870000004C004000500040001401402E2E5C4CF4
:1087100069627261726965735C7372635C73746DB4
:108720003332663278785F75736172742E6300003D
:1087300070B504460D46124884420ED0114884425A
:108740000BD01148844208D01048844205D010480C
:10875000844202D00F48844200D104E04FF40771F4
:108760000DA001F05FF9B5F5007F00DA04E040F2FA
:108770001D2109A001F056F9C5F30800A08070BDC5
:10878000001001400044004000480040004C004000
:1087900000500040001401402E2E5C4C6962726152
:1087A000726965735C7372635C73746D33326632C5
:1087B00078785F75736172742E63000000BFFEE706
:1087C0002DE9F14F86B007F03DFF05900598D0F8F0
:1087D000E870069801F0C0F904904AA1049801F0ED
:1087E00087F9044601F096F9039049A1049801F035
:1087F00088F9804648A1049801F083F9814648A190
:10880000049801F07EF9824647A1049801F079F9B5
:1088100083466EE0781C0090B86944684FF4617636
:1088200003990098F7F7A4FD002860D1B3B20022A5
:1088300011461046FDF7B2FFFDF79CF8B8F1000FA6
:1088400011D0A578608B0290B8F8140080B2019026
:108850002846DDE901210BF0A3FDB3B20022114649
:108860001046FDF79BFFB9F1000F12D0246AA578DE
:10887000608B0290B9F8140080B201902846DDE9BF
:1088800001210BF08DFDB3B2002211461046FDF719
:1088900085FFBAF1000F12D0246AA578608B029090
:1088A000BAF8140080B201902846DDE901210BF0EE
:1088B00077FDB3B2002211461046FDF76FFFBBF102
:1088C000000F12D0246AA578608B0290BBF81400C8
:1088D00080B201902846DDE901210BF061FDB3B2C1
:1088E000002211461046FDF759FFFDF755F8FF69C4
:1088F00000BF002F8ED1049801F0CEF807B0BDE87C
:10890000F08F0000646576696365496400000000CB
:10891000706F77657200000074656D700000000074
:108920006D6F64650000000066616E000FB4054B5A
:1089300010B503A9044A029800F0EEF910BC5DF8E6
:1089400014FB00002D040108040200200FB4084BA2
:1089500010B504A902AA039800F0DEF9044602A9A2
:10896000002000F05CFD204610BC5DF814FB000008
:108970001F940008490050EAC12018BF04204A0D86
:1089800018BF40F0010040F2FF72B2EB515F08BF28
:1089900040F00200012808BF0520704700487047DA
:1089A0001002002030B528B1144C031F00202168AC
:1089B0000A4605E0084630BD9A4203D81046526880
:1089C000002AF9D1002800D041680BD00468A3EB3D
:1089D0000005A54204D11B681C440346046002E064
:1089E000436000E023603AB11C68D51AA54203D168
:1089F00015682C441C6052685A6030BD0802002083
:108A00002DE9F0414F1E00EBC7010446D1E90001FA
:108A100015461E4637F006020DD02A463346F8F7B3
:108A20009CF87F1E04EBC703D3E90023F7F7EEFFA2
:108A300037F00602F1D1022F25D0042F13D0062FD4
:108A400018BFBDE8F0812A463346F8F786F8D4E926
:108A50000A23F7F7DBFF2A463346F8F77EF8D4E916
:108A60000823F7F7D3FF2A463346F8F776F8D4E918
:108A70000623F7F7CBFF2A463346F8F76EF8D4E91A
:108A80000423F7F7C3FF2A463346F8F766F8D4E91C
:108A90000223F7F7BBFF2A463346F8F75EF8D4E91E
:108AA0000023BDE8F041F7F7B1BF00002DE9F04722
:108AB00082460F4C10480D4E0E4F001B4FF0000821
:108AC00020F007054FF0010900221146504608F03A
:108AD00019FD002802D1306810B10020BDE8F087F0
:108AE0003C60C4E90058C6F80090EDE70C02002095
:108AF000F486012008020020F0A60120002213467F
:108B000010460149F8F79BB80000F03FF7F77EBF29
:108B10000022134610461146F8F791B840F2013290
:108B200000204FF0E041F8F765BB0000024A00204A
:108B30001107F8F75FBB000001FDFFFF02E008C866
:108B4000121F08C1002AFAD170477047002001E0C7
:108B500001C1121F002AFBD17047000001490860C3
:108B6000704700001002002010B50246002003E00C
:108B700012F8014B2318D8B20B1EA1F10101F7D155
:108B800010BD00002DE9FF5F82B00021DDE9043057
:108B9000020DDDF840B0034318D044F61050A2F2A5
:108BA000FF3242431514119801281FD0A5EB0B008A
:108BB000401C5FEA000A4FF000064E4FDFF8389184
:108BC000B046504615D5CAF1000413E011980124AF
:108BD0004AA3012801D16FEA0B010298119AC0E95A
:108BE0000031C0E9024206B0BDE8F09FCBF10000C1
:108BF000DFE704460021404A491842EB0450CDE922
:108C0000001012E0E00707D032463B464046494696
:108C1000F7F7A3FF8046894632463B461046194681
:108C2000F7F79BFF06460F466410002CEAD1DDE9FA
:108C30000401DDE90023BAF1000F06DAF7F78DFF32
:108C400042464B46F7F789FF05E0F7F7F8FF424643
:108C50004B46F7F7F4FF04460E460022284BF8F780
:108C6000CBF803D84FF0FF30014607E00022254B38
:108C700020463146F7F7CAFEF8F7DFFA102409E07C
:108C8000002C0ADB0A220023F7F7F2FA039B3032AA
:108C90001A55641E50EA0102F2D1641C039AC4F111
:108CA00011031444119A012A03D0012208430DD163
:108CB0000AE0084304D000204FF0110B119072E736
:108CC000A3EB0B056D1E0DE05B4504DD4FF00002CC
:108CD00005F1010504E003DA4FF00002A5F10105FA
:108CE000002AECD002981199C0E90231C0E9004590
:108CF00079E70000000014400000F03F3000000061
:108D00000000F0430000E03F30380A2801D2012083
:108D100070470020704700002DE9FF4F95B09A463C
:108D2000884606460025EEE1252877D1002427460F
:108D3000F94A0121039400E0044316F8013F203B67
:108D400001FA03F01042F7D130782A2811D06FF0E1
:108D50002F033078A0F13002092A16D8039A44F084
:108D6000020402EB820203EB42021044761C0390E1
:108D7000EFE758F8042B0392002A03DA504244F438
:108D80000054039044F00204761C30782E2816D14B
:108D900016F8010F44F004042A280DD06FF02F02BA
:108DA0003078A0F13003092B09D807EB870302EBD9
:108DB0004303C718761CF3E758F8047B761C307819
:108DC0006C280FD006DC4C2817D068280DD06A28F4
:108DD00014D104E0742810D07A280FD10DE044F4A7
:108DE00000140AE044F4801401E044F44014727862
:108DF000824202D104F58014761C761C30786628F5
:108E00000BD013DC582877D009DC002875D0452812
:108E1000F6D04628F4D047281AD193E118E0632809
:108E200035D0642879D0652812D18BE1702873D0B1
:108E300008DC6728F1D069286FD06E280DD06F2824
:108E400006D1ACE073282CD0752874D0782853D084
:108E50005246179990476D1C54E1C4F30250022802
:108E600009D003280DD0D8F8001004280DD00D60CB
:108E700008F1040846E1D8F80010EA17C1E90052E9
:108E8000F6E7D8F800100D80F2E70D70F0E718F85B
:108E9000041B8DF8001000208DF80100EB46012026
:108EA00003E058F804BB4FF0FF3061074FF00001BA
:108EB00002D40DE009F101018946B9420FDA81457A
:108EC000F8DB1BF809100029F4D108E009F10101D1
:108ED00089468142FADB1BF809100029F6D1039874
:108EE0005346A0EB090721463846179A00F080FA4E
:108EF000284400EB090507E044E008E10DE01BF819
:108F0000010B524617999047B9F10109F7D2534620
:108F100021463846179AF2E039E00A21C4F302529A
:108F20004FF0000B0091022A06D058F8040BC1172D
:108F3000032A09D00AE023E008F1070020F0070225
:108F4000F2E80201904605E000B2C117042A01D1FF
:108F500040B2C117002906DA0A460021404261EBFF
:108F600002012D2202E0220504D52B228DF80420D7
:108F7000012203E0E20701D02022F7E7914657E003
:108F80000A2100E010214FF0000B00910BE01021AE
:108F90004FF0000B44F004040827009103E0082080
:108FA0004FF0000B0090C4F30252022A05D058F88B
:108FB000040B0021032A08D008E008F1070020F084
:108FC0000702F2E80201904603E080B2042A00D1D1
:108FD000C0B24FF0000922072AD53278702A07D094
:108FE000DDF800C08CF0100C5CEA0B0C05D00EE034
:108FF00040228DF80420012208E050EA010306D047
:1090000030238DF804308DF8052002229146009B14
:1090100083F0080353EA0B030AD150EA010201D19D
:10902000620705D530228DF804204FF001097F1E1C
:109030003278582A04D039A20C920CAA02920BE082
:109040003BA2F9E75B46009AF7F712F90C9B9B5C91
:10905000029A521E0292137050EA0102F2D1029853
:1090600004A9081A00F1200B600702D524F480340B
:1090700000E001275F4502DDA7EB0B0000E00020C8
:1090800000EB0B01009003984944401A0390E00361
:1090900006D453462146179A039800F0A9F90544CF
:1090A000002706E001A85246C05D179990476D1C45
:1090B0007F1C4F45F6DBE0030CD553462146179A3B
:1090C000039800F095F9054404E0302052461799C2
:1090D00090476D1C0099481E00900029F5DC08E0BF
:1090E0000298029952460078491C029117999047BC
:1090F0006D1CBBF10001ABF1010BF1DC5BE100F099
:1091000065F90544761C307800287FF40DAE19B05F
:109110002846BDE8F08F00000928010030313233C5
:1091200034353637383961626364656600000000A3
:10913000303132333435363738394142434445468D
:1091400000000000600700D4062708F1070020F0A7
:109150000700F0E80223804603F0004C5FEA0C00B1
:1091600001D097A009E0200501D596A005E0E00711
:1091700001D095A001E0AFF24C001390307823F0BD
:10918000004365280CD006DC452809D046281DD0B0
:1091900047287FD13BE0662818D067287AD136E08F
:1091A0000021112F01DB112000E0781CCDE9000126
:1091B00004A90CA8FFF7E6FCDDE90D010C9A4FF0BD
:1091C000000B07F10109109200914EE04FF00040B2
:1091D0000097CDE9011004A90CA8FFF7D3FCDDE945
:1091E0000D020C9B0F994FF0000B914610930092CB
:1091F00011B9791C00EB0109B7EB090003D4C0F1E8
:10920000FF3B07F10109A9EB0700019042E0012FA4
:1092100000DA01270021112F01DD112000E038467E
:10922000CDE9000104A90CA8FFF7ACFCDDE90D01B4
:109230000C9A00914FF0000BB946109221070FD401
:10924000009A4A4503DA914601E0A9F10109B9F112
:10925000010F05DD109AA9F10101515C3029F4D00C
:10926000B84202DA10F1040F03DA0121CDE901104E
:1092700010E0002803DC8344A9EB000102E0411C5C
:10928000494500DD8946A0EB0B00401C01904FF0E2
:1092900000400290200705D40198484502DB4FF0BA
:1092A000FF30019000208DF84B0002980DF14B0724
:1092B000B0F1004F25D002200C902B200D90029889
:1092C00000280CDA404202902D200D9007E00A2180
:1092D0000298F7F7C5FD3031029007F8011D0C998F
:1092E000481E0C900029F2DC02980028EFD1791E6C
:1092F0000D980870307800F0200040F0450007F825
:10930000020D11A8C01BC01D02901398007800B177
:10931000012000EB0901019801EBE0710298014482
:109320000398401A401E0390E00306D4534621469A
:10933000179A039800F05CF805441398007818B168
:109340005246179990476D1CE00323D5534621469A
:10935000179A039800F04CF805441BE0BBF1000F8E
:1093600007DB0098584504DD1098179910F80B009A
:1093700001E0179930205246904701980BF1010BFC
:10938000401E05F10105019004D12E205246179987
:1093900090476D1CB9F10001A9F10109DEDC05E07F
:1093A00017F8010B5246179990476D1C0299481EF9
:1093B00002900029F4DC53462146179A03989EE652
:1093C0002D0000002B000000200000002DE9F041DE
:1093D000044600251E461746880404D405E0394695
:1093E0002020B0476D1C641EF9D52846BDE8F081E9
:1093F0002DE9F041044600251E469046C80301D5DC
:10940000302700E02027880404D505E0414638468F
:10941000B0476D1C641EF9D52846BDE8F0810A6886
:10942000531C0B601070704770B506460D46242023
:10943000FFF73CFB0446621D13A130460CF044FFCD
:1094400015A130460CF02BFFE07018A130460CF04F
:1094500026FFA07019A130460CF021FF60831CA1EB
:1094600030460CF01CFF2080A869406810B9A8693C
:10947000446008E0A969486800E0006A016A0029C0
:10948000FBD1046200BF70BD226964656E746966B9
:10949000696572223A220000227746756E6374690C
:1094A0006F6E436F6465223A0000000022736C61A6
:1094B000766541646472657373223A00227265674F
:1094C000697374657241646472657373223A000053
:1094D000227265676973746572427974654E756D41
:1094E000223A000070B5064635462020FFF7DEFA26
:1094F00004460020E06136A130460CF0D0FE6075D5
:1095000036A130460CF0CBFEE07537A130460CF0AA
:10951000C6FEA075621C39A130460CF0D5FE0C20A9
:10952000FFF7C4FAA06139A12846F6F708FF0546FF
:1095300011E02146284600F047F900BF37A1284630
:10954000F6F7FDFE0546412028706D1C28785D2841
:1095500001D1354600E0ECE700BF607D032824D14F
:10956000354621A128460CF09AFEA0751BA128467D
:109570000CF095FEE0752AA12846F6F7E0FE0546B8
:109580009DB110E021462846FFF74EFF23A1284653
:10959000F6F7D5FE0546412028706D1C28785D2819
:1095A00001D1354600E0EDE700BF2148D0F8E800E2
:1095B00018B91F48C0F8E84009E01D49D1F8E80093
:1095C00000E0C069C1690029FBD1C46100BF70BD62
:1095D0002270726F746F636F6C223A002264617440
:1095E0006154797065223A00226269674C6974742B
:1095F0006C65466F726D6174223A00002264657674
:109600006963654964223A22000000002273656E96
:10961000736F7244617461223A5B00007D00000048
:1096200022636F6D6D616E6444617461223A5B0008
:10963000347A002070B5054633A128460CF02FFE81
:109640003349C88233A128460CF029FE304981F8FD
:10965000F20033A128460CF022FE2D4981F8F000DB
:1096600032A128460CF01BFE2949C1F8EC0032A1BA
:1096700028460CF014FE264981F8F10031A1284655
:109680000CF00DFE2249C1F8C4004A1C31A1284645
:109690000CF01AFE1E4AA43231A128460CF014FE2A
:1096A0001B4A4A3232A128460CF00EFE184A1832E4
:1096B00034A128460CF008FE154A7C3236A1284613
:1096C0000CF002FE124A903237A128460CF0FCFD45
:1096D00039A12846F6F733FE044611E07CB1204656
:1096E000FFF700FF00BF37A12046F6F728FE04462B
:1096F00041202070641C20785D2801D101E070BDFC
:10970000ECE700BF00BFFAE722706F7274223A00E4
:10971000347A00202273746F70426974223A000018
:109720002264617461426974223A000022626175A8
:109730006472617465223A0022636865636B4269F2
:1097400074223A0022696E626F756E6454696D65A9
:10975000223A000022686F7374223A22000000004F
:10976000226465766963654964223A22000000003C
:1097700022636F6D6D616E64546F706963223A226B
:1097800000000000226D657373616765546F706936
:1097900063223A220000000022757365726E616DCB
:1097A00065223A22000000002270617373776F72A5
:1097B00064223A22000000006465766963654C69A2
:1097C000737400007D0000002DE9F84380460C46CC
:1097D000607D012804D0022803D003286ED13AE02E
:1097E00000BF3020FFF762F9054636A140460CF075
:1097F00056FDE861AA1D38A140460CF065FD0D211B
:1098000000200BF0F9FD07463A4637A140460CF020
:109810005BFD002609E007EB46006A4636A1F6F735
:10982000DBFD9DF80000A855761C062EF3DB3946BB
:1098300000200BF0CFFDA069806810B9A069856099
:1098400008E0A169886800E0C06AC16A0029FBD10C
:10985000C56200BF33E02820FFF728F90546AA1C9F
:109860001DA140460CF030FD25A140460CF017FD2F
:1098700085F8200025A140460CF011FD687028A154
:1098800040460CF00CFD287029A140460CF007FD65
:10989000E8822CA140460CF002FDE883A069006834
:1098A00010B9A069056008E0A169086800E0406A95
:1098B000416A0029FBD1456200BF00E000BF00BF44
:1098C000BDE8F883226964656E74696669657236FD
:1098D0003435223A00000000226964656E746966BE
:1098E000696572223A2200002264657669636549DF
:1098F00044363435223A2200253268687800000068
:109900002270726563697365223A0000227246759F
:109910006E6374696F6E436F6465223A00000000E5
:1099200022736C61766541646472657373223A00D8
:1099300022726567697374657241646472657373DA
:10994000223A000022726567697374657242797405
:10995000654E756D223A00002DE9F04105460E4630
:10996000002447E0F6F72CFC074604EB44002449AA
:1099700051F83000C8BB04EB440041F83050384681
:10998000F6F722FC002004EB44011D4A02EBC10162
:10999000486004EB440102EBC101088104EB44017F
:1099A00002EBC10148812878102804D10EB10120B2
:1099B00002E0002000E0012004EB4401104A02EB29
:1099C000C1018881002004EB440102EBC101C88180
:1099D00004EB440102EBC101086104EB440102EB1A
:1099E000C10148612046BDE8F081FFE73846F6F73F
:1099F000EBFB641C082CB5DB4FF0FF30F3E70000F5
:109A0000C05B012010B5044600BF00BF05F004F99B
:109A10000022034941F288300FF032FA10BD0000F5
:109A2000059A00087047000010B50246002309E0BF
:109A3000064800680078107004480068401C034C19
:109A400020605B1C8B42F3DB084610BDA8010020A0
:109A5000014609B1086808B90020704719B1D1E979
:109A60000120904201D30846F7E702E08868401CD5
:109A7000886041B1D1E90120904204D28A68086827
:109A8000805C2028F2DDD1E90120904202D1886873
:109A9000401E88600846E0E770B50446002522E0D5
:109AA0002568A08900F4807020B9A06810B1A06872
:109AB000FFF7F2FFA08900F4807028B9206918B17F
:109AC0000A4A206951688847A08900F4007028B9C3
:109AD000206A18B1054A206A5168884703484168DE
:109AE000204688472C46002CDAD170BDBC010020EE
:109AF00070B504460D4600222946204606F0CBFDEF
:109B000070BD70B504460D4601222946204606F078
:109B1000C2FD70BD00B50246104600F005F808B958
:109B2000002000BD1069FCE7014609B9002070471C
:109B3000087B102801D10120F9E70020F7E770B574
:109B4000044628202168884705461DB1282128465B
:109B5000F6F7DEFB284670BD10B50446002211461C
:109B6000204600F06BF810BD2DE9F0478AB004469E
:109B70000E46154698461C2103A8F6F7C9FB002798
:109B800000202C490860486004B106B932E0039413
:109B9000049600200590284A07CA07AB07C3264849
:109BA000FFF7CDFF074607B924E003A80EF072FFC8
:109BB0008246FFF74DFF8146494638460CF04AFE83
:109BC00000B917E0B8F1000F0BD003A8FFF740FF72
:109BD000DDE90410884203D205990398405C00B186
:109BE00008E01DB1059903980844286038460AB07A
:109BF000BDE8F08717B13846FFF74EFFC4B10194B6
:109C000000200290DDE90410884202D205980290FB
:109C100004E0049810B10498401E02901DB1DDE9E3
:109C20000101084428600348DDE9011206C000BFB5
:109C30000020DCE7B4010020BC0100202DE9F04148
:109C400004460D46164614B90020BDE8F0812046B2
:109C5000F6F787FB471C33462A4639462046FFF76E
:109C600083FFF2E770B504460D4604B10DB901203B
:109C700070BDAC4201D10020FAE705E0207808B9B8
:109C80000020F5E7641C6D1C2078F6F722FB0646E1
:109C90002878F6F71EFB8642F0D02078F6F719FBFD
:109CA00006462878F6F715FB301AE1E770B504464A
:109CB0000D4600202071401EE062294620460AF031
:109CC000B1FB08B1032070BD94F82E1294F82F0256
:109CD00041EA00204AF65521884201D00220F2E7ED
:109CE00094F86900010694F8680041EA004194F88C
:109CF000670041EA002094F86610084320F07F4096
:109D00000D49884201D10020DDE794F88500010665
:109D100094F8840041EA004194F8830041EA00206D
:109D200094F88210084320F07F400349884201D113
:109D30000020C8E70120C6E746415400024600E083
:109D4000521C107810B110788842F9D11078704701
:109D500030B502460B4600200446014621E001EBE7
:109D600041001D4D55F82000C8B101EB410055F8E8
:109D700020001568A84213D101EB4100164D05EBF8
:109D8000800040689568A8420AD101EB4100124D5D
:109D900005EB80000089D588A84201D103E00124A9
:109DA000491C0329DBD300BF032906D10CB9022BC0
:109DB00001D1002030BD1220FCE743B901EB410086
:109DC000054D05EB80004089B0F5807F01D1102062
:109DD000F0E70020EEE700002CE3002010B501467C
:109DE00000200DE000EB4002074B53F822208A428E
:109DF00005D1002200EB4003034C44F82320401C13
:109E00000328EFD310BD00002CE300200246891E7A
:109E10005069801E884201D8002070479378906A6C
:109E200001FB0300F9E700002DE9F04705460C4669
:109E3000207820F04000401E00EB800101EBC006BE
:109E400000274FF0010800BF1A48C05D205C194987
:109E5000C95D2144497840EA0129B8F1000F10D0CA
:109E6000484606F079F88046FF2E07D23146761C28
:109E700035F8110006F070F8404508D00020BDE824
:109E8000F0874FF6FF70814501D00020F7E7781C7E
:109E900007460D28D8D3207800F0400038B1B8F13B
:109EA000000F04D035F8160008B10020E7E70120C4
:109EB000E5E70000948404082DE9F047044689464C
:109EC000B9F1000F06D1E76817B16069B84215D83B
:109ED000012713E04946204606F03CFB0646022EC9
:109EE00002D20120BDE8F087701C08B93046F9E7BE
:109EF0006069B04201D93046F4E74F463D4600BFA5
:109F00006D1C6069A84204D80225BD4201D9002019
:109F1000E8E72946204606F01DFB064606B909E09B
:109F2000701C08B1012E01D13046DBE7BD42E7D1FC
:109F30000020D7E700BF6FF07042294620460EF0A0
:109F40001FF98046B8F1000F08D1B9F1000F05D014
:109F50002A46494620460EF013F98046B8F1000F14
:109F60000BD1E5602069401C78B12069401E20615A
:109F7000607940F00100607107E0B8F1010F02D193
:109F80004FF0FF3000E0012005462846AAE7000018
:109F90002DE9F34F83B0814604980068019002E0F8
:109FA0000198401C0190019800782F28F8D0019862
:109FB00000785C28F4D0D9F820A000252F4600BFF7
:109FC00038467F1C01990C5C202C03DB2F2C01D020
:109FD0005C2C00D132E0FF2D03D3062005B0BDE894
:109FE000F08FE4B2812C13DBE0B2FE2810DC38469F
:109FF0007F1C01990E5C402E01DB7E2E05DD802E3C
:10A0000001DBFE2E01DD0620E8E706EB042084B22A
:10A010000121204605F062FF04460CB90620DDE769
:10A02000802C06DA214671A0FFF788FE08B10620D1
:10A03000D4E728466D1C2AF81040C1E700BF0198FC
:10A04000C11904980160202C01DA042000E00020EE
:10A05000804608E0681E3AF81040202C02D02E2CD2
:10A0600000D002E06D1E002DF4D100BF0DB9062016
:10A07000B4E700202AF815000B222021D9F8180097
:10A0800009F054FE002700E07F1C3AF81700202852
:10A09000FAD03AF817002E28F6D00FB148F003088E
:10A0A00000E06D1E25B1681E3AF810002E28F8D188
:10A0B0000020064602904FF0080B00BF38467F1C78
:10A0C0003AF8104004B963E0202C03D02E2C04D1C0
:10A0D000AF4202D048F00308F0E70298584501D299
:10A0E000AF4214D1BBF10B0F02D148F003084FE08F
:10A0F000AF4201D048F00308AF4200D948E02F46F4
:10A10000082002904FF00B0BB006060ED6E7802C0D
:10A1100009DB204605F020FF0021009005F0DEFE5F
:10A12000044648F00208FF2C11DDABF10100029952
:10A13000884204D848F00308CDF808B0BEE72212E0
:10A14000D9F818300298411C02911A5419E024B130
:10A15000214629A0FFF7F2FD18B15F2448F003085B
:10A160000FE0412C04DB5A2C02DC46F0020608E02A
:10A17000612C06DB7A2C04DC46F00106A4F12000F9
:10A1800084B2D9F818300298411C02911C5495E70A
:10A1900000BFD9F818000078E52803D10520D9F8C8
:10A1A00018100870BBF1080F01D1B006060E06F0BA
:10A1B0000C000C2803D006F00300032801D148F05E
:10A1C000020808F0020058B906F00300012801D186
:10A1D00048F0100806F00C00042801D148F00808E7
:10A1E000D9F8180080F80B800020F7E6222A3A3CC4
:10A1F0003E3F7C7F000000002B2C3B3D5B5D000060
:10A200002DE9F04F8BB00446894600250026AA466A
:10A21000AB4669E04FF0010A00BFBAF1010F03D06D
:10A22000BAF1020F5AD12DE02846F6F78DFD02460D
:10A230000B46CDE90001002031490DF0B5FA074683
:10A240008846A15DC91E01F00F00F6F76CFD3A4685
:10A250004346CDE90201F6F780FCCDE906015846F8
:10A26000F6F761FDCDE90401DDE90623F6F7CEFB43
:10A27000CDE90801F6F775FD8346681CC5B24FF0BD
:10A28000020A2BE02846F6F75FFD02460B46CDE9B1
:10A29000000100201A490DF087FACDE90201A15D05
:10A2A00033390811F6F73FFD0746DDE90223F6F7DB
:10A2B00054FCCDE906015846F6F735FDCDE9040119
:10A2C000DDE90623F6F7A2FBCDE90801F6F749FD23
:10A2D0008346681CC5B24FF0000A00BF00BFBAF148
:10A2E000000F9AD1701CC6B2B9F10000A9F10101AA
:10A2F0001FFA81F98ED158460BB0BDE8F08F0000EF
:10A30000000024402DE9FF5F064600BF012009F050
:10A31000DDFE4FF4105101200BF06EF8039023A0E6
:10A3200003990EF0F3F80398FFF784F901200399DD
:10A330000BF050F806F086F904460020029054F81D
:10A34000E85F676894F8088094F80A9094F80DA084
:10A3500094F80BB0E83C53464A4641463846CDF89F
:10A3600000B0F7F7ABF91CE02846FDF7E7F8E8691D
:10A3700008B1ED6915E01048019010480068012807
:10A3800004D101A90E480068FBF70EFC0D48F5F753
:10A39000E8FF014600900B48F5F7BAFFD4F8E85003
:10A3A00000BF002DE0D1BDE8FF9F00006465766925
:10A3B00063652E7478740000030000201C000020E8
:10A3C000180000204C54002030B50246531E1A4697
:10A3D000032B1BD202EB42030D4C04EB8303598980
:10A3E000B1F5807F00D1002109B14B1E99B202EB7B
:10A3F0004203074C04EB8303598129B9002302EB84
:10A400004204034D45F82430002000E0022030BD16
:10A410002CE3002010B56FF00400FDF745FC104858
:10A4200000681049B0FBF1F00F4908700C48006853
:10A430000C49B0FBF1F44FF47A70444301200B490E
:10A4400008804FF0E020006940F002004FF0E0216A
:10A45000086108464461006940F00100086110BDD0
:10A460000000002000127A005E0000206000002042
:10A4700070B504460F480078A0B10F48007888B93D
:10A480000E480088844206DB0C48008894FBF0F5F7
:10A49000284600F01DF80948008894FBF0F100FB05
:10A4A000114084B24FF47A7104FB01F000F016F809
:10A4B00070BD00009D00002094000020600000207E
:10A4C00010B5FBF745FD10BD10B5FBF761FD10BDE4
:10A4D00010B504462046FCF725F910BD2DE9F047DC
:10A4E000074600264FF0E020D0F81490114800787D
:10A4F00007FB00F800BFFFF7E3FF4FF0E02085699E
:10A5000011E04FF0E0208469AC420CD0AC4202D2A2
:10A51000281B064403E0A9EB040028440644254612
:10A52000464500D300E0ECE700BFFFF7CDFFBDE8F4
:10A53000F08700005E00002070B504460D4600BFA5
:10A540001CB90DA0FEF7F2F970BD00BF00BF00BF3F
:10A55000606A78B1606A007B08280BD100BF00BF39
:10A560002868616A496A884204D100BF00BF20465A
:10A5700000F020FA00BFE7E76E6574696620213DB0
:10A58000204E554C4C0000007CB5064600BF1EB95D
:10A5900041A0FEF7CBF97CBD00BF746A00BF1CB9B7
:10A5A00044A0FEF7C3F9F6E700BF00BF00BF606B31
:10A5B000401C90B100BF00BF606B1E303C21B0FB5F
:10A5C000F1F5B5F5803F01D34FF6FF75A583A08B5C
:10A5D00008B90120A08300BF00BFA06B401C90B150
:10A5E00000BF00BFA06B1E303C21B0FBF1F5B5F5FC
:10A5F000803F01D34FF6FF75E583E08B08B901205A
:10A60000E08300BF00BFA08BE18B884204DBE08BBE
:10A61000002801DD0020A083A07B10B1A06A01907A
:10A6200010E094F824007F2802DCFF21019108E06B
:10A63000C02803DB6FF07F41019102E04FF6FF710C
:10A64000019100BFE06A0090684608B1009838B9EF
:10A65000606A019908400090009840F08070009076
:10A6600000BF00BF04F1240130460BF073FD00BFB2
:10A6700000BF01A930460BF0EFFD00BF00BF6946E7
:10A6800030460BF05EFD30460BF0EEFD0A21204611
:10A6900001F036F900BF7EE7646863705F62696E3F
:10A6A000643A206E6574696620213D204E554C4CFD
:10A6B00000000000646863705F62696E643A206441
:10A6C00068637020213D204E554C4C002DE9F0412F
:10A6D0000646746A00BF00BF0821204601F010F949
:10A6E000002204F12401304604F0C4F805460DB1FF
:10A6F00000BF00BF607B401C60734FF4FA7707F225
:10A70000F310394690FBF1F0608300BF00BFBDE855
:10A71000F081000010B51248046800BF00BF1BE0C4
:10A72000606AC0B1606AC18B481E626AD083012929
:10A7300005D100BF00BF204601F0E4F90BE0606ADC
:10A74000818B481E626A9083012904D100BF00BF3B
:10A75000204601F0C3F92468002CE1D110BD0000AF
:10A76000080100202DE9F04106460C46174600BFBF
:10A7700036B95AA0FEF7DAF86FF00D00BDE8F081A7
:10A7800000BF00BF2CB95DA0FEF7D0F86FF0050048
:10A79000F4E700BF00BF206910B160A0FEF7C6F863
:10A7A00000BF00BF606910B166A0FEF7BFF800BF30
:10A7B00000224FF49A7110460CF0EAF820612069EB
:10A7C00020B900BF00BF4FF0FF30D7E700BF2069BE
:10A7D0004089B0F59A7F02D264A0FEF7A7F800BFC7
:10A7E000607B20B971480068401C704908606F4860
:10A7F0000068206000BF00BF2069406860610120E0
:10A80000616908706169487096F82A00616988700A
:10A8100000206169C870206808F040FB61694860E9
:10A82000002061690881616948816169C860082FF9
:10A8300009D0042F07D0032F08D1207B052802D090
:10A84000207B042802D170686169C86000206169BA
:10A850000861616948616169886100250DE096F8C9
:10A860002A00A84203DD06F12B00405D00E0002035
:10A8700061691C314855681C85B2102DEFD3002545
:10A8800005E0002160692C304155681C85B2402DDF
:10A89000F7D3002505E0002160696C304155681C44
:10A8A00085B2802DF7D342486169C1F8EC000020E1
:10A8B0002083002504E06069F0304555681C85B2AE
:10A8C000442DF8D301223521204600F067FA39469D
:10A8D000204600F081FA002050E7000064686370B1
:10A8E0005F6372656174655F6D73673A206E65744E
:10A8F000696620213D204E554C4C00006468637011
:10A900005F6372656174655F6D73673A2064686345
:10A910007020213D204E554C4C000000646863704F
:10A920005F6372656174655F6D73673A2064686325
:10A93000702D3E705F6F7574203D3D204E554C4C20
:10A9400000000000646863705F6372656174655F36
:10A950006D73673A20646863702D3E6D73675F6F37
:10A960007574203D3D204E554C4C0000646863706A
:10A970005F6372656174655F6D73673A20636865D4
:10A98000636B2074686174206669727374207062EE
:10A9900075662063616E20686F6C642073747275D5
:10A9A000637420646863705F6D736700E00000206B
:10A9B000638253632DE9F84305466C6A002600BFA5
:10A9C00000BF0C21204600F09BFF042221462846B0
:10A9D000FFF7C8FE06460EBB04223221204600F0D7
:10A9E000DDF9606A08F081FA80464146204600F0B1
:10A9F00023FA204600F086FA228BF03291B22069C9
:10AA00000CF09AFC009543230E4A2169606812F00D
:10AA1000BFFC204600F018F800BF01E000BF00BFF7
:10AA2000607B401C607342F2107707F2F3104FF422
:10AA3000FA7190FBF1F0608300BF00BF3046BDE8C3
:10AA4000F88300006086040810B5044600BF1CB9F6
:10AA50000EA0FDF76BFF10BD00BF00BF206910B94D
:10AA600012A0FDF763FF00BF00BF606910B919A015
:10AA7000FDF75CFF00BF206910B120690CF04CFBB2
:10AA800000202061606100BFE5E70000646863703A
:10AA90005F64656C6574655F6D73673A20646863B5
:10AAA0007020213D204E554C4C00000064686370BE
:10AAB0005F64656C6574655F6D73673A2064686395
:10AAC000702D3E705F6F757420213D204E554C4CAB
:10AAD00000000000646863705F64656C6574655FA6
:10AAE0006D73673A20646863702D3E6D73675F6FA6
:10AAF000757420213D204E554C4C0000F8B505469C
:10AB00006C6A002600BF00BF00206062062120465C
:10AB100000F0F6FE012221462846FFF723FE0646F6
:10AB2000002E3AD100BF00BF02223921204600F09A
:10AB300035F9298D204600F0C9F904223721204635
:10AB400000F02CF90121204600F046F903212046AF
:10AB500000F042F91C21204600F03EF90621204673
:10AB600000F03AF9204600F0CDF900BF00BF228B7B
:10AB7000F03291B220690CF0DFFB00BF00BF0095FE
:10AB80004323164A2169606812F002FC00BF00BF2F
:10AB90002046FFF759FF00BF01E000BF00BF607B08
:10ABA000401C6073607B062803DA617B01208840CB
:10ABB00000E03C2000EB4001C1EBC0104FF6FF71FC
:10ABC00001EAC00707F2F3104FF4FA7190FBF1F0BD
:10ABD000608300BF00BF3046F8BD000060860408F7
:10ABE00010B5104804681AE0606AB8B1606A408B1A
:10ABF000012805DD606A408B401E616A48830DE0D4
:10AC0000606A408B012809D1606A408B401E616AEE
:10AC1000488300BF00BF204600F088FF2468002C56
:10AC2000E2D110BD08010020F8B50646746A002084
:10AC3000A062E0622448C07810B12448C068206354
:10AC40002148007918B121480069606302E0206B57
:10AC5000400860631C48407918B11C484069A063F3
:10AC600001E0206BA063A0680069606216488079EB
:10AC700038B11649886908F011F9A0620120A07363
:10AC800001E00020A0731048C07920B10F49C869C5
:10AC900008F004F9E06200250EE005F108010B4A16
:10ACA00052F8210008F0FAF800906946284602F0B0
:10ACB0002BFB681CC5B200BF05F108000249085C07
:10ACC00008B1022DE9DBF8BDACFB002084FB0020BD
:10ACD00070B50446656A00BF00BF20460BF01CFA41
:10ACE000094920460BF036FA074920460BF029FAAD
:10ACF000054920460BF0B0FA0C21284600F000FE72
:10AD00002046FFF7FBFE70BD5C86040870B5054663
:10AD10006C6A00BF00BF0B48807878B10A49886828
:10AD200008F0BCF8206200BF00BFA0680069606244
:10AD300000BF00BF284600F061FD01E000BF00BF7A
:10AD400070BD0000ACFB002084FB002070B5054600
:10AD50006C6A04B970BD207B042809D003DC98B16B
:10AD6000032812D107E0052803D00A280DD101E0FD
:10AD700000BF00BF00BF28460BF0CEF90020607373
:10AD8000284600F093FB06E005E0002060732846AB
:10AD9000FFF7B4FE00BF00BF00BFDBE770B504469D
:10ADA0000E46154600BF208B801C2844442802D93B
:10ADB0000848FDF7BBFD00BF218B481C208360695C
:10ADC000F0304654218B481C20836069F030455494
:10ADD00070BD00009C8B040870B504460D4600BF92
:10ADE000208B442802D305A0FDF7A0FD00BF218BD6
:10ADF000481C20836069F030455470BD64686370FE
:10AE00005F6F7074696F6E5F627974653A20646811
:10AE100063702D3E6F7074696F6E735F6F75745FD2
:10AE20006C656E203C20444843505F4F5054494F5E
:10AE30004E535F4C454E000070B504460D4600BFB2
:10AE4000208B001D442802D910A0FDF76FFD00BF24
:10AE5000290E228B501C20836069F0308154C5F389
:10AE60000741228B501C20836069F0308154C5F368
:10AE70000721228B501C20836069F0308154228B83
:10AE8000501C20836069F030855470BD6468637025
:10AE90005F6F7074696F6E5F6C6F6E673A20646885
:10AEA00063702D3E6F7074696F6E735F6F75745F42
:10AEB0006C656E202B2034203C3D20444843505F7D
:10AEC0004F5054494F4E535F4C454E0070B50446A9
:10AED0000D4600BF208B801C442802D90848FDF78E
:10AEE00025FD00BF290A228B501C20836069F030A9
:10AEF0008154228B501C20836069F030855470BDD2
:10AF0000588B040810B5044600BF1CB917A0FDF704
:10AF10000DFD10BD00BF00BF606910B91CA0FDF79A
:10AF200005FD00BF00BF208B442802D323A0FDF7FE
:10AF3000FDFC00BFFF21228B501C20836069F03094
:10AF4000815406E00021228B501C20836069F03080
:10AF50008154208B442803D3207E00F0030010B1DD
:10AF6000208B4428EED300BFD3E7000064686370F1
:10AF70005F6F7074696F6E5F747261696C65723A4D
:10AF8000206468637020213D204E554C4C00000029
:10AF9000646863705F6F7074696F6E5F747261690B
:10AFA0006C65723A20646863702D3E6D73675F6FE5
:10AFB000757420213D204E554C4C0A006468637026
:10AFC0005F6F7074696F6E5F747261696C65723AFD
:10AFD00020646863702D3E6F7074696F6E735F6F6D
:10AFE00075745F6C656E203C20444843505F4F5041
:10AFF00054494F4E535F4C454E0A00002DE9F34F24
:10B0000089B089460020069005900A21DC48F5F7B2
:10B010007FF9B9F80A002C2804DA6FF001000BB0B0
:10B02000BDE8F08FD9F80410099881604FF0F00B5B
:10B03000B9F80800079000BF4C460AE06089ABEB06
:10B0400000001FFA80FB61890798401A80B20790C0
:10B05000246814B160895845F0DD14B96FF001001F
:10B06000DDE75F46DDF81CA0606808904CE10898B9
:10B07000C05D049000264FF0FF38B81C80B20390EA
:10B080006189781C814203DD791C0898455C07E0E2
:10B09000206818B120684068007800E0002005466C
:10B0A0002E460498342865D00BDC032825D003DC19
:10B0B00080B1012874D113E006282CD03328F9D1AF
:10B0C0004BE0352863D0362871D03A287CD03B2815
:10B0D000F0D186E0002005460646781E87B291E052
:10B0E00000BF042D05D0A7A0FDF720FC6FF00500E0
:10B0F00095E700BF4FF0060884E0042600BFB54284
:10B1000005DAA3A0FDF712FC6FF0050087E700BF8A
:10B110004FF0070876E000BFE91705EB9171891041
:10B12000A5EB810129B19FA0FDF700FC6FF00500A0
:10B1300075E700BF082D01DA284600E00820064622
:10B1400000BFB54205DA92A0FDF7F0FB6FF00500F5
:10B1500065E700BF4FF0080854E000BF042D05D09C
:10B1600088A0FDF7E3FB6FF0050058E700BF4FF044
:10B17000030847E000BF012D05D08EA0FDF7D6FBE8
:10B180006FF005004BE700BF4FF000083AE000BF4A
:10B19000012D08D087A0FDF7C9FB6FF005003EE741
:10B1A0002CE004E010E000BF4FF001082AE000BFEF
:10B1B000042D05D073A0FDF7B9FB6FF005002EE755
:10B1C00000BF4FF002081DE000BF042D05D06DA0A8
:10B1D000FDF7ACFB6FF0050021E700BF4FF004085E
:10B1E00010E000BF042D05D066A0FDF79FFB6FF0B7
:10B1F000050014E700BF4FF0050803E0002600BF7C
:10B2000000BF00BF00BFA81C384487B2002E5FDD1E
:10B210000020029000BF00BFB8F1000F02DBB8F1C0
:10B220000A0F02DB66A0FDF781FB00BF544810F84F
:10B23000080078BB042E01DA304600E004200190BB
:10B2400002A92046039B019A0BF0F4FE042E22DD96
:10B2500000BFF11706EB91718910A6EB810129B1AE
:10B260005CA0FDF763FB6FF00500D8E600BF01208E
:10B27000434901F80800029807F010FE5A4941F8C6
:10B280002800301FC6B20398001D80B2039008F159
:10B290000108C0E71BE0042E04D1029807F025FE48
:10B2A00002900CE000BF012E05D050A0FDF73EFB40
:10B2B0006FF00500B3E600BF9DF808000290012082
:10B2C0002F4901F808004849029841F8280000BFBA
:10B2D0006089B84217DC6089381A87B26089AAEBA6
:10B2E00000001FFA80FA57450CDABAF1000F09D0B6
:10B2F000246800BF14B942A0FDF718FB00BF6068C6
:10B30000089000E008E000BF34B10898C05DFF2855
:10B3100002D05745FFF6ABAE00BF19480078D0B158
:10B32000314908680021164A1170012803D1012112
:10B33000069100BF0EE0022803D10121059100BF54
:10B3400008E0032804D101210591069100BF01E026
:10B3500000BF00BF00BF069830B1002006904FF03C
:10B360006C0BEC20079067E6059830B10020059043
:10B370004FF02C0B6C2007905EE600204FE600009B
:10B38000ACFB00206C656E203D3D203400000000C9
:10B390006C656E203E3D206465636F64655F6C651F
:10B3A0006E0000006C656E20252034203D3D20306D
:10B3B000000000006C656E203D3D20310000000063
:10B3C000636865636B206465636F64655F69647857
:10B3D000000000006465636F64655F6C656E202526
:10B3E0002034203D3D20300084FB0020696E7661D2
:10B3F0006C6964206465636F64655F6C656E0000F2
:10B400006E657874207062756620776173206E7542
:10B410006C6C0000F8B505466C6A00BF00BF0421E3
:10B42000204600F06DFA032221462846FFF79AF9DC
:10B430000646EEB9022239212046FFF7AFFC298DDE
:10B440002046FFF743FD2046FFF75CFD228BF032DC
:10B4500091B220690BF070FF00954323124A2169D5
:10B46000606811F095FF2046FFF7EEFA00BF01E09B
:10B4700000BF00BF607B401C6073607B0A2804DA59
:10B48000607B4FF47A71484301E042F2107087B25A
:10B4900007F2F3104FF4FA7190FBF1F0608300BFF4
:10B4A00000BF3046F8BD0000608604082DE9F8436F
:10B4B00005466C6A00BF00BF0321204600F020FA59
:10B4C000032221462846FFF74DF906465EBB0222BD
:10B4D00039212046FFF762FC4FF410712046FFF738
:10B4E000F5FC042232212046FFF758FC606A07F081
:10B4F000FCFC804641462046FFF79EFC2046FFF7B5
:10B5000001FD228BF03291B220690BF015FF0095FE
:10B510004323134A2169606811F03AFF2046FFF780
:10B5200093FA00BF01E000BF00BF607B401C607366
:10B53000607B0A2804DA607B4FF47A71484301E0AB
:10B5400042F2107087B207F2F3104FF4FA7190FBD9
:10B55000F1F0608300BF00BF3046BDE8F883000013
:10B56000608604082DE9F05F81461546DDF828B0B5
:10B570004F467C6AD5F804A000BF00BF00BF00BFE3
:10B5800000BF00BF00BFA06810B143A0FDF7CEF917
:10B5900000BF68892C2802DA00BF00BF75E09AF866
:10B5A0000000022802D000BF00BF6EE000260CE0C1
:10B5B00007F12B00815D0AF11C00805D814202D001
:10B5C00000BF00BF61E0701CC6B297F82A00B0420D
:10B5D000EEDCDAF8040007F088FC2168884202D02B
:10B5E00000BF00BF51E029462046FFF707FD10B11C
:10B5F00000BF00BF49E000BF00BF2C48407810B931
:10B6000000BF00BF41E02A4890F80480B8F1050F60
:10B6100018D100BF00BF207B012806D13846FFF7B4
:10B6200003FB3846FFF752F82EE0207B032805D0B5
:10B63000207B042802D0207B052825D13846FEF740
:10B64000A3FF21E0B8F1060F11D1207B032808D019
:10B65000207B012805D0207B042802D0207B0528F0
:10B6600005D100BF00BF3846FFF732FB0CE0B8F150
:10B67000020F09D1207B062806D100BF00BF0020A1
:10B6800060833846FFF742FB00BF0020A0602846D9
:10B690000BF042FDBDE8F09F7265706C7920776118
:10B6A000736E27742066726565640000ACFB002031
:10B6B00084FB0020F8B505466C6A00BF00BF00217E
:10B6C000204600F01DF9002020626062A062E06266
:10B6D000A06360632063072221462846FFF742F8F3
:10B6E0000646AEB92046FFF70DFC228BF03291B230
:10B6F00020690BF021FE0095432304F1200221690B
:10B70000606811F045FE2046FFF79EF900BF01E09A
:10B7100000BF00BF607B401C6073607B0A2804DAB6
:10B72000607B4FF47A71484301E042F2107087B2B7
:10B7300007F2F3104FF4FA7190FBF1F0608300BF51
:10B7400000BF28460AF0E8FC064928460AF002FD38
:10B75000044928460AF0F5FC024928460AF07CFD17
:10B760003046F8BD5C860408F8B505466C6A00BF33
:10B7700000BF0521204600F0C3F8032221462846D9
:10B78000FEF7F0FF0646F6B9022239212046FFF700
:10B7900005FB298D2046FFF799FB2046FFF7B2FBFA
:10B7A000228BF03291B220690BF0C6FD0095432345
:10B7B00004F120022169606811F0EAFD2046FFF7DC
:10B7C00043F900BF01E000BF00BF607B401C607315
:10B7D000607B0A2804DA607B4FF4FA61484301E099
:10B7E00044F6206087B207F2F3104FF4FA7190FB31
:10B7F000F1F0608300BF00BF3046F8BD2DE9F8438B
:10B8000005466C6A00BF00BF0121204600F078F8B1
:10B81000032221462846FEF7A5FF0646002E4CD1FE
:10B82000022239212046FFF7B9FA298D2046FFF779
:10B830004DFB042232212046FFF7B0FA606A07F080
:10B8400054FB804641462046FFF7F6FA0422362193
:10B850002046FFF7A3FA206A07F047FB80464146DF
:10B860002046FFF7E9FA042237212046FFF796FA2F
:10B8700001212046FFF7B0FA03212046FFF7ACFA7A
:10B880001C212046FFF7A8FA06212046FFF7A4FA5C
:10B890002046FFF737FB228BF03291B220690BF084
:10B8A0004BFD00954323154A2169606811F070FD36
:10B8B0002046FFF7C9F800BF01E000BF00BF607B72
:10B8C000401C6073607B062803DA617B012088409E
:10B8D00000E03C2000EB4001C1EBC0104FF6FF71CF
:10B8E00001EAC00707F2F3104FF4FA7190FBF1F090
:10B8F000608300BF00BF3046BDE8F883608604085F
:10B90000027B8A4203D00173002242734283704754
:10B9100070B50546002600BF2DB93FA0FDF706F81B
:10B920006FF00D0070BD00BF6C6A00BF00BF15F85E
:10B93000310F20F00800287015F8310900F02000C0
:10B9400020B900BF00BF6FF00D00EBE7288DB0F508
:10B95000107F04DA00BF00BF4FF0FF30E2E774B998
:10B9600000BF00BF3C2008F0DDF8044624B900BF4A
:10B9700000BF4FF0FF30D5E76C6200BF14E000BF9E
:10B9800000BF606810B1606811F0BCFC00BF2069A6
:10B9900010B125A0FCF7CAFF00BF00BFA06810B11E
:10B9A00027A0FCF7C3FF00BF3C212046F4F7B0FC02
:10B9B00011F06AFC6060606820B900BF00BF4FF002
:10B9C000FF30AFE76068007A40F0200061680872DD
:10B9D00044222049606811F0B3FA43221D4960688F
:10B9E00011F006FB2A461C49606811F087FC00BF75
:10B9F00000BF2846FFF782F806462EB1284600F021
:10BA00002DF84FF0FF308DE795F8310040F0080039
:10BA100085F83100304685E76E6574696620213D02
:10BA2000204E554C4C0000007062756620705F6FB0
:10BA30007574207761736E27742066726565640083
:10BA40007265706C79207761736E277420667265F9
:10BA5000656400005C86040865B5000870B505469D
:10BA600000BF1DB911A0FCF761FF70BD00BF6C6A7B
:10BA700095F8310020F0080085F8310000BF00BFC4
:10BA80008CB1606820B1606811F03CFC00206060FF
:10BA900000BFA06810B10CA0FCF748FF00BF002158
:10BAA0002046FFF72DFF00BFDFE7000064686370EA
:10BAB0005F73746F703A206E6574696620213D2053
:10BAC0004E554C4C000000007265706C7920776117
:10BAD000736E2774206672656564000070B5054654
:10BAE0006C6A00BF00BF207B012805D0207B0A289C
:10BAF00002D0207B052804D100BF00BF2846FFF7F5
:10BB000033FE70BD70B505466C6A00BF00BF207B78
:10BB1000012805D0207B0A2802D0207B052804D1EB
:10BB200000BF00BF2846FFF775FC70BD70B5054625
:10BB30006C6A00BF00BF207B0C2802D0207B062847
:10BB400005D100BF00BF2846FEF7D8FF4FE0207B9D
:10BB5000012811D100BF00BF607B052803DC284607
:10BB6000FFF74CFE43E000BF00BF2846FFF7A2FDF1
:10BB70002846FEF7C3FF3AE0207B08280CD100BF1F
:10BB800000BF607B012803DC2846FEF79FFD2EE006
:10BB90002846FEF7F9FC2AE0207B052805D100BFE6
:10BBA00000BF2846FFF7E0FD21E0207B042811D1EB
:10BBB00000BF00BF607B082803DC2846FFF72AFC93
:10BBC00015E000BF00BF2846FFF774FD2846FEF7CA
:10BBD00095FF0CE0207B032809D1607B022803DA63
:10BBE0002846FFF763FC02E02846FEF787FF70BD9A
:10BBF00010B5044600BF00BFFEF78CFD00220349CC
:10BC00004EF660200DF03CF910BD0000F1BB0008BD
:10BC100010B5044600BF00BFFEF7E2FF0022034953
:10BC20004FF4FA700DF02CF910BD000011BC0008A3
:10BC30002DE9F04104460E460021204600F04FFA5F
:10BC40000546EDB9002700BF2169206808F0EAFB2E
:10BC5000054605B113E060690078E52802D0606907
:10BC6000007820B9781C0746B04201D107E00027D0
:10BC70000121204600F07FF80546002DE4D000BFEA
:10BC8000042D00D107252846BDE8F0812DE9F047B5
:10BC900004460021204600F022FA074617B1384634
:10BCA000BDE8F0874FF0FF09CA464FF6FF70A08449
:10BCB00000BF2169206808F0B5FB074607B157E0CF
:10BCC00065692E780EB9042752E0E87A00F03F0843
:10BCD000E52E05D008F0080040B1B8F10F0F05D0EF
:10BCE0004FF0FF094FF6FF70A0843AE0B8F10F0F54
:10BCF0001CD1206A78B306F0400030B195F80DA051
:10BD000026F04006B146E088A0844E450AD1687B03
:10BD1000504507D12946206AFEF786F810B1A9F1EF
:10BD2000010000E0FF2000F0FF091AE0B9F1000F68
:10BD300005D128460CF008FF504500D118E0A06955
:10BD4000C07A00F0010038B90B222846A16907F03B
:10BD500007FE08B90CE004E04FF0FF094FF6FF7052
:10BD6000A0840021204600F006F80746002FA0D04E
:10BD700000BF384694E72DE9F04104468846E08844
:10BD8000461CB0B208B1206910B90420BDE8F081AA
:10BD900006F00F0000286CD12069401C2061E0688B
:10BDA00028B920680089B04263D80420EEE72068F3
:10BDB0008078401E00EA161000285AD1E1682068F9
:10BDC00004F0C8FB0546012D01D80220DEE7681CFF
:10BDD00008B90120DAE720684069A84243D8B8F1E1
:10BDE000000F01D10420D1E7E1682068FEF764F874
:10BDF00005460DB90720C9E7012D01D10220C5E78D
:10BE0000681C08B90120C1E720680CF011FF08B1D7
:10BE10000120BBE7216801F130004FF400720021DE
:10BE200007F084FF29462068FDF7F0FF2168C8620B
:10BE300000270EE001202168087120680CF0F8FE50
:10BE400008B10120A2E72068C06A401C2168C862CE
:10BE50007F1C20688078B842ECD82068C06AC01B7C
:10BE60002168C86200BFE56029462068FDF7CEFF63
:10BE70002061E6802068303006F00F0100EB4110B1
:10BE80006061002082E72DE9F05F04468A464FF0AA
:10BE9000FF09CB4604274EE02169206808F0C2FA6A
:10BEA000074607B14AE0666935780DB9042745E0D1
:10BEB000F07A00F03F08E52D09D02E2D07D0B8F11B
:10BEC000080F01D1012000E00020504502D04FF0C2
:10BED000FF0929E0B8F10F0F1AD105F0400030B189
:10BEE00096F80DB025F04005A946E088A0844D45A0
:10BEF0000AD1707B584507D13146206A0BF038FBD8
:10BF000010B1A9F1010000E0FF2000F0FF090BE0F3
:10BF1000B9F1000F04D130460CF016FE584502D09E
:10BF20004FF6FF70A08409E000212046FFF723FFB1
:10BF3000074607B102E020690028ADD100BF0FB16C
:10BF4000002020613846BDE8F09F2DE9FE4F0446F1
:10BF5000D4F81880D4F820900C224146684607F0A7
:10BF600012FD00BF9DF80B0000F0010020B300207F
:10BF700088F80B00206201260CE033464A466946E9
:10BF8000404604F081FA2046FFF780FE054605B1E1
:10BF900002E0761C642EF0D300BF642E02D107208D
:10BFA000BDE8FE8F042D01D02846F9E79DF80B006F
:10BFB00088F80B00C4F820909DF80B0000F00200F8
:10BFC00060B1002600E0761C39F816000028FAD18E
:10BFD00006F119000D21B0FBF1F700E00127394609
:10BFE0002046FFF725FE054645BB781E071E25D0D7
:10BFF000E088C11B204600F072F80546F5B9A0693B
:10C000000CF0A2FD824600BF2169206808F00AFA00
:10C01000054605B111E0FAB253466169206A04F0A1
:10C020007DF901202168087100212046FFF7A3FE59
:10C03000054615B9781E071EE6D100BFC5B92169AE
:10C04000206808F0EFF9054695B9202200216069C3
:10C0500007F06CFE0B22D4E9050107F094FCA069FF
:10C06000C07A00F018006169087301202168087126
:10C07000284695E770B50446E688A08C4FF6FF7217
:10C08000904201D1304600E0A08C0146204600F0ED
:10C0900026F805460DBB00BF2169206808F0C2F9EB
:10C0A000054605B115E020220021606907F03EFE3B
:10C0B000E52061690870012021680871E088B042BC
:10C0C00000D306E000212046FFF755FE0546002D6F
:10C0D000E2D000BF042D00D10225284670BD2DE915
:10C0E000F04104460E46E680A568012D03D0206885
:10C0F0004069A84202D80220BDE8F0812DB920682D
:10C100000078032801D12068456A45B92068008974
:10C11000B04201D80220EFE72068476A1EE020689D
:10C1200080784FEA001812E02946206804F012FADD
:10C130000546681C08B90120DEE7022D03D32068FC
:10C140004069A84201D80220D6E7A6EB080646457A
:10C15000EAD229462068FDF759FE0746E5600FB987
:10C160000220C9E707EB161020612068303006F086
:10C170000F0100EB411060610020BDE70146012086
:10C1800009B9002000E000BF00BF70472DE9F04171
:10C1900005460E4614460427F5B9012736B1012E8F
:10C1A00006D0022E0AD0032E12D10CE0002711E097
:10C1B000F9F724F8400A206000270BE04FF40070E4
:10C1C0002080002706E04FF400702060002701E087
:10C1D000042700BF00BF01E0042700BF00BF3846AE
:10C1E000BDE8F0812DE9F04104460D4616461F4694
:10C1F0004FF000085CB93B464FF4007231462846C8
:10C20000F9F78CF800B901E04FF0010802E04FF0B7
:10C21000040800BF00BF4046BDE8F0810146012090
:10C2200009B9002000E000BF00BF70472DE9F041D0
:10C2300004460D4616461F464FF0000884B93B469B
:10C240004FF4007231462846F9F7D0F800B906E0FD
:10C250003A46314606A0FCF769FB4FF0010802E0C0
:10C260004FF0040800BF00BF4046BDE8F081000069
:10C270004E414E445F57726974654D756C746953D5
:10C280006563746F72732829204572726F72212062
:10C29000736563746F72203D2025642C20636F7575
:10C2A0006E74203D202564200D0A00002DE9F04128
:10C2B00006460C4615461F464BF23061701A8E42F8
:10C2C0003AD015DC4BF22161A6EB01008E422AD058
:10C2D00009DCA6F53640A0F11100C0B1012817D045
:10C2E000022833D115E001281ED002282ED11CE0EF
:10C2F00061280FD006DC01281FD002281ED0032899
:10C3000024D11CE0622806D063281FD104E000BFBE
:10C3100000BF00BF00BF00BF3B4618A2022120465D
:10C3200000F05CFB25E000BF00BF3B4614A20221E9
:10C33000204600F053FB1CE000BF00BF00BF3B469F
:10C3400011A20321204600F049FB12E000200DE07D
:10C35000215CC91E01F00F02215C3339091101EB88
:10C36000810102EB41013954411C88B2A842EFDB44
:10C3700000BF00BF2846BDE8F081000058585800B3
:10C3800058582E585800000058582E5858585800E1
:10C3900070B596B005460C4616463C2103A8F3F747
:10C3A000B7FF002012901390149015902868CDF8D4
:10C3B0004900A888ADF84D0001208DF850000220FA
:10C3C0008DF851000020029004F13300C0B28DF8C6
:10C3D0000800200A3330C0B28DF80900BDF808000B
:10C3E000ADF852000E2212A9284600F0E7FB002803
:10C3F00003DA4FF0FF3016B070BD022023463C2216
:10C4000003A90090284600F0B6FB002802DA4FF09E
:10C41000FF30F0E79DF81500801E82B2334606A972
:10C420002046FFF743FFE6E72DE9FF4104460E46AD
:10C4300017463A463146204600F091FA002804DAC1
:10C440004FF0FF3004B0BDE8F081207A842801D19C
:10C450000020F7E703AD002004E0295C33312954C4
:10C46000411CC8B20228F8DB60890399884202D0D7
:10C470004FF0FF30E6E70020E4E700002DE9F0414F
:10C4800007460C4615461E46DA49781A8F4271D087
:10C4900074DCD949A7EB01008F426DD033DCD7495A
:10C4A000A7EB01008F4268D016DCB7F5407F7CD047
:10C4B00008DC002F7AD0B7F5807F78D0B7F5007F01
:10C4C00076D1E6E0B7F5806F73D0B7F5803F71D0D5
:10C4D000B7F1011FF4D1E1E040F2FE32811A90423F
:10C4E00069D009DCFE2867D0B0F5FF7F70D0A0F2DC
:10C4F000FE200028E4D1D4E0B1F57C4F69D0B1F53D
:10C500007D4FDDD1D0E0BE4A811A904271D018DC57
:10C51000B0F5FF3F6ED009DCB0F5807F6BD0B0F591
:10C52000007F69D0B0F57E4FCAD1C1E0B54908445B
:10C5300000287DD0B0F5803F7BD0B0F5003FBFD163
:10C54000BAE0B1F57A0F75D00BDCB1F5803F72D04F
:10C55000B1F5790F70D06FF4790008440028AFD19D
:10C56000BBE06FF47A000844002872D0B0F1FF1FDE
:10C57000A6D1CBE0CBE001E097E090E0A24A811A9F
:10C58000904267D041DCB0F5003F75D022DCB0F5B9
:10C59000803F72D011DCB0F5807F6FD0B0F57D4F59
:10C5A0006DD0B0F57F4F8BD1BEE073E06FE06FE0F0
:10C5B00009E170E070E075E06FE0944908440028FC
:10C5C0007ED0B0F57D4F7CD0B0F57E4F92D1B5E0F6
:10C5D00066E068E0B0F5403F74D00EDC8C4908445A
:10C5E000002870D0B0F57D4F6ED0B0F57E4F88D169
:10C5F000A8E062E05DE059E059E08649084400287F
:10C6000074D0B0F57D4F8FD19FE0834A881A914254
:10C610006DD020DCB1F5803F6AD00EDCB1F5807FB3
:10C6200067D0B1F5007F6FD0B1F57F4F87D19AE029
:10C6300040E040E050E041E04DE07448084400280C
:10C6400070D0B0F5807F6ED074490844002886D140
:10C650005FE043E07AE0724A811A90427DD00FDCBD
:10C66000B0F5807F57D06F490844002876D06E49D6
:10C670000844002897D19AE061E056E048E044E0A1
:10C680006A48084400286AD001288CD191E000BF94
:10C6900000BF00BF00BF00BF00BF00BF00BF00BFA2
:10C6A00000BF00BF00BF00BF00BF00BF00BF00BF92
:10C6B00000BF00BF00BF00BF00BF00BF334604E0A3
:10C6C00034E03AE03FE03BE03BE059A20421204661
:10C6D00000F084F98AE000BF00BF00BF334657A2D4
:10C6E0000321204600F07AF900200AE02CE011E056
:10C6F0003AE02CE0C11C615C3339CAB2011D7254AE
:10C70000401C0528F6DB71E022E000BF00BF00BF3F
:10C7100000BF00BF00BF33464AA20221204600F0FE
:10C720005DF963E021E021E000BF00BF334647A28E
:10C730000321204600F052F958E000BF00BF00BFBF
:10C7400000BF00BF00BF00BF00BF00BF00BF00BFF1
:10C7500033463AA20321204602E015E00DE027E02F
:10C7600000F03CF942E000BF00BF00BF334639A2F1
:10C770000221204600F032F938E033462DA2022192
:10C78000204600F02BF931E000200DE0215CC91EAD
:10C7900001F00F02215C3339091101EB810102EB39
:10C7A00041013154411C88B2A842EFDB1EE000BFBA
:10C7B00000BF002004E0215C33393154411C88B2B1
:10C7C000A842F8DB12E000200DE0215CC91E01F058
:10C7D0000F02215C3339091101EB810102EB4101A8
:10C7E0003154411C88B2A842EFDB00BF00BF28468D
:10C7F000BDE8F08100020102000202000200010017
:10C8000000FE05000002FDFF00FF030000FFFEFF29
:10C8100000FFFDFF00FFFCFF000107000001FAFF21
:10C8200001FFF902FE018CFFFFFB7FFE000106FE07
:10C830005858585858582E585800000058582E58D4
:10C84000585858005858582E580000005858582E1C
:10C8500058585800582E58585800000070B596B0D7
:10C8600005460C4616463C2103A8F3F751FD00206F
:10C8700012901390149015902868CDF84900A8885C
:10C88000ADF84D0011208DF8500004208DF85100B6
:10C890000020029004F13300C0B28DF80800200A95
:10C8A0003330C0B28DF80900200C3330C0B28DF89F
:10C8B0000A00332000EB1460C0B28DF80B00029820
:10C8C000CDF85200102212A9284600F077F900286E
:10C8D00003DA4FF0FF3016B070BD012023463C2232
:10C8E00003A90090284600F046F9002802DA4FF02C
:10C8F000FF30F0E79DF81500001F82B233460DF1BE
:10C900001A012046FFF7BAFDE5E72DE9FF4104468D
:10C910000E4617463A463146204600F020F80028D9
:10C9200004DA4FF0FF3004B0BDE8F081207A94289B
:10C9300001D10020F7E703AD002004E0295C33318A
:10C940002954411CC8B20428F8DBD4F80A00039922
:10C95000884202D04FF0FF30E5E70020E3E72DE901
:10C96000F04104460D461646072D03DA4FF0FF301E
:10C97000BDE8F0812078682806D1E079682803D1E5
:10C98000681E205C162802D04FF0FF30F0E7A91E89
:10C990002046FCF7E9F8C7B2A81E205CB84202D0D6
:10C9A0004FF0FF30E4E7207A00F0800010B94FF03C
:10C9B000FF30DDE7207A00F04000402802D1E81E79
:10C9C000205CD5E706223146601CF3F7DFFC10B18E
:10C9D0004FF0FF30CCE70020CAE700002DE9FF4F01
:10C9E00085B0144699464FF0000ADDE90501FDF7D0
:10C9F00007FC0490002512E0605D2E280ED1204631
:10CA0000F3F7AFFC401BA0F1010ABAF1000F04DA02
:10CA10004FF0FF3009B0BDE8F08F05E06D1C2046F7
:10CA2000F3F79FFCA842E7D800BF5046F4F77BF924
:10CA300002460B46CDE9000100200A490AF0B4FE87
:10CA4000CDE902010498F4F76EF90746DDE9022307
:10CA5000F4F7F5F80546F4F7E7F98346C9F800B0AE
:10CA60000020D7E7000024402DE9F04180460C4625
:10CA700015460026F9F7C2FE07461DE0F9F7BEFE8F
:10CA8000C01B0E494968884202D90020BDE8F081E8
:10CA90000A4890F8D00001280ED1084890F8D160DB
:10CAA0002A1F00F10C012046F3F719FC034890F807
:10CAB000D100061F3046E9E7E0E70000C485012009
:10CAC0002DE9F04107460E461446C8211748F3F7F2
:10CAD0001FFC0A20FDF7CCFCF8F74CFF01221103E4
:10CAE0001348F7F74DFE00250CE0715D1148FBF788
:10CAF0001FFE00BF80210F48FBF71CFB0028F9D068
:10CB0000681C85B2A542F0DDF8F746FF00224FF41D
:10CB100080510748F7F734FE00200449083981F8AE
:10CB2000D10081F8D0002046BDE8F081CC850120FD
:10CB300000080240004800402DE9F04105460E463D
:10CB400017461C464FF0FF38012C08D0022C0DD19F
:10CB50003A4631462846FFF71BFC804607E03A4636
:10CB600031462846FFF77AFE804600E000BF00BF4E
:10CB70004046BDE8F0812DE9F04704460D461746D2
:10CB80009846089E3A4629462046E36898478146DB
:10CB9000022E07D14346224649462846FFF744FC69
:10CBA000BDE8F087012E06D1434622464946284675
:10CBB000FFF7ABFEF4E74FF0FF30F1E770B5064644
:10CBC0000C46154668202070E0711621681E21541D
:10CBD000A91E2046FBF7C8FFC1B2A81E2154AAB265
:10CBE00021463046B368984770BD3CB502460020E8
:10CBF0000090019000BF05E00B5CC0F105040DF84A
:10CC00000430401C0628F7DB00981060BDF80400D3
:10CC100090803CBD10B5002404E0204600F006F8EA
:10CC2000601CC4B2042CF8DB10BD000070B50646D1
:10CC3000C6EBC60000EB80003E4901EBC00400BF1C
:10CC4000042E02DB3CA0FBF771FE00BF2078002819
:10CC500066D0012804D0022815D0032861D154E001
:10CC600002202070002060700120A0700020E07081
:10CC70006078324604F10C0100F08AFA05460DB1E5
:10CC800000BF00BF53E0A078401EC0B2A0700028D3
:10CC90003AD1E078401CC0B2E070042828D1607816
:10CCA000401C022812DA6078401C2A4901EB8000FF
:10CCB00060B16078401C51F8200038B16078401CA9
:10CCC00060700120A0700020E07030E000BF00BF65
:10CCD000D4F8100138B1002104F10C00D4F810315F
:10CCE000D4F81421984700202070C4F810011EE0E9
:10CCF000E078A0706078324604F10C0100F048FA48
:10CD000005460DB100BF00BF11E0A068401EA06045
:10CD100028B900BF00BF00202070C4F8100106E051
:10CD200005E000BF0CA0FBF701FE00BF00BF00BF85
:10CD300070BD0000B8FB0020617272617920696EDD
:10CD4000646578206F7574206F6620626F756E64FD
:10CD500073000000EC000020756E6B6E6F776E2024
:10CD6000646E735F7461626C6520656E74727920A5
:10CD700073746174653A000010B5024600BF11F883
:10CD8000013B03F0C000C02800D110E009E010789A
:10CD90000C78A04201D0012010BD491C521C581E25
:10CDA000C3B2002BF3DC521C08780028E7D100BF87
:10CDB0000020F1E72DE9F05F074688469146002400
:10CDC00000200646834600251BE0C5EBC50000EBAE
:10CDD0008000314901EBC004207800B913E02078CD
:10CDE00003280CD120792D490978081A584506DD09
:10CDF00020792A490978081A00F0FF0B2E46681C92
:10CE0000C5B2042DE1DB00BF042D18D1042E08DAD1
:10CE1000C6EBC60000EB80001F4911F83000032864
:10CE200005D000BF00BF4FF0FF30BDE8F09F354692
:10CE3000C5EBC50000EB8000174901EBC00400BF43
:10CE400000BF012020701548007820711348007839
:10CE5000401C12490870C4F81081C4F81491384677
:10CE6000F3F77FFAFF2803D23846F3F77AFA00E0A7
:10CE7000FF2082465246394604F10C00F3F72FFAA0
:10CE8000002104F10C0000F80A102846FFF7CEFE3E
:10CE90006FF00400C9E70000B8FB0020E8000020A4
:10CEA0002DE9F04105460E4617469846124800689F
:10CEB00040B13EB135B1287820B12846F3F751FA98
:10CEC000FF2803D96FF00D00BDE8F081284605F07A
:10CED000BBF90446601C18B9284600F04BF804461C
:10CEE000601C10B134600020EEE742463946284607
:10CEF000FFF760FFE8E70000E400002008B51448F1
:10CF000020F003001349086013A005F09DF900907C
:10CF100000BF00BF14480068C0B910F0B5F912494D
:10CF200008600846006888B100BF00BF00220F49B2
:10CF30000D48006810F004F800220D490A48006806
:10CF400010F0DCF96946002000F0DEF908BD0000B1
:10CF50001B000120F40000203230382E36372E32EC
:10CF600032322E3232320000E40000205C860408A7
:10CF700009D0000870B50546002427E0C4EBC400C2
:10CF800000EB8000144911F8300003281CD1C4EBD9
:10CF9000C40000EB80000A4602EBC00000F10C0167
:10CFA0002846F3F7E5F978B900BF00BF00BF00BF1E
:10CFB00000BF00BFC4EBC40000EB8000064901EBDA
:10CFC000C000D0F80C0170BD601CC4B2042CD5DBCD
:10CFD0004FF0FF30F7E70000B8FB0020014600BF2C
:10CFE00011F8012B02F0C000C02800D108E002E0D7
:10CFF000491C501EC2B2002AFADC08780028EFD182
:10D0000000BF481C704700002DE9FE4F1546DDF8B3
:10D0100030B02889B0F5007F02DD00BF00BFACE072
:10D0200028891A2802DA00BF00BFA6E02A89002357
:10D0300054480168284609F0FDFF2989884279D1C2
:10D0400050480668308805F036FF8046B8F1040F76
:10D0500070DAC8EBC80000EB80004B4901EBC0045C
:10D060002078022878D103202070F07800F00F009B
:10D070006071B08805F01FFF8246F08805F01BFF45
:10D080008146B07800F0800020B1607910B9BAF123
:10D09000010F02D000BF00BF5FE03A4801680C31C9
:10D0A00004F10C00FFF768FE10B100BF00BF54E0B0
:10D0B000344800680C30FFF791FF071D46E0384602
:10D0C000FFF78CFF07463868009078680190388930
:10D0D000ADF80800BDF80000B0F5807F2BD1BDF899
:10D0E0000200B0F5807F26D1BDF80800B0F5806F52
:10D0F00021D1019805F0F9FEA0602449A06888427A
:10D1000001D90846A060D7F80A10C4F80C1100BF76
:10D1100000BF00BF00BF00BF00BFD4F8100140B186
:10D1200004F5867104F10C00D4F81031D4F8142100
:10D13000984722E010E0BDF8080005F0BCFE07F1BA
:10D140000A014718A9F101001FFA80F9B9F1000F8F
:10D15000B5DC00BF00BF00E00FE0D4F8100138B12B
:10D16000002104F10C00D4F81031D4F814219847B0
:10D1700000202070C4F8100100BF284609F0CCFF41
:10D18000BDE8FE8FF4000020B8FB0020803A0900C3
:10D190002DE9F74F82B00746894600BF00BF00BFA8
:10D1A000022F02DB40A0FBF7C1FB00BF00BF4448D9
:10D1B00000EB870018B1424850F8270010B941A091
:10D1C000FBF7B4FB00BF00224FF48871104609F052
:10D1D000DFFB0546002D60D000BF286810B142A0DB
:10D1E000FBF7A4FB00BFD5F804800020C8F80000BE
:10D1F000C8F80400C8F80800049805F05CFEA8F818
:10D200000000012088F802000002A8F8040008F1DC
:10D210000C044E46761E00BF761CA346641C0020FC
:10D22000009007E030782070641C0098401CC0B269
:10D230000090761C30782E2802D030780028F1D16A
:10D2400000988BF8000030780028E5D104F8010B35
:10D250004FF48070ADF80400ADF80600019820602E
:10D26000AA88201D801A81B228460AF065F8144861
:10D2700000EB87013522234800680FF0B9FE104803
:10D2800000EB8702352329461E48006810F064F839
:10D290008246284609F040FF01E04FF0FF3A504631
:10D2A00005B0BDE8F08F0000646E73207365727680
:10D2B0006572206F7574206F6620617272617900EB
:10D2C000EC000020646E73207365727665722068CE
:10D2D0006173206E6F2049502061646472657373BE
:10D2E000207365740000000070627566206D7573B0
:10D2F0007420626520696E206F6E652070696563B9
:10D3000065000000E400002002280ADA054A1268DD
:10D310003AB131B129B10A681AB1034A0B6842F82F
:10D3200020307047E4000020EC00002010B50446D7
:10D3300000BF00BF00F00AF8002203494FF47A70E2
:10D340000BF09EFD10BD00002DD3000810B5044861
:10D35000006818B100BF00BFFFF75CFC10BD000003
:10D36000E400002010B504462068407878B12068B9
:10D37000407802280BD000BF20680078102802D027
:10D380001FA0FBF7D3FA00BFFB20207130E020681C
:10D39000406858B320680078102827D1207A0328E5
:10D3A00006D020684078022802D1F32020711FE0C7
:10D3B000207A00F0010010B1206808F0C9F900BF20
:10D3C0002068D0F82C0118B92068D0F8280110B1D5
:10D3D00013A0FBF7ABFA00BF042021684870206857
:10D3E000C0F82C41206800F029F810BDFA20207107
:10D3F000216801F10C000BF01AFD00BFF5E70000F9
:10D400006D73672D3E636F6E6E2D3E74797065206F
:10D410003D3D204E4554434F4E4E5F544350000017
:10D42000616C72656164792077726974696E6720D6
:10D430006F7220636C6F73696E6700002DE9F047AF
:10D44000044600BF14B95BA0FBF770FA00BF00BF31
:10D450002078102802D05BA0FBF768FA00BF00BF5D
:10D460006078042802D05FA0FBF760FA00BF00BF1D
:10D47000606810B964A0FBF759FA00BF00BFD4F888
:10D480002C0110B965A0FBF751FA00BFD4F82C01AC
:10D49000067A06F0010706F00208032E01D10120EA
:10D4A00000E000208146B9F1000F03D00021606840
:10D4B0000BF0E6FE6068007E012804D10021606860
:10D4C0000BF075FE1BE03FB1002160680EF0A2F981
:10D4D000002160680BF06BFEB8F1000F03D0002153
:10D4E00060680EF079FBB9F1000F08D0042200212A
:10D4F00060680DF001FA002160680CF011FAB9F1D2
:10D50000000F04D060680BF0BDFE054605E0424602
:10D51000394660680EF082FB054675BB0020D4F8E2
:10D520002C110871C4F82C016070B9F1000F09D0FA
:10D530006060D4F8300128B1002204212046D4F8DC
:10D540003031984747B1D4F8300128B10022114654
:10D550002046D4F830319847B8F1000F08D0D4F8FD
:10D56000300128B1002202212046D4F830319847FA
:10D5700004F10C000BF05BFC1AE0FFE700BF6068F1
:10D58000007E012802D12CA0FBF7D0F900BF33495F
:10D5900060680EF021FB0422314960680DF0ACF99F
:10D5A000304960680CF0BCF9214660680BF068FEF9
:10D5B000BDE8F087696E76616C696420636F6E6E9A
:10D5C000000000007468697320697320666F722020
:10D5D000746370206E6574636F6E6E73206F6E6C13
:10D5E00079000000636F6E6E206D75737420626544
:10D5F00020696E207374617465204E4554434F4E0C
:10D600004E5F434C4F53450070636220616C7265FE
:10D6100061647920636C6F7365640000636F6E6E84
:10D620002D3E63757272656E745F6D736720213D68
:10D63000204E554C4C000000436C6F73696E6720A0
:10D6400061206C697374656E20706362206D61790E
:10D65000206E6F74206661696C210000CD8901081D
:10D660002177010895DF000810B50446206840685E
:10D6700010B9F42020715CE02068007800F0F00020
:10D68000102812D0202808D0402847D12268A1684D
:10D6900050680AF010FE20714AE0A2892368A16850
:10D6A00058680FF0A5FC207142E02068407810B166
:10D6B000F720207131E020680BF0CAF9A2892368B5
:10D6C000A16858681E4B0BF0E5FE2071207920BB45
:10D6D000216891F82411C1F34000032122685170A0
:10D6E00000BF40B1216891F8241141F00401226883
:10D6F00082F8241107E0216891F8241121F0040137
:10D70000226882F8241100BF10B1FB21217103E0CF
:10D710002168C1F82C4110BD00BF09E000BF09A07D
:10D72000FBF704F900BFFA20207100BF00BF00BF63
:10D7300000BF216801F10C000BF079FB00BFEAE7A4
:10D740005DD70008496E76616C6964206E6574630C
:10D750006F6E6E2074797065000000002DE9F0474F
:10D760000546894616462C461CB96FF00500BDE8F3
:10D77000F08700BF6078032802D027A0FBF7D6F817
:10D7800000BF00BFD4F82C0138B994F8240100F090
:10D79000040010B928A0FBF7C9F800BFD4F82C0189
:10D7A00010B1D4F82C0106712078102803D116B9D5
:10D7B00020460BF04DF994F82401012121EA90074D
:10D7C00000BF94F8240120F0040084F8240100BF75
:10D7D0000020C4F82C01607077B900BFF2F7F0FCAC
:10D7E000804694F9080010F1090F01DB0020207237
:10D7F0004046F2F7E9FC00BFD4F8300128B100221E
:10D8000002212046D4F8303198471FB104F10C00B2
:10D810000BF00DFB0020AAE7636F6E6E2D3E737454
:10D82000617465203D3D204E4554434F4E4E5F434D
:10D830004F4E4E454354000028636F6E6E2D3E637D
:10D84000757272656E745F6D736720213D204E5551
:10D850004C4C29207C7C20636F6E6E2D3E696E5F80
:10D860006E6F6E5F626C6F636B696E675F636F6E26
:10D870006E6563740000000010B5044620684078AF
:10D8800098B12068407802280FD02068407803289B
:10D890000BD000BF20680078102802D039A0FBF719
:10D8A00045F800BFFB2020715FE000BF2068407892
:10D8B000032808D1206890F8240100F0040010B972
:10D8C00038A0FBF733F800BF206807F041FF20685D
:10D8D0004068002835D02068007800F0F00010285B
:10D8E00011D0202806D0402826D1216848680AF0A7
:10D8F00043FD22E0002021684968C861216848682A
:10D900000FF000FD19E000BF2068D0F82C0118B915
:10D910002068D0F8280110B12AA0FBF707F800BF53
:10D92000042021684870032020722068C0F82C4130
:10D930002068FFF783FD10BD00BF00BF00202168F5
:10D9400048602068D0F8300128B1206800221146D4
:10D95000D0F8303198472068D0F8300128B12068DD
:10D9600000220221D0F830319847216801F10C00E3
:10D970000BF063FA20B1216801F10C000BF057FAAB
:10D9800000BFD8E76D73672D3E636F6E6E2D3E74DA
:10D99000797065203D3D204E4554434F4E4E5F54B7
:10D9A00043500000626C6F636B696E6720636F6E3B
:10D9B0006E65637420696E2070726F677265737331
:10D9C00000000000616C726561647920777269748F
:10D9D000696E67206F7220636C6F73696E670000F9
:10D9E00010B504462068007800F0F000202806D129
:10D9F000216848680FF030FB0020207101E0FA2018
:10DA00002071216801F10C000BF011FA10BD00002B
:10DA100010B504462068406800284DD0207C28B10D
:10DA20002168A06849680968016004E02168A0686D
:10DA3000496849680160002020712068007800F082
:10DA4000F000102825D020280CD040282DD1207C93
:10DA500028B120684068017CE068018001E0F32083
:10DA6000207128E0207C28B120684068418AE06865
:10DA700001800DE020684068007C00F0040010B9CF
:10DA8000F320207104E020684068818AE06801800A
:10DA900011E0207C18B120684068408B02E02068CB
:10DAA0004068808BE168088005E000BF06A0FAF7B7
:10DAB0003DFF00BF00BF01E0F3202071216801F1AC
:10DAC0000C000BF0B4F910BD696E76616C696420CE
:10DAD0006E6574636F6E6E5F747970650000000030
:10DAE00010B50446002020712068406810B9204617
:10DAF00009F0CCFC216801F10C000BF098F910BD85
:10DB000070B504460020207120684068B0B12068DC
:10DB10000078102812D1A56800BFB5F5803F02D368
:10DB20004FF6FF7000E0A8B206462168486831460B
:10DB30000DF0AAFEAD1B002DEFD100BF216801F151
:10DB40000C000BF074F970BD70B50446206890F9B4
:10DB5000080010F1090F03DA2068007A207140E014
:10DB6000F32020712068406800283AD020680078AF
:10DB700000F0F000202819D0402830D1A0680830EB
:10DB800010B1A068806838B9A2681168226850682E
:10DB90000AF012FC207108E0A36803F1080219687A
:10DBA000236858680AF012FC207119E0A068083058
:10DBB00010B1A068806838B9A268116822685068FE
:10DBC0000FF0C0FB207109E0A568AB8905F10802E0
:10DBD0002968256868680FF0BFFB207100E000BF6E
:10DBE00000BF216801F10C000BF021F970BD0000AD
:10DBF00010B50446206890F9080010F1090F03DA07
:10DC00002068007A207133E02068007810282DD138
:10DC10002068407810B1FB20207129E0206840681E
:10DC200008B301202168487000BF2068D0F82C019B
:10DC300018B92068D0F8280110B111A0FAF776FEC3
:10DC400000BF00BFE06810B914A0FAF76FFE00BF74
:10DC50002068C0F82C4100202168C1F82801206804
:10DC600000F026F810BDF320207101E0FA202071A9
:10DC7000216801F10C000BF0DAF800BFF2E70000B8
:10DC8000616C72656164792077726974696E67206E
:10DC90006F7220636C6F73696E6700006D73672D20
:10DCA0003E6D73672E772E6C656E20213D2030000F
:10DCB0002DE9F84F04460020009094F8240100F06C
:10DCC000020028B9D4F82C01007C00F0040008B14F
:10DCD000012000E000200746D4F82C0190F81080C5
:10DCE00000BF14B973A0FAF721FE00BF00BF60782F
:10DCF000012802D073A0FAF719FE00BF00BFD4F8C4
:10DD00002C0110B977A0FAF711FE00BF00BF6068C0
:10DD100010B97BA0FAF70AFE00BF00BFD4F82811A3
:10DD2000D4F82C01C068814202D37BA0FAF7FEFD33
:10DD300000BFD4F81C01E0B10BF05AF8D4F82C1154
:10DD40004969401AD4F81C11884212DB0120009066
:10DD5000D4F8280130B96FF006050021D4F82C0161
:10DD6000C16097E00025D4F82811D4F82C01C160D7
:10DD700090E0D4F82C018068D4F8281100EB010B56
:10DD8000D4F82C01C068D4F82811A0EB010ABAF528
:10DD9000803F04D34FF6FF7648F0020801E01FFAF7
:10DDA0008AF66068B0F86690B14507DA4E461FB152
:10DDB00026B96FF0060519E048F0020800BFD4F854
:10DDC00028018119D4F82C01C068814202D95FA0D2
:10DDD000FAF7ACFD00BF43463246594660680EF084
:10DDE0009FFA05460DB1681C58BB00BFA7B1D4F817
:10DDF0002C01C068B0420FD9D4F8300128B13246A6
:10DE000003212046D4F83031984794F8240140F09B
:10DE1000100084F8240114E06068B0F8660040F651
:10DE20006931884204DD6068B0F86800082808DBC2
:10DE3000D4F8300128B1324603212046D4F83031DD
:10DE40009847D5B9D4F828013044C4F82801D4F84B
:10DE50002811D4F82C01C068814200D04FB1D4F809
:10DE60002811D4F82C01C160012000900020C4F8D2
:10DE7000280160680CF01EFA0CE0681C20B91FB97C
:10DE800060680CF017FA05E0012000900021D4F83A
:10DE90002C01C160009850B1D4F82C01057100200C
:10DEA000C4F82C01607004F10C000AF0C0FF0020DF
:10DEB000BDE8F88F636F6E6E20213D204E554C4CAF
:10DEC00000000000636F6E6E2D3E737461746520F8
:10DED0003D3D204E4554434F4E4E5F5752495445A9
:10DEE00000000000636F6E6E2D3E63757272656E8A
:10DEF000745F6D736720213D204E554C4C0000002F
:10DF0000636F6E6E2D3E7063622E74637020213DD0
:10DF1000204E554C4C000000636F6E6E2D3E7772A4
:10DF20006974655F6F6666736574203C20636F6E0D
:10DF30006E2D3E63757272656E745F6D73672D3EF4
:10DF40006D73672E772E6C656E000000646F5F77CF
:10DF5000726974656D6F72653A20696E76616C697D
:10DF600064206C656E67746821000000002100E089
:10DF7000491C032906D201EB4100054A52F8200052
:10DF80000028F5D1032901D0012070470020FCE7CB
:10DF90002CE300202DE9F04707460E463C4600BF23
:10DFA00014B938A0FAF7C2FC00BF00206060F2F795
:10DFB00007F9814626724846F2F706F9657800208F
:10DFC0006070D4F8300128B1002204212046D4F832
:10DFD00030319847D4F8300128B10022114620464C
:10DFE000D4F830319847D4F8300128B1002202210A
:10DFF0002046D4F83031984704F110000AF0F1FEC1
:10E0000020B1002104F110000AF0DEFE04F19400BA
:10E010000AF0E7FE20B1002104F194000AF0D4FEDA
:10E02000012D03D0042D01D0032D21D194F824011A
:10E03000C0F3800800BF94F8240120F0040084F8A5
:10E04000240100BFB8F1000F11D100BFD4F82C019A
:10E0500010B910A0FAF76AFC00BFD4F82C010671C1
:10E060000020C4F82C0104F10C000AF0E0FE07E0E7
:10E0700000BFD4F82C0110B10DA0FAF757FC00BF77
:10E08000BDE8F087636F6E6E20213D204E554C4CED
:10E0900000000000636F6E6E2D3E63757272656ED8
:10E0A000745F6D736720213D204E554C4C0000007D
:10E0B000636F6E6E2D3E63757272656E745F6D7305
:10E0C00067203D3D204E554C4C000000F8B50646FB
:10E0D0000020009096F83100C0F3001000284FD0C7
:10E0E0002CA0FAF723FC2F480068002842D000201B
:10E0F00000904FF4805200210120F5F723F900BF72
:10E100000098401C009001210846F5F73DF800F00A
:10E11000200018B9244900988842F1D31021012029
:10E12000F5F732F8044604F0040020B14FF4006023
:10E130001C49086202E000201A49086204F002004B
:10E1400018B100201749486103E04FF48040154999
:10E15000486116480568134840691249096A08432E
:10E160000543124805604FF6FF70F4F778F80F4842
:10E1700005680560F5F76CF80D4808F075F807E0DC
:10E180000CA0FAF7D3FBF5F773F8094807F0C4FFC2
:10E19000F8BD00006E6574776F726B20697320752F
:10E1A00070000000E4D90020FFFF0400008002405E
:10E1B000ACD900206E6574776F726B206973206430
:10E1C0006F776E002DE9FC4705468846164600BF6E
:10E1D00025B94EA0FAF7AAFBBDE8FC8700BF7089FD
:10E1E0002A2805DA00BF00BF304608F095FFF3E7A4
:10E1F000776807F10E042088B0F5807F08D1207978
:10E20000062805D16079042802D16088082805D045
:10E2100000BF00BF304608F07FFFDDE7D4F80E00F6
:10E220000190A0690090281D08B1686810B94FF0EE
:10E23000000907E000986968884201D1012000E0E8
:10E2400000208146B9F1000F01D0012000E002203A
:10E25000034604F1080201A9284600F027FDE088E2
:10E26000B0F5807F03D0B0F5007F45D13DE000BF21
:10E2700000BFB9F1000F2FD000BF00BF022004F093
:10E280001AFEE080D4F80E00A0616868C4F80E00A1
:10E2900000BF95F82A00062802D02048FAF746FB6E
:10E2A00000BFA068C4F81200A089E082A0683860AE
:10E2B000A089B880D8F80000A060B8F80400A08158
:10E2C000D8F80000C7F80600B8F804007881314695
:10E2D0002846AA69904707E0281D08B1686808B970
:10E2E00000BF01E000BF00BF09E000BF00BF01A9FF
:10E2F0002846FCF721F902E000BF00BF00BF00BFC5
:10E30000304608F009FF00BF66E700006E657469DB
:10E310006620213D204E554C4C000000B48C040872
:10E3200070B50546002412E004EB8400094901EBB6
:10E330008000867C4EB104EB840001EB8000806895
:10E34000A84202D1204600F037F9601CC4B20A2C62
:10E35000EADB70BD046D01202DE9FE4F06468846BC
:10E360004FF00A09CA460A270024002002900190B3
:10E37000BB46009000BF69E004EB8400674901EBF5
:10E380008000857C0A2F04D11DB900BF00BF67B291
:10E390005AE0002D58D000BF012D04D0022D02DA22
:10E3A0005FA0FAF7C3FA00BF6EB104EB84015B4AC9
:10E3B00002EB810130684968884204D100BF00BF88
:10E3C00060B2BDE8FE8F012D2AD104EB84005349D1
:10E3D00051F8200088B104EB840001EB8000C17C7F
:10E3E0000098814230DB4FFA84FB04EB84004B49F8
:10E3F00001EB8000C07C009026E004EB84004749DC
:10E4000001EB8000C17C029881421DDB4FFA84F948
:10E4100004EB8400414901EB8000C07C029013E0D2
:10E42000022D11DB04EB84003C4901EB8000C17C30
:10E430000198814208DB4FFA84FA04EB84003749E3
:10E4400001EB8000C07C0190601CC4B20A2C93DBFD
:10E4500008F0020020B90A2F07D108F0010020B906
:10E4600000BF00BF4FF0FF30ABE70A2F02DAFCB26B
:10E4700000BF2EE0BAF10A0F0EDA0AF0FF0400BF67
:10E4800000BF00BF04EB8400244951F8200010B104
:10E4900033A0FAF74BFA12E0B9F10A0F03DA09F0E8
:10E4A000FF0400BF0BE0BBF10A0F03DA0BF0FF041F
:10E4B00000BF04E000BF00BF4FF0FF3081E700BFA6
:10E4C0000A2C02DB2CA0FAF731FA00BF204600F03C
:10E4D00073F800BF0A2C02DB27A0FAF727FA00BF67
:10E4E00000BF04EB84000D4901EB8000807C10B17B
:10E4F00026A0FAF71BFA00BF36B104EB8401074AE5
:10E5000002EB810130684860002004EB8401034A7B
:10E5100002EB8101C87460B253E70000046D012072
:10E520007374617465203D3D204554484152505FED
:10E5300053544154455F50454E44494E47207C7CDE
:10E54000207374617465203E3D204554484152500B
:10E550005F53544154455F535441424C45000000C1
:10E560006172705F7461626C655B695D2E71203DE4
:10E570003D204E554C4C000069203C204152505FDC
:10E580005441424C455F53495A4500006172705FE7
:10E590007461626C655B695D2E7374617465203DA6
:10E5A0003D204554484152505F53544154455F45C6
:10E5B0004D5054590000000010B5044604EB84008F
:10E5C000194951F8200070B100BF00BF04EB84016D
:10E5D000154A52F8210008F09FFD002004EB840149
:10E5E000114A42F82100002004EB84010E4A02EB9C
:10E5F0008101887404EB840102EB8101C87404EB8F
:10E60000840102EB8101886004EB840102EB81014B
:10E61000486004EB8400114601EB800003490A685E
:10E62000C2608988018210BD046D0120AA86040899
:10E630002DE9FC4704460F461546A94600BF14B90C
:10E6400051A0FAF773F900BF00BF17B952A0FAF74B
:10E650006DF900BF00BF15B952A0FAF767F900BF06
:10E660000E21384608F0F8FD28B100BF00BF6FF05A
:10E670000100BDE8FC872146286802F06BFF10B15D
:10E68000DFF8308177E0287800F0F000E02815D13D
:10E6900001208DF8000000208DF801005E208DF82B
:10E6A0000200687800F07F008DF80300A8788DF8EC
:10E6B0000400E8788DF80500E8465BE02868A1686A
:10E6C0000840D4E901121140884210D0288880B255
:10E6D0004FF6A96188420AD004F10C0020B1E0682D
:10E6E00010B104F10C0902E06FF00300C1E73248F9
:10E6F000007800EB8000314901EB8000807C02282B
:10E7000012DB2D49097801EB81012C4A02EB8101D2
:10E71000D9F800004968884206D12748027839466E
:10E72000204600F04DF8A4E700261BE006EB86002B
:10E73000224901EB8000807C022811DB06EB860178
:10E740001E4A02EB8101D9F800004968884207D1CE
:10E7500019490E70F2B23946204600F031F888E7C8
:10E76000701C46B20A2EE1DB3A464946204600F0CC
:10E7700081F87EE700BF434604F12B02394620466C
:10E7800000F022FA75E700006E6574696620213D8D
:10E79000204E554C4C0000007120213D204E554C20
:10E7A0004C00000069706164647220213D204E5568
:10E7B0004C4C0000A4860408A4010020046D012034
:10E7C00070B505460E46144600BF04EB84001C4994
:10E7D00001EB8000807C022802DA1AA0FAF7A6F882
:10E7E00000BF04EB8400164901EB8000807C022806
:10E7F00017D104EB840001EB8000C07CE42810DB1F
:10E8000004EB84000A4602EB8000011D284600F05C
:10E81000C3F930B9032004EB8401094A02EB8101FA
:10E82000887404EB8400064901EB800000F10C03BE
:10E8300005F12B023146284600F0C6F970BD0000F4
:10E84000046D01206172705F7461626C655B61725E
:10E85000705F6964785D2E7374617465203E3D203D
:10E860004554484152505F53544154455F535441BD
:10E87000424C45002DE9F05F80460F46164608F1F0
:10E880002B094FF0FF3A4146386802F063FE38B971
:10E89000387800F0F000E02802D00FB1386828B9CD
:10E8A00000BF00BF6FF00D00BDE8F09F01213846AA
:10E8B000FFF752FD0446002C06DA00BF00BF0EB180
:10E8C00000BF00BF2046EFE704EB8400534901EB93
:10E8D0008000807C30B9012004EB84014F4A02EBB8
:10E8E0008101887400BF04EB84004C4901EB800077
:10E8F000807C012809D004EB840001EB8000807C3F
:10E90000022802DA46A0FAF711F800BF04EB8400EF
:10E91000424901EB8000807C012800D03EB9394695
:10E92000404600F039F982460EB95046BCE700BFB8
:10E9300016B945A0F9F7FAFF00BF04EB8400374988
:10E9400001EB8000807C02280FDB42490C7004EB55
:10E950008400324901EB800000F10C034A46314645
:10E96000404600F031F9824656E004EB84002B4922
:10E9700001EB8000807C01284ED14FF0000B354622
:10E9800011E000BF68892989884204D1286810B144
:10E9900031A0F9F7CBFF00BF287B012802D04FF050
:10E9A000010B02E02D68002DEBD100BFBBF1000F81
:10E9B00010D029890022032007F0EAFF05466DB137
:10E9C0003146284608F06AFA40B1284608F0A4FB10
:10E9D000002503E03546284608F04AFDBDB104EBAA
:10E9E00084000E4951F8200040B100BF00BF04EB85
:10E9F00084010A4A52F8210008F08EFB04EB8400DF
:10EA0000064941F820504FF0000A00BF03E000BF64
:10EA100000BF4FF0FF3A00BF504645E7046D0120AC
:10EA20006172705F7461626C655B695D2E737461A5
:10EA30007465203D3D2050454E44494E47206F723D
:10EA400020535441424C45007120213D204E554CED
:10EA50004C000000A40100206E6F207061636B65A4
:10EA6000742071756575657320616C6C6F77656472
:10EA7000210000002DE9F84F0746884691469A4646
:10EA8000DDF828B00020009000BF17B930A0F9F7DA
:10EA90004DFF00BF00222A21032007F079FF054621
:10EAA0002DB900BF00BF4FF0FF30BDE8F88F00BFA9
:10EAB00068892A2802DA2AA0F9F738FF00BF6E68B1
:10EAC00006F10E0400BF00BF0D9804F0F4F9E080D9
:10EAD00000BF97F82A00062802D02E48F9F726FF33
:10EAE00000BFDAF80000A060BAF80400A0810B981B
:10EAF0000168C4F812108088E082D9F80000306004
:10EB0000B9F80400B080D8F80000C6F80600B8F8DC
:10EB100004007081DBF80000C4F80E000C98006857
:10EB2000A0614FF480702080082060800620207152
:10EB3000042060714FF4C160B08129463846BA693B
:10EB400090470090284608F0E7FA00250098ACE7C7
:10EB50006E6574696620213D204E554C4C000000C6
:10EB6000636865636B20746861742066697273748E
:10EB700020706275662063616E20686F6C6420731C
:10EB80007472756374206574686172705F68647212
:10EB900000000000B48C04087FB504460D4600BF99
:10EBA00000BF0121064A201D04F12B038DE825003A
:10EBB0000391044A19462046FFF75CFF04B070BD7C
:10EBC000AA860408A48604082DE9F04104460E46EE
:10EBD00017469846756800BF94F82A00062802D0A8
:10EBE0000C48F9F7A3FE00BFD8F800002860B8F879
:10EBF0000400A8803868C5F80600B8886881082035
:10EC0000A88100BF00BF31462046A2699047BDE8F9
:10EC1000F0810000B48C040870B500BF00BF002470
:10EC20003FE004EB8400204901EB8000857C35B394
:10EC300004EB840001EB8000C07C401C04EB8401E9
:10EC4000194A02EB8101C87404EB8400114601EB00
:10EC50008000C07CF0280DDA04EB840001EB80001A
:10EC6000807C01280CD104EB840001EB8000C07C87
:10EC7000022805DB00BF00BF2046FFF79DFC0EE029
:10EC800004EB8400084901EB8000807C032806D156
:10EC9000022004EB8401044A02EB81018874601CA9
:10ECA000C4B20A2CBDDB70BD046D01202DE9F04714
:10ECB00006460D461746984600BF96F82A000628D5
:10ECC00002D02DA0F9F732FE00BF00BF00BF5DB13A
:10ECD000286848B13146286802F03CFC20B9287801
:10ECE00000F0F000E02805D100BF00BF6FF00D007C
:10ECF000BDE8F08741462846FFF72EFB0446002C6E
:10ED000001DA2046F4E7022004EB8401244A02EBF6
:10ED10008101887404EB8400114601EB8000866059
:10ED200000BF00BF04EB840001EB80003968C160C4
:10ED3000B9880182002004EB840102EB8101C874D0
:10ED400004EB8400114651F8200098B104EB8400D4
:10ED500051F82090002004EB840142F821003B464A
:10ED600006F12B0249463046FFF72EFF484608F0D1
:10ED7000D3F900BF0020BBE76E657469662D3E685D
:10ED800077616464725F6C656E203D3D2045544838
:10ED90004152505F4857414444525F4C454E000039
:10EDA000046D01202DE9F04104460E464FF00E0897
:10EDB00060890E2800DC4EE0656800BF00BFAF89A7
:10EDC000287800F00100B0B12878012809D16878CE
:10EDD00088B9A8785E280ED1607B40F0100060737F
:10EDE00009E006221E492846F1F7D0FA18B9607BDF
:10EDF00040F008006073082F03D0B7F5C16F25D12C
:10EE000017E096F8310000F0200000B923E0C8F1C7
:10EE1000000001B2204608F01FFA28B100BF11A07F
:10EE2000F9F784FD00BF16E03146204602F0C0FC31
:10EE30000DE096F8310000F0200000B90BE022460A
:10EE400006F12B013046FFF7BDF900E003E000BFFB
:10EE50000020BDE8F081204608F05EF90020F8E7C8
:10EE6000A486040843616E2774206D6F7665206F59
:10EE70007665722068656164657220696E207061D4
:10EE8000636B65740000000010B5044600BF14B940
:10EE900014A0F9F74BFD00BF652084F832006E2105
:10EEA00033200155134860611348A061204603F0E8
:10EEB000BBFB1248006820B90020F7F799F80F490A
:10EEC00008600F48006820B90120F7F791F80C4955
:10EED000086003230B4A21460B48F7F7EBF90020A3
:10EEE00010BD00006E6574696620213D204E554CB2
:10EEF0004C00000031E60008C927010898010020F5
:10EF00009C010020006501200DEF000808B50646B1
:10EF1000354600BF6A4600210A480068F7F702F943
:10EF200000BF284603F0D4FB0446002CF2D029464B
:10EF300020462A69904720B100BF00BF204608F054
:10EF4000EBF8EEE79801002010B50446012001F02F
:10EF5000E3FB0022AFF20F014FF47A7009F090FF4B
:10EF600010BD00002DE9F05F0746884617B3D7F8BB
:10EF70001841002C18DAF1F723F98346D7F8180165
:10EF800000280CDAB8F1000F04D1D7F81801401EA0
:10EF9000C7F818015846F1F717F9BDE8F09FD7F800
:10EFA00018415846F1F710F9204601F09DFB05463F
:10EFB0000DB9F2E7F1E7F1F703F98346B8F1050F70
:10EFC00017D2DFE808F003080D1013006889401C11
:10EFD00000B2688113E06889401E00B268810EE0CB
:10EFE0000120A8810BE00020A88108E00120E88131
:10EFF00005E000BF38A0F9F799FC00BF00BF00BFD3
:10F00000686918B95846F1F7DFF8C6E700BF364817
:10F0100006685AE07069002848D18146B5F90A00AF
:10F0200000280FDDB16869B1E11704EB5171C91017
:10F03000B268515C04F0070301229A40114009B103
:10F040004FF00109A88990B1B9F1000F0FD1F16813
:10F0500069B1E11704EB5171C910F268515C04F019
:10F06000070301229A40114009B14FF00109E889D4
:10F0700090B1B9F1000F0FD1316969B1E11704EB1B
:10F080005171C9103269515C04F0070301229A40A2
:10F09000114009B14FF00109B9F1000F05D001206D
:10F0A000706106F1180009F0C2FE00BF0F48D0F8E9
:10F0B00000A05846F1F788F8F1F782F883460B482C
:10F0C0000068824500D0A2E73668002EA2D15846DB
:10F0D000F1F77AF800BF60E7756E6B6E6F776E20A0
:10F0E0006576656E74000000880100208C010020A8
:10F0F00070B50546284600F04DFD04465CB928462B
:10F100000EF072FA044634B9686AFBF75DF90446FA
:10F110000CB900202860204670BD00002DE9F74F93
:10F1200090B0914610A801F091FA0F900F98002826
:10F1300003DA0B2013B0BDE8F08F1198012801DD30
:10F140001320F7E7A9F1010000EA090008B1132034
:10F15000F0E7FE490F9851F820B0BBF1000F01D144
:10F160000C20E7E700208BF800000F98C0B20C904D
:10F1700000200B900C98FDF701F80190019800F029
:10F18000010008B10320D5E7019800F0040008B1A0
:10F190000A20CFE700BF04AA01210C98FCF7F6FF74
:10F1A00010B90498802801D20120C3E7119808B152
:10F1B000002000E03F2080460498A0EB0800049067
:10F1C000B9F1000F13D14FF4FA610498B0FBF1F0DC
:10F1D0000A904FF0000A01E00AF1010ADC4830F819
:10F1E0001A100A988142F7D8DA4830F81A904FEA94
:10F1F0005929B9F1000F01D14FF00109B9F1800F80
:10F2000001D94FF080090498B0FBF9F7012540F6C9
:10F21000F670874200D302254FF6F670874200D37E
:10F220000325032D0AD1082000EB870000F2FF1010
:10F23000460A202003900020029011E0012D05D104
:10F2400007EB4700401C4008C01C01E07800001D8F
:10F25000064606F2FF10460A012003902020029085
:10F260000398404407900798304406900299069806
:10F270000844059005984844A0EB0800049988428A
:10F2800001D90E2056E709AA03210C98FCF77EFF4E
:10F2900028B9099818B10998B0F5004F01D9012093
:10F2A0000990099905980844401E491E8843099011
:10F2B00009990598081A0990032D08D1099903980E
:10F2C00008440390099907980844079001E00998B9
:10F2D0000644DDE90301081A811B0298081AB0FBF5
:10F2E000F9F7022D03D140F6F670874205D3032DBE
:10F2F00005D14FF6F670874201D20E201AE7032D92
:10F3000002D10C200D9010E0012D06D10498B0F52B
:10F31000803F02D201200D9007E00498B0F5803FB5
:10F3200001D2042000E006200D9000BF119810B11A
:10F33000F0200E9044E04FF4007200210BF13000F9
:10F3400004F0F4FC0BF5F77401206070A07000204D
:10F35000E0700D982071FE206071049840443F21B8
:10F36000B0FBF1F0FF21B0FBF1F009903F210998CB
:10F3700041EA9000A0710998E0713F2020720021BD
:10F380006172A172E172049820730498010A61739A
:10F390000498010CA1730498010EE17355218BF8B8
:10F3A0002E12AA218BF82F12012300220BF130011B
:10F3B0000C98FCF73BFF08B10120BBE6F8200E904B
:10F3C0000BF130044FF400720021204604F0AEFC33
:10F3D0000B2261A1204604F0D6FA4FF4007A84F89B
:10F3E0000BA04FEA1A21217384F80D900398A073A3
:10F3F0000398010AE17301202074032D01D100203C
:10F4000001E04FF40070824684F811A04FEA1A21FF
:10F41000A1740498B0F5803F05D20498E074049874
:10F42000010A217510E0049884F820000498C0F3C4
:10F430000721212001550498C0F3074122200155DE
:10F440000498010E232001550E9860753F20207608
:10F4500000216176FF20A076E17684F81C804FEAD7
:10F46000182161774FEA1841A1774FEA1861E177D7
:10F4700001F0E4F80990032D3ED1099884F8430087
:10F480000998C0F30721442001550998C0F30741AA
:10F49000452001550998010E4620015584F8246045
:10F4A000C6F3072125200155C6F307412620015543
:10F4B000310E27200155022084F82C0000212D2038
:10F4C00001552E2001552F200155012084F83000D0
:10F4D00031200155062084F8320033200155802068
:10F4E00084F84000292084F8420013221DA104F171
:10F4F000470004F048FA1FE0099884F827000998AB
:10F50000C0F30721282001550998C0F3074129209D
:10F5100001550998010E2A200155A675310AE17599
:10F52000802084F82400292084F82600132212A1C8
:10F5300004F12B0004F027FA552084F8FE01AA21DB
:10F5400040F2FF100155012342461FE020E3002056
:10F55000A2840408B8840408EBFE904D53444F5332
:10F56000352E30004E4F204E414D45202020204664
:10F5700041543332202020004E4F204E414D452033
:10F5800020202046415420202020200021460C9895
:10F59000FCF74CFE08B10120CCE5032D06D1012378
:10F5A00008F1060221460C98FCF740FE07980890E7
:10F5B0004FF0000A61E04FF400720021204604F091
:10F5C000B5FB0E980990032D14D0012D01D162488E
:10F5D00001E06FF0FF000999084309900998207035
:10F5E0000998000A60700998000CA0700998000E34
:10F5F000E07019E0099860F0FF0009900998207008
:10F600000998000A60700998000CA0700998000E13
:10F61000E070FF202071FF216171A171E171207202
:10F620006172A1720F21E1720898411C0246012308
:10F63000089121460C98FCF7F9FD08B1012079E505
:10F640004FF400720021204604F070FB0120099065
:10F650000EE00898411C02460123089121460C98AF
:10F66000FCF7E4FD08B1012064E50998401C09900D
:10F670000998B042EDD30AF1010ABAF1000F9AD00D
:10F68000032D01D1484600E00298824600BF089849
:10F69000411C02460123089121460C98FCF7C6FD47
:10F6A00008B1012046E5AAF10100B0F1000AEED14F
:10F6B000032D46D15220207060706120A07041203F
:10F6C000E070722084F8E401722140F2E5100155E7
:10F6D0004121401C01556121401C0155781E84F8D0
:10F6E000E801C0F3072140F2E9100155781EC0F38C
:10F6F00007414FF4F5700155781E010E40F2EB10F2
:10F700000155022084F8EC01002140F2ED10015572
:10F71000401C0155401C0155552084F8FE01AA21CA
:10F7200040F2FF100155012308F1010221460C9817
:10F73000FCF77CFD012308F1070221460C98FCF739
:10F7400075FD002211460C98FCF720FD08B1012040
:10F75000F0E40020EEE4000000FFFF00F7B582B007
:10F7600016460398019001A800F070FF0546002D91
:10F7700002DA0B2005B0F0BD0F4850F8254024B147
:10F780002046FAF72BFB00202070029810B10020D1
:10F79000029908700849029841F82500029808B1BA
:10F7A000012E01D00020E5E7002203A902A800F005
:10F7B000EFFB07463846DDE720E300202DE9F7435D
:10F7C000ADF50E7D0546164625B909200DF5117DCE
:10F7D000BDE8F0830020286006F01F0626F0010235
:10F7E0008FA984A800F0D4FB0746002F72D181A80E
:10F7F0008A9001A88C9084A88F9900F0CFFD0746CD
:10F80000899C6FB90CB906270AE026F0010008B1FF
:10F81000012000E00020014684A8FAF799FA074683
:10F8200006F01C00002856D077B1042F08D1FEF74F
:10F830009DFB18B184A8FCF788FB00E01220074666
:10F8400046F00806899C09E0E07A00F0110008B152
:10F85000072703E006F0040000B10827002F38D185
:10F8600006F00800A8B300F0E9FE804684F80E8098
:10F870004FEA1821E1734FEA184121744FEA1861E9
:10F8800061740020E072207700216177A177E17731
:10F890002146849802F020FE81460021204609F08E
:10F8A0003DF9012084990871B9F1000F11D08498B5
:10F8B000D0F82C804946849809F052F8074647B999
:10F8C000A9F101008499C8604146849804F0AAFD1A
:10F8D00007460FE042E06FB9E07A00F0100008B18F
:10F8E000042707E006F0020020B1E07A00F00100F2
:10F8F00000B10727B7B906F0080008B146F02006A6
:10F900008498C06AE8612C6226F0010008B10120E9
:10F9100000E00020014684A801F050FD6862686A9A
:10F9200000B90227D7B9AE710020E871214684984A
:10F9300002F0D2FD2861E07F0106A07F41EA00418C
:10F94000607F41EA0020217F0843E8600020A86032
:10F95000A861849828602868C088A880384635E760
:10F9600033B5ADF5057D04461CB909200DF5077DBD
:10F9700030BD002286A984A800F00AFB0546002DB0
:10F9800033D18498206081A8A06101A8206220461C
:10F99000869900F003FD05460DBB606958B16069AA
:10F9A000C07A00F0100028B16169849802F094FDDB
:10F9B000A06000E0052595B98498C088A08000214A
:10F9C0002046FCF78CFB05464DB9A06840B10021EC
:10F9D000204601F0F3FCE061E06900B9122501E086
:10F9E0000020E061042D00D105250DB1002020602C
:10F9F0002846BBE72DE9FF4F83B0044615469A46DB
:10FA0000DDF810B00020CAF8000020460DF0ECFD33
:10FA10000290029818B1029807B0BDE8F08FE07923
:10FA200008B1E079F8E7A07900F0010008B90720F3
:10FA3000F2E7D4E90210401A00900098854200D9FC
:10FA4000009DA2E02089C0F3080000287ED1206834
:10FA50008078401EA16800EA512000F0FF09B9F14A
:10FA6000000F17D1A06810B92069019004E0616906
:10FA7000206800F06FFD01900198022802D2022058
:10FA8000E071C9E70198401C10B90120E071C3E79B
:10FA90000198606161692068FAF7B8F9064616B9FD
:10FAA0000220E071B8E74E444FEA5528B8F1000F44
:10FAB00029D009EB080021688978884203D9206899
:10FAC0008078A0EB090821684878434632465946B9
:10FAD000FCF788FB10B10120E0719DE7A07900F0F0
:10FAE000400068B1A069801B404509D2A169891B0B
:10FAF0000BEB41204FF4007204F1280103F043FFA7
:10FB00004FEA482737E0A069B04220D0A07900F042
:10FB1000400078B121684878012304F12801A269E6
:10FB2000FCF784FB10B10120E07175E7A07920F0AB
:10FB30004000A071216848780123324604F1280171
:10FB4000FCF750FB18B10120E07165E700E0A66109
:10FB50002089C0F30800C0F50077AF4200D92F46D6
:10FB60002089C0F3080204F1280011183A465846CB
:10FB700003F009FF00BFBB44A0683844A060DAF876
:10FB800000003844CAF80000ED1B002D7FF45AAF86
:10FB9000002041E72DE9F041044620460DF024FD08
:10FBA0000746002F4CD1A07900F02000002847D054
:10FBB000A07900F0400078B121684878012304F171
:10FBC0002801A269FCF732FB10B10120BDE8F081E9
:10FBD000A07920F04000A071E169206804F022FCC7
:10FBE0000746002F2CD1256AE87A40F02000E87201
:10FBF000207B2877A089010A6977E068010CA97742
:10FC0000E068010EE9772846216908F087FF00F0D7
:10FC100015FD0646AE75310AE975310C2976310EAF
:10FC200069760020A8740021E974A07920F02000F2
:10FC3000A071012021680871206808F095FF07462F
:10FC40003846C3E771B5ADF5177D012297A98DA898
:10FC500000F09EF90446002C4FD180A89390CDF877
:10FC600054D28DA8979900F099FB044600BF24B99F
:10FC700002218DA8FAF76CF80446002C3DD1929E23
:10FC80000EB9062404E0F07A00F0010000B1072468
:10FC900031468D9802F020FC0546ECB9F07A00F070
:10FCA0001000C8B1022D01D2022415E028228DA92E
:10FCB00083A803F068FE8595022183A8FCF70FFA5C
:10FCC00004464CB9002183A8FCF7DDF8044604B9CA
:10FCD0000724042C00D100247CB98DA8FCF7CAF9B4
:10FCE000044654B925B129468D9808F039FE0446DA
:10FCF0001CB98D9808F038FF044620460DF5187D94
:10FD000070BD2DE9FF4F83B0044615469B4604980D
:10FD100001900020CBF8000020460DF065FC029019
:10FD2000029818B1029807B0BDE8F08FE07908B1E9
:10FD3000E079F8E7A07900F0020008B90720F2E7BF
:10FD4000A0682844A168884200D20025B5E0208937
:10FD5000C0F30800002877D120688078401EA16891
:10FD600000EA512000F0FF0ABAF1000F1ED1A0688E
:10FD700038B9276957B900212068FAF79DF8074676
:10FD800004E061692068FAF797F8074607B997E039
:10FD9000012F02D10220E071C5E7781C10B90120C3
:10FDA000E071C0E76761206900B92761A07900F0C0
:10FDB000400078B121684878012304F12801A26944
:10FDC000FCF734FA10B10120E071ACE7A07920F023
:10FDD0004000A07161692068FAF718F8064616B964
:10FDE0000220E0719FE756444FEA5529B9F1000F10
:10FDF0002BD00AEB090021688978884203D9206852
:10FE00008078A0EB0A09216848784B463246019970
:10FE1000FCF70CFA10B10120E07184E7A069801BA7
:10FE200048450ED2A069801B019A02EB40214FF495
:10FE3000007204F1280003F0A6FDA07920F0400034
:10FE4000A0714FEA49282BE013E0A069B0420FD01F
:10FE5000D4E9020188420BD2216848780123324656
:10FE600004F12801FCF7BEF910B10120E0715AE756
:10FE7000A6612089C0F30800C0F50078A84500D924
:10FE8000A8462189C1F3080204F12801501842460E
:10FE9000019903F078FDA07940F04000A07100BF07
:10FEA000019840440190A0684044A060DBF8000045
:10FEB0004044CBF80000A5EB0805002D7FF447AFC8
:10FEC00000BFD4E90201884201D9A068E060A079AE
:10FED00040F02000A071002025E700002DE9F0414E
:10FEE00002460F46802A01DA10462FE01FB1184B58
:10FEF00045F2205602E0174B45F22056002510240B
:10FF000016E0A6EB050C0CEBDC7805EB68014FEA7C
:10FF1000410C33F81CC0944500D10BE04FEA410C72
:10FF200033F81CC0944501DA0D4600E00E46641E0D
:10FF3000002CE6D100BF34B14FF0010C0CEB410CAA
:10FF400033F81CC001E04FF0000C6046BDE8F081C2
:10FF5000502C0308CCD701080246002100E0491CC0
:10FF6000094830F8110020B1074830F811009042DC
:10FF7000F5D1054830F8110018B1044830F81100E7
:10FF800070471046FCE70000D4800408B4820408DF
:10FF90002DE9F74F88B0002108980160099800F01A
:10FFA00055FB07900798002803DA0B200BB0BDE83B
:10FFB000F08FD649079851F820400CB90C20F5E78E
:10FFC00008980460207878B16078FCF727F98046BB
:10FFD00008F0010040B90A9820B108F0040008B107
:10FFE0000A20E3E70020E1E7002020700798607016
:10FFF0006078FCF7C3F8804608F0010008B10320E0
:020000040801F1
:10000000D4E70A9820B108F0040008B10A20CDE72F
:10001000002739462046F9F749FE0546012D01D053
:100020006DBB2CE0002614E004F5F77101EB06101F
:10003000017951B1C17A0A06817A42EA0142417AD4
:1000400042EA0121027A114300E000214DF8261016
:10005000761C042EE8D3002606B1761E00BF5DF89C
:10006000267027B139462046F9F720FE00E002202D
:1000700005461DB1701C06460428F0D300BF032DB1
:1000800001D1012092E70DB10D208FE73B20015DEA
:1000900094F83C0041EA0020B0F5007F01D00D202B
:1000A00084E74620015D94F8470041EA0029B9F150
:1000B000000F0ED194F85700010694F8560041EA5B
:1000C000004194F8550041EA002094F8541040EAA9
:1000D0000109C4F818904020005DE070E078012824
:1000E00004D0E078022801D00D205FE7E07809FB1A
:1000F00000F93D20005DA070A07818B1A078411EE5
:10010000084008B10D2051E74120015D94F84200FC
:1001100041EA00202081207A00F00F0008B10D2074
:1001200044E74320015D94F8440041EA002BBBF111
:10013000000F0ED194F85300010694F8520041EAE2
:10014000004194F8510041EA002094F8501040EA30
:10015000010B3E20015D94F83F0041EA002004902D
:10016000049808B90D2021E704984844218900EB40
:10017000111006900698834501D20D2016E70698C7
:10018000ABEB0000A178B0FBF1FABAF1000F01D19E
:100190000D200BE7012540F6F670824500D30225BD
:1001A0004FF6F670824500D303250AF10200606124
:1001B000E76104983844206206983844A062032D11
:1001C00016D1208908B10D20F0E694F85F000106F1
:1001D00094F85E0041EA004194F85D0041EA002095
:1001E00094F85C100843606260698000059014E038
:1001F000208908B90D20D9E6206A48446062022DA2
:1002000002D16069400007E0207D00F001006169D3
:1002100001EB410100EB51000590A169059800F246
:10022000FF10B1EB502F01D20D20BFE64FF0FF3091
:100230002061E06080206071032D5AD194F8601035
:1002400094F8610041EA0020012852D1791C20462F
:1002500004F0E8F8E8BB0020607194F82E1294F8DE
:100260002F0241EA00204AF65521884241D133202D
:10027000005D01063220005D41EA00413120005D51
:1002800041EA002094F8301008432149884230D1D7
:1002900094F81702010694F8160241EA004194F816
:1002A000150241EA002094F81412084319498842C3
:1002B0001FD194F81B02010694F81A0241EA00418A
:1002C00094F8190241EA002094F8181208432061BA
:1002D00000E00EE094F81F02010694F81E0241EAC5
:1002E000004194F81D0241EA002094F81C120843D2
:1002F000E060257008480088401C80B206490880EC
:10030000E0802046F9F76AFD00204FE620E3002058
:10031000525261417272416184000020F0B504467E
:100320001D464D730F27CF7200270F738F76BC4683
:1003300081F81BC0571E07EB870C0CEBC706002784
:1003400038463B4600BF4FF6FF77B84203D03746EA
:10035000761C34F81700DFF840C01CF803C001F821
:100360000C000712DFF830C01CF803C08C448CF876
:10037000017008B94FF6FF705F1C3B460D2FE2D3AA
:100380004FF6FF77B84202D034F816700FB942F03A
:1003900040020A70F0BD0000948404082DE9F34186
:1003A0000446019800782F2803D0019800785C2833
:1003B00002D10198401C01900020A06001980078B3
:1003C000202807D200212046FBF789FE05460020A1
:1003D000606128E000BF01A92046F9F7D9FD054674
:1003E00005B11FE02046FBF751FC0546A069C67A1F
:1003F0003DB1042D04D100BF06F0040000B905256D
:1004000010E006F0040000B10CE06769F87A00F033
:10041000100008B9052505E03946206802F05CF8AF
:10042000A060D8E700BF2846BDE8FC8170B504464F
:100430000D46E1B20548F8F77BF900BF802103487B
:10044000F7F778FE0028F9D0204670BD004800403C
:100450002DE9F04104460D46666800206060208169
:100460002061EFF7ADFE0746002020603846EFF729
:10047000ABFE3EB11DB1304606F04EFE02E0304606
:1004800004F0D8FFBDE8F0812DE9FC4707468A4615
:1004900090461E460B225146384603F074FA052E4C
:1004A00018D9304610E038F8021B00250AE00A4649
:1004B00060F35F021046491000F480320AB1234A0B
:1004C00050406D1C102DF2D3B8F80020002AEAD15C
:1004D000064600BF072500BF06F00F0000F13009F7
:1004E000B9F1390F03DD09F1070000F0FF092846D3
:1004F0006D1E0DF800903609002EEDD17E200DF80E
:10050000050000240BE0385D812807DB385DFE28FC
:1005100004DC681EA04200D106E0641C641CAC42EE
:1005200002D2385D2028EED100BF00BF082D04D2D2
:1005300028466D1C1DF8001000E020212046641C98
:100540003954082CF2D3BDE8FC87000021100100CB
:100550002E2070472DE9F04105460C46022C02D3AF
:100560006869A04202D80120BDE8F08128780128FE
:1005700004D002282CD003285AD13DE0274607EBAF
:100580005707286A00EB5721284603F04BFF00B1BC
:1005900050E0C7F3080105F1300010F801807F1C1E
:1005A000286A00EB5721284603F03CFF00B141E0E8
:1005B000C7F3080105F13000405C48EA002804F068
:1005C000010010B14FEA1810CEE7C8F30B00CBE7DB
:1005D000286A00EB1421284603F024FF00B129E02B
:1005E00040F2FF1000EA440105F130000E183078A7
:1005F000717840EA0120B7E7286A00EBD411284659
:1006000003F010FF00B115E040F2FF1000EA840192
:1006100005F130000E18F0780006B17840EA01408C
:10062000717840EA01203178084320F070409BE760
:10063000012099E700BF4FF0FF3095E70048704771
:100640000000E24400487047347A002070B502464A
:100650004FF0FF301568E5B1116800E0491C0D78D6
:10066000202D02D30D783A2DF8D10D783A2D0FD1E7
:10067000146814F8015BA5F130030A2B07D28C42F1
:1006800005D1032B03D218464D1C2946156070BDB9
:10069000002000BFFBE72DE9F04105460E46174656
:1006A000002405B116B90020BDE8F081AC685FB147
:1006B00000E024688CB1206A78B13046216AEFF7F7
:1006C00057FE0028F5D108E000E024682CB1304640
:1006D000216AF9F7C7FA0028F7D10CB1206A08B9E6
:1006E0000020E1E72046DFE70146002901DB082979
:1006F00003DB00BF00BF0020704701EB4100054B4A
:1007000003EBC002106818B900BF00BF0020F3E778
:100710001046F1E7C05B012070B5054600F030F8E7
:1007200004461548007800F00100D0B11248007866
:1007300000F0100050B1F4B9104805F050FD0E481B
:10074000006820F010000C49086014E09CB10B48D0
:1007500005F05AFD0848006840F01000064908609E
:1007600009E044B1054801F05FFF044805F04CFD85
:100770000248FBF7CDF870BD64000020ACD9002022
:1007800010B501210846F2F7FFFC00F0040008B1A3
:10079000012010BD0020FCE710B50446204602F001
:1007A00001F910BD2DE9F04186B007460C4615460B
:1007B00000220121022002F0F9FF0646002E04DA91
:1007C0006FF0010006B0BDE8F08145BB002000904D
:1007D0006B462A4A69463846FCF762FB00200590C2
:1007E00005E00A20F5F79EFF05980A30059000986D
:1007F00018B90598B0F5FA6FF3DB0598B0F5FA6F04
:1008000005DB1FA0F8F792F86FF00100DAE7684601
:1008100001F0DEFD804601F017FD029003E038464E
:1008200001F012FD029010208DF8040002208DF8D6
:100830000500A0B202F03FFBADF8060000200390D7
:100840000490102201A9304602F0E0F828B111A06E
:10085000F8F76CF84FF0FF30B4E740F6B830059089
:10086000042005AB41F20602D11F0090304602F091
:10087000A9FD0EA0F8F75AF83046A3E7E10D0108EC
:10088000646E7320676574206661696C757265209B
:100890000A000000636F6E6E656374207365727684
:1008A0006572206572726F72200D0A00636F6E6E42
:1008B0006563742073657276657220737563636512
:1008C0007373200D0A0000002DE9F05F05460E4607
:1008D00017469846DDE90A9A4FF0FF3442463946FA
:1008E0002846FFF75FFF0446002C00DA12E032468C
:1008F0002946204600F040F88346002C00DA09E043
:1009000052464946204600F0D3F98346002C00DACF
:1009100000E000BF002C02DB2046FFF73DFF5846F9
:10092000BDE8F09F2DE9F04107460E46144610E061
:100930004FF47A723146384602F0BEFF0546002D6C
:1009400003DC4FF0FF30BDE8F081A4F57A7406F5C2
:100950007A76B4F57A7FEBDC002C0ADD224631464C
:10096000384602F0A9FF0546002D02DC4FF0FF30AB
:10097000E9E70120E7E700002DE9F04106460F46D0
:1009800014464FF480612548EFF7C2FC24A12348A8
:10099000F7F7DCFF24B924A12048EFF7C4FC03E0FB
:1009A00021461E48EFF7BFFC20A11C48EFF7BBFC17
:1009B00021A11A48EFF7B7FC39461848EFF7B3FC06
:1009C0001FA11648EFF7AFFC1EA11448EFF7ABFCD0
:1009D00021A11248EFF7A7FC26A11048EFF7A3FCCE
:1009E0002AA10E48EFF79FFC15A10C48EFF79BFCDE
:1009F0000A48EFF7B6FC054608492BA0F7F796FF23
:100A00002A460649304602F057FF0546002D03DC12
:100A10004FF0FF30BDE8F0810120FBE7847F01202B
:100A200047455420000000002F0000002048545487
:100A3000502F312E310D0A00486F73743A20000098
:100A40000D0A0000436F6E6E656374696F6E3A2025
:100A5000636C6F73650D0A004163636570743A20BF
:100A60006170706C69636174696F6E2F6A736F6E09
:100A70000D0A0000557365722D4167656E743A204A
:100A800073746D3332663230370D0A004361636828
:100A9000652D436F6E74726F6C3A206E6F2D6361BB
:100AA0006368650D0A000000257300002DE9F04120
:100AB00080460D4614461E464FF480612E48EFF7DF
:100AC00027FC2EA12C48F7F741FF24B92DA12A4875
:100AD000EFF729FC03E021462748EFF724FC2AA181
:100AE0002548EFF720FC40212A48EFF711FC2A4661
:100AF00029A12848F7F72AFF26491F48EFF713FCDA
:100B000028A11D48EFF70FFC2BA11B48EFF70BFCAA
:100B100030A11948EFF707FC34A11748EFF703FCA1
:100B200039A11548EFF7FFFB40211A48EFF7F0FB1A
:100B300032463EA11748F7F709FF16490E48EFF76E
:100B4000F2FB17A10C48EFF7EEFB0B48EFF709FC9F
:100B5000074609493BA0F7F7E9FE3A4606494046F1
:100B600002F0AAFE0746002F03DC4FF0FF30BDE87D
:100B7000F0810120FBE70000847F0120504F535497
:100B8000200000002F00000020485454502F312E28
:100B9000310D0A0084850120486F73743A20257353
:100BA0000D0A0000436F6E6E656374696F6E3A20C4
:100BB000636C6F73650D0A004163636570743A205E
:100BC0006170706C69636174696F6E2F6A736F6EA8
:100BD0000D0A0000557365722D4167656E743A20E9
:100BE00073746D3332663230370D0A0043616368C7
:100BF000652D436F6E74726F6C3A206E6F2D63615A
:100C00006368650D0A000000436F6E74656E742D95
:100C1000547970653A206170706C69636174696FB2
:100C20006E2F6A736F6E0D0A00000000436F6E74C2
:100C3000656E742D4C656E6774683A2025640D0AE4
:100C400000000000257300002DE9F05F06460F4606
:100C500090469946DDE90ABA4A4641463046FFF7D2
:100C6000A1FD0546002D00DA19E053463A4631460B
:100C70002846FFF71BFF0446002C00DA0FE052461F
:100C800059462846FFF74EFE0446002C00DA06E0DF
:100C90002846DDE90C1200F057F8044600BF002D8D
:100CA00002DB2846FFF778FD2046BDE8F09F0000F4
:100CB0002DE9F04780460E46174600254FF4007296
:100CC0001F49404600F012F90446002C02DC681E61
:100CD000BDE8F0871A491BA0F7F728FE184800F076
:100CE0002BF9814600BF4FF400721549404600F0D1
:100CF000FDF80446124913A0F7F718FE022C04DC95
:100D000000D104E04FF0FF30E2E7002CEBDC00BF45
:100D1000002500BF00234FF400720949404602F04D
:100D2000FEF80446002C05DD701922460449EFF751
:100D3000D6FA2544002CEDDC3D604846C8E70000AB
:100D400084830120257300002DE9F04780460E467C
:100D5000174600254FF400721F49404600F0C6F8C0
:100D60000446002C02DC681EBDE8F0871A491BA06F
:100D7000F7F7DCFD184800F0DFF8814600BF4FF4BC
:100D800000721549404600F0B1F80446124913A01C
:100D9000F7F7CCFD022C04DC00D104E04FF0FF306B
:100DA000E2E7002CEBDC00BF002500BF00234FF47E
:100DB00000720949404602F0B2F80446002C05DDF5
:100DC000701922460449EFF78AFA2544002CEDDC1D
:100DD0003D604846C8E70000848301202573000079
:100DE0002DE9F04105460C46164620683060204645
:100DF00001F0EEFA07463A46294602A0F7F796FDBB
:100E0000BDE8F08125733A25730D0A00FEB54FF455
:100E10007041012004F0F0FA04463221012004F070
:100E2000EBFA0646194A1AA13046F7F78FFD02A8D9
:100E3000002341F692723146CDE900401DA0FFF734
:100E400043FD0546C82D0ED11EA0F1F705F820463A
:100E5000EFF787FA07463A4621461AA00CF030FC15
:100E600001201B490870214611A0F7F75FFD2946B4
:100E700018A0029AF7F75AFD2146012004F0AAFAB9
:100E80003146012004F0A6FAFEBD000018540020EF
:100E90002F696F742F7472616E736D69742F67653B
:100EA000745472616E736D6974436F6E6669672FF7
:100EB000257300006770752E72696E677A6C652EF7
:100EC000636F6D006465766963652E7478740000E5
:100ED000280000200D0A207265743D25642064619D
:100EE00074616C656E3D25640D0A00002DE9F843C0
:100EF00080460D4617460024002000900FE0002396
:100F000001226946404602F00AF80646002E01DC3E
:100F10000A2000909DF800202046641C2A54781E68
:100F2000A04203DD9DF800000A28E8D100202855E2
:100F30002046BDE8F88300002DE9F041044609226F
:100F400010A12046EFF738FA28B1092210A1204657
:100F5000EFF732FA90B909342078A0F130076078C1
:100F6000A0F13005A078A0F130066420784305EBAD
:100F7000850100EB41003044BDE8F0814FF0FF30C7
:100F8000FAE70000485454502F312E312000000061
:100F9000687474702F312E312000000030B585B098
:100FA0004FF400711148EFF7B3F911480068EFF7FB
:100FB000D8F9054604A80D490D4A12680023CDE969
:100FC0000025CDE9021041F692720AA10EA0FFF7AA
:100FD0003BFE0446054910A0F7F7A8FC21460FA0E8
:100FE000049AF7F7A3FC05B030BD00003478002068
:100FF0002C0000202F696F742F746573742F687430
:1010000074705465737400006770752E72696E6732
:101010007A6C652E636F6D00257300000D0A2072D7
:1010200065743D256420646174616C656E3D256462
:101030000D0A000070B505460C46224603212846DD
:1010400000F052F970BD00002DE9FE4F04468946BC
:10105000666830780007870E7942204606F0FCF873
:1010600010B92089042802D200BF00BFB9E060682F
:1010700090F800A0606890F801B0BAF1000F03D0BA
:10108000BAF1080F78D100E0A6E0012559480078B0
:1010900000F0F000E02800D10025564908684946D4
:1010A00000F058FA00B1002535B900BF00BF204656
:1010B00006F032F8BDE8FE8F00BF00BF2089082887
:1010C00002D200BF00BF8CE0204600F0EFF928B14B
:1010D00000BF00BF204606F01FF8EBE722212046A4
:1010E00006F0BAF800283BD03946204606F0B4F89E
:1010F00028B100BF40A0F7F719FC00BF75E02189B7
:101100000022022005F044FC054615B900BF00BFCF
:101110006BE000BF698907F10800814202D243A059
:10112000F7F704FC00BF2146284605F0B7FE28B1BA
:1011300000BF4CA0F7F7FAFB00BF56E06E6878429C
:1011400001B2284606F088F828B100BF4FA0F7F793
:10115000EDFB00BF49E0204605F0DEFF2C460CE029
:101160006FF02101204606F077F830B100BF47A0AC
:10117000F7F7DCFB00BF38E02BE0D4F804801D4813
:101180000068F0604E4800683061002088F8000078
:10119000A8F80200FF2030720020708139462046F6
:1011A00006F05AF820B100BF46A0F7F7BFFB0FE0EA
:1011B00001200021FF230A46CDE9010900910D49D4
:1011C000204600F01BFC05460DB100BF00BF00BF6C
:1011D00002E000BF00BF00BF00BF204605F09CFF3B
:1011E00068E7204605F098FF64E7204605F094FF85
:1011F00000BF5FE77801002069636D705F696E7002
:1012000075743A206D6F76696E6720702D3E70613F
:10121000796C6F616420746F206970206865616407
:101220006572206661696C65640A000063686563C5
:101230006B207468617420666972737420706275C3
:10124000662063616E20686F6C64207374727563CE
:1012500074207468652049434D5020686561646559
:101260007200000069636D705F696E7075743A207A
:10127000636F7079696E6720746F206E6577207078
:10128000627566206661696C65640A0069636D70E9
:101290005F696E7075743A20726573746F72696EEF
:1012A00067206F726967696E616C20702D3E706196
:1012B000796C6F6164206661696C65640A00000086
:1012C0007401002043616E2774206D6F7665206F76
:1012D0007665722068656164657220696E20706150
:1012E000636B6574000000002DE9FE4306460F465F
:1012F000904600222421012005F04AFB05461DB935
:1013000000BF00BFBDE8FE8300BF6889242802D269
:101310001AA0F7F70BFB00BFD6F8049000BF00BF80
:1013200000BF00BF00BF00BF00BF00BF00BF00BFC5
:101330006C68277084F801800020A080E0807168CC
:101340006A6802F108001C22EEF7C9FF00206080E5
:101350006989204600F0A0F86080D9F80C0002905E
:1013600001200021FF2302AACDE90010284600F049
:101370001BFB284605F0D0FE00BFC3E7636865632A
:101380006B20746861742066697273742070627572
:10139000662063616E20686F6C642069636D7020E5
:1013A0006D6573736167650070B505460C4622462E
:1013B0000B212846FFF798FF70BD000030B50246AC
:1013C0000B4600211BE001EB4100324C54F8200099
:1013D0001468A04212D101EB41002E4C04EB8000B6
:1013E00040689468A04209D101EB4100294C04EB0C
:1013F00080000089D488A04200D102E0491C032962
:10140000E1D300BF032927D1002100E0491C0329B3
:1014100006D201EB41001F4C54F820000028F5D102
:10142000032901D1002030BD01EB4104194D1068A2
:1014300045F8240001EB410405EB840490686060EA
:10144000D08801EB410405EB84042081002001EBEE
:10145000410405EB8404608143B101EB41000D4C74
:1014600004EB8000408908B10020DCE713B14FF4A1
:10147000807006E001EB4100064C04EB80004089DF
:10148000401C01EB4104034D05EB84046081481CC2
:10149000C9E700002CE3002070B504460D4629463C
:1014A000204602F0DAF9C04380B270BD2DE9F04168
:1014B000064600240027354617E06989686802F06F
:1014C000CCF90444A0B200EB1444688900EBD0715D
:1014D0004910A0EB410139B1C7F10100C7B2E0B238
:1014E000C4F3072141EA00242D68002DE5D127B17E
:1014F000E0B2C4F3072141EA0024E04380B2BDE832
:10150000F08100002DE9F0410B3020F00706104D6E
:1015100019E02068B04215D3B0420AD9871B201DBC
:10152000D4F80480EEF7DBFEA019C0E9007828604B
:1015300004E060682860201DEEF7D1FE201D2660C3
:10154000BDE8F081251D2C68002CE2D10020F7E7D2
:101550000802002018B502460092D04300B10AB933
:10156000012018BD91F8310000F0020008B90020F8
:10157000F7E74868904201D10020F2E700988B68B5
:101580001840D1E901342340984208D1886822EA02
:1015900000008C68E343984201D10120E1E700207C
:1015A000DFE700002DE9F74F8CB004468946B9F813
:1015B00028000890142004904FF0000860680B90F9
:1015C0000B9EF08801F097FC03900398C0F30C0089
:1015D0000790039800F4005006902089143880B2D8
:1015E00009900899A1F11400C11700EB5171C1F3E2
:1015F000CF010A91AAE0089814380999884201DBC2
:10160000012000E0002005900798C0F30C00069927
:1016100008430390059818B9039840F400500390CC
:10162000059808B1099801E00A98C0001FFA80FBEC
:1016300000221421022005F0ABF9054625B94FF030
:10164000FF300FB0BDE8F08F00BF6089142802DAC8
:1016500041A0F7F76BF900BF142268680B99EEF709
:101660003EFE6E6861680498084460606189049871
:10167000081A6081CDF808B03FE061890298814284
:1016800001DD029800E060898046B8F1000F01D1C9
:10169000246832E000F072F807462FB9284605F0BA
:1016A0003BFD4FF0FF30CCE760683B4602224146ED
:1016B000CDE90008032005F01DFB8246BAF1000FBA
:1016C00008D1384600F060F8284605F025FD4FF0B7
:1016D000FF30B6E7204605F0CBFE7C612648386136
:1016E0005146284605F05CFB0298A0EB080080B24A
:1016F0000290029800B1246800BF02980028BCD173
:10170000CDF81080039801F0D6FBF0800BF11401A6
:1017100088B201F0D0FB7080002070811421304627
:10172000FFF7BAFE7081D9F81430294648460E9A60
:101730009847284605F0F0FC0998A0EB0B0080B212
:1017400009900A990798084480B2079009980028E0
:101750007FF451AF00BF74E774686973206E6565EC
:1017600064732061207062756620696E206F6E65FB
:1017700020706965636521008D24010810B506207D
:1017800002F004FC10BD000010B5044600BF14B9FF
:1017900004A0F7F7CBF800BF2146062002F092FB29
:1017A00010BD00007020213D204E554C4C00000023
:1017B0002DE9F05F06460F464FF0010A756828785C
:1017C0000421B1EB201F07D000BF00BF304605F059
:1017D000A3FC0020BDE8F09F287800F00F084FF62A
:1017E000FF7000EA8808688801F085FB81467089EF
:1017F000404502DB308948450EDA7089404501DA00
:1018000000BF00BF3089484501DA00BF00BF304645
:1018100005F082FC0020DDE74946304605F08CFDEE
:1018200028695C490860E8685B4908604FF0010B73
:101830003C4600BF00BF00BF94F8310000F001003B
:1018400088B1201D78B1606868B15248006861684D
:10185000884205D04F4908682146FFF77BFE10B14A
:1018600000BF00BF0DE0BBF1000F04D04FF0000B34
:101870004A48046800E02468BC4200D12468002C77
:10188000D8D100BF84B9687A11280DD105EB0800C2
:1018900000BF00BF4188B1F5884F04D100BF00BF31
:1018A0003C464FF0000A00BFBAF1000F15D03A488D
:1018B000006890B1384908683946FFF74BFE28B9EF
:1018C0003548007800F0F000E02806D100BF00BFE6
:1018D000304605F021FC00207CE734B900BF00BF92
:1018E000304605F019FC002074E7E8884FF63F7198
:1018F000084048B100BF00BF304600F011F906466D
:101900000EB9002066E7756800BF00BF00BF00BFCA
:1019100023480760234805603946304606F0D4FC6A
:1019200068BB687A01280DD0062806D011280ED190
:10193000394630460BF09AFB20E03946304608F035
:1019400053F81BE039463046FFF77EFB16E011499D
:1019500008683946FFF7FEFD50B90E48007800F0E0
:10196000F000E02804D0756002213046FFF762FBEA
:10197000304605F0D1FB00BF00BF00BF00BF002014
:101980000749086007490860034908600149086081
:1019900000BF1FE77801002074010020080100202B
:1019A0006C010020700100202DE9FE4F05460F4616
:1019B00016469846DDE90C9A00BFE889012802D056
:1019C0000BA0F6F7B3FF00BF304600F011FC041E79
:1019D00004D100BF00BF001FBDE8FE8F4346324662
:1019E00039462846CDE9009A029400F007F8F3E75B
:1019F000702D3E726566203D3D2031002DE9F84F87
:101A000005460F4690469A46DDF828B00C9E00BF6A
:101A1000E889012802D032A0F6F788FF00BFB8F1AC
:101A2000000F43D04FF014091421284605F014FC90
:101A300028B100BF00BF6FF00100BDE8F88F6C68EF
:101A400000BF6889142802D228A0F6F76FFF00BFF4
:101A500084F808A00B986072D8F80000206148460E
:101A60004FEAE97109EB9171C1F3870141F040013F
:101A7000217084F801B0288901F01DFA60800020EF
:101A8000E0802648008801F016FAA08023480088EC
:101A9000401C224908800FB1386810B97068E060B6
:101AA00001E03868E0600020608103E06C68206934
:101AB0000090E84600BF00BF308D48B12889318DC5
:101AC000884205DD424631462846FFF76BFDB4E704
:101AD00000BF00BF42462946304673699847ACE7CD
:101AE000702D3E726566203D3D2031006368656360
:101AF0006B207468617420666972737420706275FB
:101B0000662063616E20686F6C6420737472756305
:101B1000742069705F686472000000007C0100201E
:101B20002DE9F84F804600200090D8F8045028781E
:101B300000F00F001421B1EB800F02D000BF00BFF6
:101B4000B4E0E88801F0D7F9C0F30C004FF6FF715C
:101B500001EAC00A688801F0CEF9297801F00F0186
:101B6000A0EB81001FFA80FB404605F08EF9064687
:101B70005248018888190A280CDD3146284600F0B1
:101B8000CBFA20B14D48008830440A2802DD00BF5E
:101B900000BF8BE04A48046814E06069E968884245
:101BA00009D1A0692969884205D1A089A9888842FC
:101BB00001D1012000E0002010B100BF00BF03E010
:101BC00000942468002CE8D100BF34B9314628467F
:101BD00000F0D6F9044694B968E0E88801F08BF982
:101BE000C0F30C0058B9E08901F085F9C0F30C008E
:101BF00028B11422294604F10800EEF770FB2F48A3
